:020000040000FA
:1000000000F80202F94600002D11000099130000CB
:1000100000000000000000000000000000000000E0
:1000200000000000F0020100380301002D11000063
:1000300000000000000000002D110000F949000040
:10004000AD0D00002D1100002D110000AD47000086
:10005000912200005D420000BD1000005D11000013
:10006000090C0000450B00002D11000031110000AB
:10007000D11D00007956000099460000C5460000D9
:100080003D4300002D1100002D110000214A000009
:10009000414A00002D1100002D1100002D1100001B
:1000A000E14F0000EB4F0000AF0D0000AD45000038
:1000B0002D110000C54200000000000000000000FB
:1000C0000348854600F00EFD004800476D9600008D
:1000D00000F8020230B50B46014600202022012420
:1000E00009E00D46D5409D4205D31D469540491B6C
:1000F0002546954040191546521E002DF1DC30BDB5
:1001000070B500242546002801DA01244042002968
:1001100001DA01254942FFF7DDFFAC4200D0404241
:10012000002C00D0494270BD0549064A086850437A
:10013000054A801808604008704701490860704708
:10014000089001026D4EC6413930000003460B4352
:100150009B0703D009E008C9121F08C0042AFAD27D
:1001600003E00B780370401C491C521EF9D2704703
:10017000D2B201E00270401C491EFBD2704700223F
:10018000F6E710B513460A4604461946FFF7F0FF96
:10019000204610BD421C0178401C0029FBD1801A6A
:1001A0007047F8B502464A40D40F42004B0052084F
:1001B0005B089A4202D20246084611464A0023D002
:1001C000C30D4A00DDB2120EAD1A202D35DA4902F8
:1001D0000126490AF6058A19002C00D05242202136
:1001E0004F1B1146B9402A411018C20D9A4221D026
:1001F000002C17D0012D08DCDA05801AD20F8019E7
:10020000D207DBB200F0D6FBF8BDDA05801A012375
:1002100040001B06C01880185A428018CA0F1043AD
:10022000490007E04908C2071143DA05801A80191E
:100230004008801800F0B6FBF8BD61000122511A99
:10024000001BF7E70122D2075140AAE70122D2079B
:100250005040A6E7024670B54A40D30FDB07400086
:100260002DD04A002AD0010E140E000212020919E4
:10027000400A520A8418E50104465443000A120A4F
:100280002E045043A4194219200CC543AA18120C7D
:100290000125AD03521C521912047F39240400D0E9
:1002A000521C104301D44000491EC2B20C06C009C2
:1002B0002018401C4008802A02D003E0002070BDB6
:1002C00040084000002900DA0020184370BD70B5D6
:1002D00002464A40D50F40004A00ED074008520848
:1002E000002814D0002A12D0C40DD30D41020120E1
:1002F000C0055202490A520AE41A091812187D343C
:10030000914201D3641C00E04900002C01DA002076
:1003100070BD0023914201D3891A0343400849006C
:100320000028F7D100290AD0914202D10121C90742
:1003300005E0914201D2012101E00121C943E0051C
:10034000C018401900F02EFB70BD0000F0B5074644
:100350000846584087B0C00F049048000E46590028
:1003600040084908BC1A884105D2384631461E4625
:1003700017460B4602465800400810434CD0300D3B
:10038000039040055900400D490D0590401A029018
:10039000402872DA18030121000B09050843019077
:1003A00004980092002805D001995242002088410B
:1003B00000920190029840210A1A0199009800F0D9
:1003C000BDFA05460C466B4607CB00F0D8FAC019BB
:1003D0007141039A0E0D0023D71756401A467A40F2
:1003E000164344D0049A002A2DD0029A012A039A77
:1003F00015DC1205C01A914101263605001C714119
:10040000D20F059ED2070093019202962A462346F8
:1004100000F016FB07B0F0BD38463146FAE7160586
:10042000224A0F46B218C01AB74101210905001C23
:100430004F4100187F41114618187941E20F1043CF
:100440006D19644113E0E2076D0815436408C207A3
:100450001443039A01261205C01A91413605001C67
:100460007141CE07400830434908C01851412A461F
:10047000234600F0D8FACDE7FFE7049801224000B8
:10048000C117121A00238B4104983146C417381A39
:10049000A141EEE730B40124E407634030BC55E7E6
:1004A00030B40124E407614030BC4FE70000E0FFB6
:1004B000F0B51FB488B00B990998002448400999F9
:1004C000C00F490049080991C0070B9900904900E5
:1004D00049080B9109990898A64608431CD00B9926
:1004E0000A98084318D0099801244000420D48009A
:1004F000410D099824050003000B204309900B9837
:100500000003000B20430B9050181C494018002298
:1005100001901446104605E0002001460DB0F0BDE4
:10052000032801DA034600E003239C46C11A0AAE01
:100530000AE05F0008ADED5B4F00F75B7D430027ED
:10054000AA187C41491C5B1E6145F2DD410004ABE9
:100550005A522104120C0A43240C401C0828DFDBE9
:10056000019802900099704601910090059B049AB1
:100570000799069800F064FAD0E700000DFCFFFF31
:10058000F0B50C465C4085B0E40FE40703944C00E2
:100590000026640859009446490802460296224300
:1005A00021D062460A431ED06200570D4A000E0356
:1005B0002303550D012402462C492405781B1B0BEF
:1005C000360B401823432643614600901C46501AC0
:1005D000B44103D30098401C009002E092180098A8
:1005E0005B41002803DA0020014605B0F0BD002081
:1005F000012109050746864611E064461D46141B85
:10060000B54106D36546521BB341744607430C43BC
:10061000A646CD0740084908284392185B41054685
:100620000D43EAD11046184313D060461946504096
:100630007140084306D06046101AB34106D2012229
:10064000002306E000220123DB0702E00122D2435F
:100650005310009874460105381C6141029C039DAB
:100660000019694100F0DFF9BFE70000FD03000059
:100670000122D207002800DB101A002900DB511AE2
:10068000814201D801207047002070470122D20723
:10069000002800DB101A002900DB511A814201D228
:1006A00001207047002070470122D207002800DB9C
:1006B000101A002900DB511A814201D30120704732
:1006C000002070470122D207002800DB101A002901
:1006D00000DB511A814201D9012070470020704788
:1006E0000122D207002800DB101A002900DB511A72
:1006F000814201D1012070470020704710B50029C8
:1007000004DB0C460121C9074042A141002B04DB58
:100710001C460123DB075242A341101A8B4101D230
:10072000012010BD002010BD10B5002904DB0C46CF
:100730000121C9074042A141002B04DB1C460123D3
:10074000DB075242A341801A994101D2012010BD1A
:10075000002010BDC217C10F504010B54018CA0785
:100760009623002100F026F910BD10B50022962333
:10077000114600F01FF910BD0EB5C217C10F504051
:10078000CA0740180021054B0293019200910A46C6
:100790000B4600F055F903B000BD00003304000023
:1007A0000EB505490291002100910A460B460191C0
:1007B00000F046F903B000BD330400003EB5CA178F
:1007C000CB0F002450405140C0186141DA07054B5F
:1007D0000293019200942246234600F031F903B0BF
:1007E00030BD000033040000C20F4100400201236D
:1007F000400ADB05D207090EC0187F2901DA002064
:100800007047962903DC9623591AC84001E09639AF
:100810008840002AF4D04042704741004002012243
:10082000400AD205090E80187F2901DA002070479E
:10083000962903DC9622511AC840704796398840A1
:100840007047000070B5CD0F4A0009030123090B62
:100850001B0519430B4BED070024520D9A4201DA98
:10086000002070BD074B34339A4203DC9A1A00F023
:1008700075F802E00449511888402C43F1D04042F9
:1008800070BD0000FF030000CDFBFFFF70B5CD0F72
:100890004A0009030123090B1B0519430D4BED0702
:1008A0000024520D9A4202DA0020014670BD094B25
:1008B00034339A4203DC9A1A00F050F803E0064BF6
:1008C000D21800F03BF82C43F0D0002240428A417D
:1008D000114670BDFF030000CDFBFFFFC20FD20722
:1008E000400040080BD0C10D0723DB01C9184002AE
:1008F0000905400A1143C208400711437047002010
:1009000001467047CB0FDB07490010B54908024686
:100910000A4307D00A0D07240903E401090B121B3F
:10092000002A01DC002010BDC900440F0C43C100A7
:10093000E018D205801800F035F810BD10B5202A57
:1009400004DB0146203A9140002010BD9140202355
:100950009C1A0346E3401943904010BD10B5202A6D
:1009600004DB0846203AD040002110BD0B46D3409E
:10097000D0402024A21A91400843194610BD10B55A
:10098000202A06DBCB170846203A1041C1170B433B
:1009900006E00B461341D0402024A21A91400843A0
:1009A000194610BD002904DA401C490001D1400855
:1009B0004000704770B40024050C05D110240004D9
:1009C00002D1002921D01124050E01D100020834E2
:1009D000050F01D10001241D850F01D18000A41C49
:1009E000002801DB4000641C002908D020252E1BB4
:1009F0000D46F540A14000D00121294308430106DE
:100A00001B1B000ADB1D02D5002070BC7047DB05F4
:100A1000181880180029F8DA401C4900F5D170BC7C
:100A200040084000704710B5002B08DA0024401C35
:100A3000614192185B411A4301D14008400010BD4A
:100A4000F0B51FB482B005460C0003D008460DF087
:100A5000BFFB02E00DF0BCFB2030024600902146B7
:100A60002846FFF76BFF049B059A04460F46184380
:100A70001143084314D0184610431BD0009840215E
:100A80000A1A18460599FFF769FF05460E46009AAF
:100A900005990498FFF752FF084305D0012004E0B0
:100AA0002046394607B0F0BD0020C11705430E436C
:100AB0002C43374300990E986305401A7905E40AE0
:100AC00000220C43FD0A0A3002D500200146E9E766
:100AD0000105101969410C9C0D9D00196941FFF732
:100AE000A2FFDFE7064C0125064E05E0E36807CCD0
:100AF0002B430C3C98471034B442F7D3FFF7E4FA89
:100B000080FD0000A0FD000030B58C180278401C6C
:100B100013071B0F01D10378401C120906D102787C
:100B2000401C03E005780D70401C491C5B1EF9D188
:100B300001E00B70491C521EFBD1A142E6D30020FC
:100B400030BD000010B52148016A8A0715D44A0754
:100B500015D4C90732D01E498A89002A15D0531EE0
:100B60008B8182688C6904C48C610A691B040DD076
:100B7000002A22D10121016010BD022100E00421E0
:100B8000C16113488021416110BD0A69012A09D160
:100B9000026801239A430260C361FF2068309930E4
:100BA0000C4A106001204861CA69002A05D0886992
:100BB00009898B00C01A904710BD10BDFF22683212
:100BC000054806A109A30BF0CDF8C04608D00140A6
:100BD0005895010280E200E008ED00004144435FC7
:100BE00049525148616E646C65720000556E6578BB
:100BF0007065637465642041444320696E74657256
:100C0000727570740D0A000070B582B000230193F4
:100C1000444801688A6A4C6813252540132D02D187
:100C2000CB689B07DB0F4361930772D453070AD449
:100C3000D30711D1130724D5048F838E1C1B102CCE
:100C40000EDD102310E0042088620220032142A25E
:100C50000CF0E4F802B070BD0120886202B070BDF3
:100C6000048F1B1B1C0610D0DBB20024058FC66A44
:100C700075192D5D0D74641CA342F7D1048FE31820
:100C80000387D20607D400212FE04B6A0824A34330
:100C90004B62D206F7D5CB68C28E448F141B5B041F
:100CA000DB0EA34201D3438FD31ADAB2002A16D047
:100CB000097D438F046BE1540199012A10D001236F
:100CC0001C46890145582D7D41184E8F9B19096B93
:100CD000CD54641CE3B201999A42F2D800E000219D
:100CE0008B01C3185C8FA2185A878A0181184B8F19
:100CF000CC8EA3420BD301230B61805800224262A9
:100D0000CA6B002A03D03A31098801A8904702B083
:100D100070BD02208862044804A1084A08A30BF0B1
:100D200021F8C0464090010221ED00004145535F8B
:100D300049525148616E646C65720000CE02000039
:100D400041455320696E707574206F766572666CCC
:100D50006F770D0A00000000414553206F757470D5
:100D6000757420756E646572666C6F770D0A00008D
:100D700080B58AB008200790642006900948039047
:100D8000022001904B20C0010990074814300590C3
:100D90000120029080020490032001A904F02AF9A6
:100DA0000AB080BDA0AA01028C970102704770476B
:100DB000F0B581B001220092D303494A012918DB22
:100DC0004118002503E0ADB2401C884212D2009CBD
:100DD00026020778BE1904E03D4674001E422646EE
:100DE000F1D16F003406E40FE7191D42F4D05740EB
:100DF000F2E7002568001D4230D14100184231D190
:100E00004800194232D14100184233D148001942FA
:100E100034D14100184235D14C00194236D160001E
:100E20001C4237D10104C90B184238D1480019427D
:100E300039D1410018423AD1480019423BD1410012
:100E400018423CD1480019423DD1410018423ED1E0
:100E5000480019423FD180B201B0F0BD504041007E
:100E60001842CDD0514048001942CCD050404100EA
:100E70001842CBD0514048001942CAD050404100DE
:100E80001842C9D051404C001942C8D054406000AB
:100E90001C42C7D050400104C90B1842C6D0514073
:100EA00048001942C5D0504041001842C4D05140BA
:100EB00048001942C3D0504041001842C2D05140AE
:100EC00048001942C1D0504041001842C0D05140A2
:100ED00048001942BFD0504080B201B0F0BDC046BA
:100EE00021100000F0B58BB00C205949085EFFF7C7
:100EF00043FC0690059157484069FFF7EFFC0490CA
:100F00000391012358020190534802880026534957
:100F10000A93029207E049005E4B58524F49761CF3
:100F2000162E00D191E0B318C85C0528F7D10893BC
:100F3000B7004B4AD1594B4C21624B4DE8592063C5
:100F4000D219136BA361EA19126BA2620025591A18
:100F500007912164636AE16999410A9B00DB2B4692
:100F6000002B01D0019BC9183E4C6164E36A616BA0
:100F7000801A99410A9A00DB2A46002A09962C46D3
:100F800001D0019A8918FFF719FC05460E4637482B
:100F9000C059FFF7F1FB049A039BFFF7F1FA0246F1
:100FA0000B4620463249FFF775FA2A463346FFF7CB
:100FB0007FFAFFF76BFC2B4FB863F9630799401A70
:100FC000C10F401840103860FFF7D6FB294A2A4B62
:100FD000FFF76EFAB864F964284A294BFFF768FAFC
:100FE00027462246274BFFF763FA2246264BFFF798
:100FF000ADF905460E461B4805614161284622466B
:10100000224BFFF77BFB0446401E844128463146B5
:1010100007973A461E4BFFF787FB0746401E87415E
:10102000274028463146069A059BFFF78FF9FFF7C0
:1010300009FC002F01D10798C043002F029A099E96
:10104000089900D067E7314665E70BB0F0BDC046B0
:1010500042A60102FCE2000018970102B4C5010299
:1010600004980102F095010264980102389D010282
:101070000000F03F699006699006903F52257997ED
:10108000532ED33F0000594000003E40006AF84014
:1010900000408FC094C20102002909D000220378C9
:1010A000D3189AB2401C491EF9D1D84380B2704778
:1010B000014880B27047C046FFFF0000B0B582B063
:1010C000194C2068056801A90020087007E09047C6
:1010D0000198401C01A90870C0B2082822D2012240
:1010E00011048140294209D02268516080002018F3
:1010F000826A002AECD001A80121E8E713028340AC
:101100002B4201D0022104E082402A42E0D0032198
:10111000134622685360800020188268002AD7D0C6
:1011200001A8D4E702B0B0BD90920102FEE7000032
:1011300010B509480168CA6920231343CB610269CD
:10114000032A08D1012293050C689C430C605102CC
:10115000C26E0A43C26610BD00930102F0B581B0B1
:101160005C4C2068856BE80707D0E168002904D053
:1011700000208847206801218163A80707D52169DD
:10118000002904D001208847206802218163680774
:1011900007D56169002904D002208847206804210E
:1011A0008163280707D5A169002904D00320884757
:1011B000206808218163E80607D5E169002904D089
:1011C00004208847206810218163A80607D5216A7A
:1011D000002904D005208847206820218163680603
:1011E00007D5616A002904D006208847206840217D
:1011F0008163280607D5A16A002904D00720884703
:101200002068802181630126E80507D5E16A00296D
:1012100004D037020820884720688763A80507D5CF
:10122000216B002904D07702092088472068876352
:10123000680507D5616B002904D0B7020A208847EA
:1012400020688763280507D5A16B002904D0F70221
:101250000B20884720688763E80407D5E16B0029E5
:1012600004D037030C20884720688763A80407D57B
:10127000216C002904D077030D20884720688763FC
:10128000680407D5616C002904D0B7030E20884795
:1012900020688763280407D5A16C002904D0F703D0
:1012A0000F20884720688763E80307D5E16C002991
:1012B00004D037041020884720688763A80307D527
:1012C000216D002904D075041120884720688563AA
:1012D00001B0F0BD80930102F0B581B000910646E7
:1012E000C7680468A01C3946FEF7F4FE0025706844
:1012F000814201D1ED430BE0601C3946FEF7EAFE66
:10130000316032695143B06808180099FEF71EFF3A
:10131000284601B0F0BDB0B5012400250560446049
:1013200008300EC0B0BD02460020002A04D0106074
:1013300050609060D1607047C043704706480168B4
:10134000491C01600548416802680023521C026084
:101350004B4143607047C0469CA80102A0A801020F
:1013600070B505460C2058430024904211D2121A41
:10137000461829606860AE60EA6028461030194659
:10138000FFF7D1FFE96820352846FFF7CCFF20465C
:1013900070BDE443204670BD04217046084204D06D
:1013A000EFF30983EFF3088203E0EFF30883EFF331
:1013B00009829BB004A8F0C044464D4656465F469D
:1013C00008A8F0C01846F0C86846F0C018690C902C
:1013D000202018440D9058690E9098690F90D86994
:1013E0001090EFF310801190EFF3148012900949E0
:1013F000086813900849086814900849086815900F
:101400000749086816901793189270461990684615
:101410000AF0C2FE04ED00E00CED00E010ED00E08B
:1014200014ED00E0F0B581B00326002430462146DB
:1014300007F054F904252846214607F04FF9012703
:10144000304639463A4607F0DBF830462146324608
:1014500007F06CF9284639463A4607F0D1F80221E0
:101460002846224607F062F901B0F0BDF0B589B018
:1014700008900425284607F0ABF80A27384605F0FF
:10148000BFF8284607F0B4F80324204607F0A8F870
:1014900007900526304605F0B3F8284607F098F87F
:1014A000384605F0ADF8284607F0A2F8204607F0C8
:1014B00097F80690304605F0A3F8284607F088F81C
:1014C000384605F09DF8284607F092F8204607F0C8
:1014D00087F80590304605F093F8284607F078F82D
:1014E000384605F08DF8284607F082F8204607F0C8
:1014F00077F80490304605F083F8284607F068F83E
:10150000384605F07DF8284607F072F8204607F0C7
:1015100067F80390304605F073F8284607F058F84E
:101520003846019705F06CF8284607F061F8204628
:1015300007F056F80290304605F062F8284607F0AA
:1015400047F8384605F05CF8284607F051F8204681
:1015500007F046F80746304605F052F8284607F0EF
:1015600037F8019805F04CF8284607F041F8204676
:1015700007F036F80446304605F042F8284607F0F2
:1015800027F80699481E81410A460799481E81415D
:10159000480080188000059A511E8A415100401869
:1015A000049A511E8A4180188000039A511E8A4174
:1015B00051004018029A511E8A4180188000791EFD
:1015C0008F4179004018611E8C4106190898002847
:1015D00003D0032006F0FCFF02E0032007F008F828
:1015E0000A24204605F00CF80425284607F000F8E8
:1015F000204605F005F8284606F0EAFFF0B209B0EB
:10160000F0BD70B50446042006F0E2FF60B2002889
:1016100003D4032006F0DCFF02E0032006F0E8FF1D
:101620000A25284604F0ECFF0426304606F0E0FFC9
:10163000284604F0E5FF304606F0CAFF284604F0CD
:10164000DFFF600603D4032006F0C2FF02E00320A0
:1016500006F0CEFF0A25284604F0D2FF04263046C5
:1016600006F0C6FF284604F0CBFF304606F0B0FF78
:10167000284604F0C5FFA00603D4032006F0A8FF07
:1016800002E0032006F0B4FF0A25284604F0B8FF64
:101690000426304606F0ACFF284604F0B1FF304681
:1016A00006F096FF284604F0ABFFE00603D40320C3
:1016B00006F08EFF02E0032006F09AFF0A25284676
:1016C00004F09EFF0426304606F092FF284604F000
:1016D00097FF304606F07CFF284604F091FF200774
:1016E00003D4032006F074FF02E0032006F080FF1D
:1016F0000A25284604F084FF0426304606F078FFC9
:10170000284604F07DFF304606F062FF284604F0CC
:1017100077FF600703D4032006F05AFF02E003209E
:1017200006F066FF0A25284604F06AFF04263046C4
:1017300006F05EFF284604F063FF304606F048FFDF
:10174000284604F05DFFA00703D4032006F040FF05
:1017500002E0032006F04CFF0A25284604F050FF63
:101760000426304606F044FF284604F049FF304680
:1017700006F02EFF284604F043FFE00703D10320C4
:1017800006F026FF02E0032006F032FF0A2420467E
:1017900004F036FF0425284606F02AFF204604F010
:1017A0002FFF284606F014FF204604F029FF70BDE5
:1017B00070B50446042006F00BFF60B2002803D485
:1017C000032006F005FF02E0032006F011FF0A25C2
:1017D000284604F015FF0426304606F009FF284687
:1017E00004F00EFF304606F0F3FE284604F008FF32
:1017F000600603D4032006F0EBFE02E0032006F0AF
:10180000F7FE0A25284604F0FBFE0426304606F0C3
:10181000EFFE284604F0F4FE304606F0D9FE2846D6
:1018200004F0EEFEA00603D4032006F0D1FE02E091
:10183000032006F0DDFE0A25284604F0E1FE04261A
:10184000304606F0D5FE284604F0DAFE304606F0B3
:10185000BFFE284604F0D4FEE00603D4032006F0C1
:10186000B7FE02E0032006F0C3FE0A25284604F076
:10187000C7FE0426304606F0BBFE284604F0C0FE34
:10188000304606F0A5FE284604F0BAFE200703D431
:10189000032006F09DFE02E0032006F0A9FE0A25C3
:1018A000284604F0ADFE0426304606F0A1FE284688
:1018B00004F0A6FE304606F08BFE284604F0A0FE9B
:1018C000600703D4032006F083FE02E0032006F045
:1018D0008FFE0A25284604F093FE0426304606F0C3
:1018E00087FE284604F08CFE304606F071FE28463E
:1018F00004F086FEA00703D4032006F069FE02E090
:10190000032006F075FE0A25284604F079FE042619
:10191000304606F06DFE284604F072FE304606F0B2
:1019200057FE284604F06CFEE00703D1032006F0C2
:101930004FFE02E0032006F05BFE0A24204604F07E
:101940005FFE0425284606F053FE204604F058FEAC
:10195000284606F03DFE204604F052FE70BDF0B56C
:1019600081B003260025012430462946224606F090
:1019700047FE304606F03CFE0626304604F040FEA8
:10198000042006F035FE304604F03AFE032006F04F
:1019900027FE00281BD0681CFA2D0546F6D3042527
:1019A000284606F015FE0326304606F011FE0A27EB
:1019B000384604F025FE284606F01AFE304606F0AA
:1019C00017FE384604F01CFE204601B0F0BD03208F
:1019D00001210A4606F014FE042006F0F9FD002459
:1019E000204601B0F0BDF0B581B0032600250124EA
:1019F00030462946224606F003FE304606F0F8FD42
:101A00000626304604F0FCFD042006F0F1FD3046C9
:101A100004F0F6FD032006F0E3FD002820D0681C4A
:101A2000FA2D0546F6D30426304606F0D1FD0325EF
:101A3000284606F0CDFD0A27384604F0E1FD304681
:101A400006F0D6FD284606F0D3FD384604F0D8FD52
:101A500028462146224606F0D3FD204601B0F0BDBF
:101A6000032001210024224606F0CAFD042006F0CE
:101A7000AFFD204601B0F0BDF0B583B000AC0EC4A0
:101A800007460324204606F0B3FD0425284606F049
:101A9000AFFD204606F09CFD0A26304604F0B0FD5E
:101AA000284606F095FDFE2007403846FFF780FEE9
:101AB000FFF799FF134F38600098FFF779FEFFF7A3
:101AC00092FF78600198FFF773FEFFF78CFFB86014
:101AD0000298FFF76DFEFFF786FFF860284606F0D4
:101AE00077FD204606F074FD304604F089FD284657
:101AF00006F07EFD204606F07BFD304604F080FDBA
:101B000003B0F0BD9495010270B504464D4E30709F
:101B100001202040707003D1032006F059FD02E03F
:101B2000032006F065FD0825284606F061FD2846DD
:101B300006F04EFDA007C00F707003D1032006F021
:101B400047FD02E0032006F053FD0825284606F075
:101B50004FFD284606F03CFD6007C00F707003D1B2
:101B6000032006F035FD02E0032006F041FD0825C4
:101B7000284606F03DFD284606F02AFD2007C00F46
:101B8000707003D1032006F023FD02E0032006F06D
:101B90002FFD0825284606F02BFD284606F018FDE7
:101BA000E006C00F707003D1032006F011FD02E0C3
:101BB000032006F01DFD0825284606F019FD2846DD
:101BC00006F006FDA006C00F707003D1032006F0DA
:101BD000FFFC02E0032006F00BFD0825284606F076
:101BE00007FD284606F0F4FC6006C00F707003D1B4
:101BF000032006F0EDFC02E0032006F0F9FC0825C6
:101C0000284606F0F5FC284606F0E2FCE009707074
:101C100060B2002803D4032006F0DAFC02E00320BF
:101C200006F0E6FC0824204606F0E2FC204606F01A
:101C3000CFFC0724204606F0DBFC204606F0C8FC5B
:101C400070BDC04690950102B0B503F093F902242F
:101C5000204606F0C5FC0E4DA871204606F0C0FCDB
:101C60000C494A78002802D0002A08D0B0BD012AC9
:101C7000FCD101208870002048702872B0BD00207F
:101C8000E87101224A701E228A702872B0BDC046D7
:101C9000289901021890010270B5072400252046FA
:101CA000294606F01BFD0126204631462A4606F04D
:101CB000A7FC05222046314606F038FD70BDF0B580
:101CC00081B007460324204606F092FC04252846EE
:101CD00006F08EFC204606F07BFC0A26304604F017
:101CE0008FFC284606F074FC3220FFF78AFCFFF7D1
:101CF00036FEF8B2FFF785FCFFF731FE204606F00E
:101D000077FC284606F074FC204606F061FC30465D
:101D100004F076FC284606F05BFC3320FFF771FCEC
:101D2000FFF71DFE0020FFF7A1FB0746284606F03F
:101D30004FFC204606F04CFC304604F061FC28467F
:101D400006F056FC204606F053FC304604F058FCE2
:101D5000384601B0F0BDF0B581B0009107460324CC
:101D6000204606F045FC0426304606F041FC20469D
:101D700006F02EFC0A25284604F042FC304606F008
:101D800027FC3220FFF73DFCFFF7E9FDF8B2FFF733
:101D900038FCFFF7E4FD0098FFF733FCFFF7DFFDA9
:101DA000304606F015FC204606F012FC284604F0EA
:101DB00027FC304606F01CFC204606F019FC28469D
:101DC00004F01EFC284604F01BFC01B0F0BD00002E
:101DD00080B5074801210170064802680A43026085
:101DE00005480268002A02D000200146904780BDC5
:101DF000A2AE01021C100050A4AE0102F0B58BB0DF
:101E0000C54DE879002800D1FBE1012630460CF0F1
:101E100047F90CF0E9F8C14C60780BF0E1FEC049DD
:101E20008A8809A882800A88498809048918099142
:101E300007F0B0FD61780529324600D00222B9488A
:101E4000092900D080184179F74C2078621C0BF0EA
:101E50008BFF607A09F056FA3046314608F064FE8E
:101E6000F248F34907F08EF8F24C03202070F24854
:101E70000088A070698C2171000AE070080A607106
:101E800006212046FFF708F9A07108A90880002163
:101E9000E9732E72000AE071C320870108F040FE4A
:101EA0000397C319AB640A21204632460CF01AF995
:101EB0002864AE6C08F0CAFD801909F085FB06465F
:101EC0000F46D948007B09F00BFA81B2C90B4018C4
:101ED00000B2C1174010D94A3018106179415161E0
:101EE00008F01EFE286306F0BDFF0028FBD1EFF3CB
:101EF000108072B600242046214605F0B7FA2F461E
:101F00002837CF4E02230294204631463A4605F048
:101F100031FC7D2080000490288DCA49884219D068
:101F2000512002033C462F463546002630462946BE
:101F300005F0F6F9049804F05CFB022330462E46C7
:101F40003D4627463146224605F014FCBD49288D02
:101F50008842E5D162B62F46BB4D19E00196EFF3FA
:101F6000108072B66C26C14F38463146FEF720FF0E
:101F700008A90880F888698D814200D187E062B69F
:101F8000019EB14D2888A74F798D814200D1CBE0C9
:101F9000012006902E460CF083F80520A54C2070F9
:101FA000A5480088A070798C21717A8DA271000AF1
:101FB000E070080A6071100AE07108212046FFF7FE
:101FC0006BF8207208A908803D46029F2F74000A12
:101FD0006072688D6421059148433188FEF77AF874
:101FE000C3B20320014699A20AF018FF38460CF04C
:101FF000D9F808F095FD03994318AB640C212046ED
:10200000069A0CF06FF82864AE6C08F01FFD80197A
:1020100009F0DAFA06460F468348007B09F060F9BA
:1020200081B2C90B401800B2C11740103018834A62
:1020300010617941516108F073FD286306F012FFC9
:102040000028FBD108F06CFD6863A86C8349401838
:10205000E864002630463146814A0BF0F7FF2864D9
:1020600006F000FF0028FBD1E87A0128059C00D18A
:1020700074E7049804F0BDFA687C401C6874C0B230
:10208000142800D3BFE001200CF00AF879E7B85B10
:1020900008A90988814200D071E7B8886649098893
:1020A000814200D06BE77888698C814200D066E776
:1020B00000263046314605F0D9F9394608316C4FD3
:1020C00038462246FEF742F8688D60435C49411865
:1020D000009630463A46234605F024FE06460004A4
:1020E0000ED0688D60435649411800203A46234679
:1020F00005F018FE06460A2004F07BFA3004F0D101
:10210000300400D03BE700986874688D401C6885F7
:102110000A2004F06EFA32E704970102829001026D
:1021200034E20000D09D01029920424C20704248C8
:102130000088A070798C2171000AE070080A607133
:1021400006212046FEF7A8FFA07108A90880FE73AB
:102150003D46069F2F72000AE071032045A201460A
:102160000AF05CFE08F0DCFC03994318AB640A211A
:1021700020463A460BF0B6FF2864AC6C08F066FCCB
:10218000001909F021FA04460E462748007B09F0A1
:10219000A7F881B2C90B401800B2C117401020182F
:1021A000264A10617141516108F0BAFC286306F0BB
:1021B00059FE0028FBD107A8334901800025284695
:1021C000294605F053F93A03304C2846214605F0DC
:1021D000A7F80004049D05D1002007AA0223214688
:1021E00005F0A0FDEFF3108072B6284604F001FA66
:1021F000BFF34F8F1B481C490160BFF34F8F00BFD7
:10220000FDE70BB0F0BD6E856E74049804F0F1F933
:10221000BFF34F8F134814490160BFF34F8F00BFC6
:10222000FDE7C04604970102829001022DD0000014
:1022300095B900000EB6010250990102C89801023A
:1022400000F00204FFFF00003CA60102C9FDBCB67D
:10225000BDF8B6C825640D0A00000000200C01007E
:1022600050C300000CED00E00400FA0578B501024F
:10227000949B0102D5FDD4DAB7A2CBCDD7EEBAF349
:10228000D2BBB0FC0D0A0000DDDD000000F0070449
:10229000F0B599B0F548017BC67A427B0E92F44CBA
:1022A000221F1368F34A1268069242780C92027950
:1022B0000592C76A04931F4001200F907A0200D54F
:1022C000BCE03A0200D5BFE0FA0102D50F98020641
:1022D0002260502508968A191826BB0102D50F984E
:1022E000430623604123079569430A9635465543C3
:1022F0001426FC0210D50F98040538463746DC4EEC
:102300003460DA4CA469B464D84CE4697464DA4C7F
:10231000241D34603E46074690000B90D8040D9073
:10232000681809900E9B73430F988203B902D04D31
:1023300022D50F9841052960CC480E9616460246D4
:1023400081692965C169696509990D9801430898F2
:10235000000108180B994018C018C84909889279DB
:102360004A4380180A301C4604F0D6FC2346324605
:102370000E9EC04988672A600F98C404380300D5B0
:102380002C60F80302D50F98000428600F984104D0
:10239000B80300D52960380400D4E4E10394029125
:1023A0000E9308920D980B990C180A980C994143BA
:1023B0000C910F98C0030B90286007F015FB0028C4
:1023C00001D004F08BFC0C98005B410B43D10998C1
:1023D00000190E9940180599090140180E90E74D13
:1023E000287B079B4343E97A0A010D9C2243D218BC
:1023F00041188B00D2180A9B4B43D1186A7B564375
:1024000089190E9E2A791018DF4A128842438818CB
:1024100016903068C000800D10A9C8820025119563
:102420007079C0077ED110A80F998182069C009414
:102430000020E8A2049B0AF0F1FC78E00F988205E6
:1024400022603A0200D43FE70F98C2052260FA01E9
:1024500000D53BE73DE70721490308400321490335
:102460008842089A00D07EE1069706F051FF0020CE
:10247000169009901590C14CE07A217B08180A99B2
:10248000414380000D9A10434118627B0E967243BF
:102490008A186178A379079E7343D718FA683F2694
:1024A000324063789A420C976ED105960A9A4A4355
:1024B00080580F210A0702400398401EC04B1B683A
:1024C000DB090340981810900F98C0020B90B86871
:1024D000800767D42C46283C09F016FC0546206886
:1024E000000609D5C3208401786A400704D409F0A6
:1024F0000BFC401BA042F7D905980002B9684908B7
:102500000140B34803688268B868C40C20202040AA
:10251000DB0700D095E0002310221D461C460E9ECE
:102520000B9FB1E010A88582B0681190069C701DC9
:10253000924B1979E20707D1491C1971D97A1A7996
:102540008A4202D31D7100E0D970017842781202EC
:102550005118827812048918032291430170357151
:102560005878401C5870D87A197B081859788842D6
:1025700000D85D70D879401ED871596B002901D000
:1025800010A888477E4DEDE010A80B998182F8686D
:1025900030406378009000207CA20F990AF03EFC46
:1025A0000E9E94E0388A874A024010A8C2822022F8
:1025B000BA5C9307DB0F3C68C3720F9B1A408272B0
:1025C0006205D20C0D9B1A431692FA68130E037221
:1025D000BB69FC697C4D2D682D0C05745204920F6B
:1025E000427211931394654CA07B002809980E9EAB
:1025F0000B9F5FD075480068007A0328099859D06E
:102600000C98007D08400928099853D1C320840103
:1026100009F07AFB05460C98406A41070BD45949EA
:1026200009680906890F06D109F06EFB401BA0421C
:10263000F1D90C98406A41030898884310A9888210
:1026400037E0D2070E9E0B9F03D1082300221546C8
:1026500019E00C9B9A68029C224211D19A68520C94
:10266000022494430022134615460DE0ACB001024B
:1026700028A000503CA10050FC1F0000A8B001029F
:1026800004250022134614460843104318432843E8
:10269000204310A9888238420BD10C9B198A494AE1
:1026A0000A4010A9CA8219684905C90C0D9A11433C
:1026B0001691324C2921615C002908D03037B8428C
:1026C00005D010A908461130123108F01FFEE77A34
:1026D0002A48047BE519294800790E90274840785C
:1026E000401C2946FDF7F6FC88000D9A104318900F
:1026F000079961433801104340182049497B4E43F4
:1027000080191C21694340180E9909191B4B1E4A58
:1027100012884A4380181790099A0C998A60987B0E
:10272000002800D04A629879401C9871187B9979EA
:102730008142069F00D39A715978491C5970D97A01
:102740000818597888420E4D00D85A70187A401EE1
:1027500018722820185C002804D0996B002901D039
:1027600010A88847089A174202D00F9800032860E3
:102770001C480449486019B0F0BDC046ACB0010225
:1027800028A000503CA10050A8B0010248572045A5
:10279000542069647820256420616E6420455420AB
:1027A00069647820256420696E205258206465731E
:1027B00063206D69736D617463680D0A0000000029
:1027C00038200040FF03000094300040EC930102E9
:1027D000604000404D414320455654202578202537
:1027E000780D0A00FFFFFF03F0B5A5B01E460C925E
:1027F00008910024239422A90C8016A90C8024A9F6
:1028000009250D80598C0D91FDF764FC2A99012949
:1028100000D0DFE03189012900D0DBE0318C0129D3
:1028200000D0D7E00D99002900D1D3E022460796C9
:102830002C990B912B99069180B205900F9415A8B5
:10284000058090000E900C990C582E4600252046CD
:1028500029461746FDF70CFF0028119636D12C208B
:102860000A9778430899081817A90A4668C868C2E1
:10287000E8C8E8C2E8C8E8C2079F119880B28000A3
:102880000E5822AD019523A8009020463946059A9E
:10289000069B03F0C3FE0F98401C0F902888002869
:1028A0002DD03B8A239913AC039416A8029014A848
:1028B000019015AE009617A824AA04F089F825887F
:1028C000308811900120149E0A9A05E013A8058013
:1028D00014952E4628463A460E9F51000B9B119C9C
:1028E0005C52591808830D84D81986600F98188592
:1028F000521C0D9882426DD024A805889FE7099646
:1029000016A800250580149524A8068823981290FF
:102910002F46109503E06D1CA8B2B04213D8A8B2A0
:10292000800017A90C5820461299FDF7AFFE002829
:10293000F1D1002FEFD115A8058016A80127078037
:1029400014941094E7E715A80288B01A012805D15D
:1029500015A80680099F1497119628E01020079962
:10296000095E0129119221DB551CA8B20C18109F99
:102970000E9B099403E06D1CA8B2844218DDAAB234
:10298000B242F8D8800017AA105810903946344641
:102990001E46FDF76DFE33462646099C0028EAD107
:1029A00015A80580109F14971195E4E7109F0E9BC2
:1029B0001C463E4638461299FDF789FCFDF714FF88
:1029C0000546052800D3052513A8058001200A9A8D
:1029D000274682E725B0F0BDF0B58BB00243159ACB
:1029E000149C139E2BD0054601A856C0129CD86992
:1029F000196A09900A911E469F6B0123009309A84A
:102A000007AA0146059305F0B7FE716C3846FDF73D
:102A10005EFC0746E06A616BFDF759FC002D0696E7
:102A200013D0044611980199012924D10921081ACB
:102A30000421069A515E884229D16425B1E0002024
:102A40003080207010700BB0F0BDB088002264257B
:102A5000002829D0059269493846FDF733FE002841
:102A6000049C039E6FD166493846FDF72BFE002873
:102A70001DD05A2567E03C25082800D191E05F4928
:102A80002046FDF71FFE002819D0502589E00A29AD
:102A90001DDB1D293BDC59493846FDF713FE00229A
:102AA000002854D05A253AE03346049C39E0554971
:102AB0003846FDF707FE002821D0502543E0504955
:102AC0002046FDF7FFFD00282ED0462569E03C2575
:102AD000012866D049492046FDF7F4FD0028D4D1ED
:102AE00047492046FDF7EEFD0028EED14549204636
:102AF000FDF7E8FD002854D1434920466EE04249E5
:102B00003846FDF7DFFD00281CD128251BE03B4996
:102B10003846FDF7D7FD0022002832D05025049C0E
:102B2000069B0299039E41E036492046FDF7CAFD07
:102B3000002836D134492046FDF7C4FD00282FD1A6
:102B400014252EE037250299059A069B2EE0059262
:102B50002B493846FDF7B6FD002896D1294938465D
:102B6000FDF7B0FD0028B0D127493846FDF7AAFD92
:102B70000028049C069B0299039E059A3BD11E25C2
:102B800014E005921E493846FDF79CFD00289CD1B3
:102B90001C493846FDF796FD00281DD03C2500E075
:102BA0002325049C069B0299039E059A258032707A
:102BB00000200870307800280CD118681349FDF700
:102BC00073FD002806D12088102803D30F382080F9
:102BD0000BB0F0BD0BB0F0BD0B493846FDF772FDF0
:102BE0000028049C069B0299039E059A01D1142596
:102BF000DCE72325DAE72D25D8E7C046CDCCCC3D50
:102C0000CDCC4C3DCDCCCC3C0AD7233C0000204061
:102C100070B588B00C4606464088002820D0FDF7E5
:102C2000A4FD059005A804A901252A4606F00EF882
:102C30003088B188081AFDF78DFD0390049903A828
:102C400007AA2B4605F0C2FF5249079D2846FDF70B
:102C500039FD002808D0BF200006206008B070BDF4
:102C60000020206008B070BD4B492846FDF70EFDDE
:102C7000002804D03F200006206008B070BD4749FE
:102C80002846FDF71FFD002801D0002010E000219C
:102C90002846FDF717FD002801D0022008E0404932
:102CA0002846FDF70FFD002801D0042000E0062093
:102CB00001957F21C905029180003A49091801A8B0
:102CC00006AA022305F036FF0698206008B070BD02
:102CD000F0B587B00C4605464768002638463146B1
:102CE000FDF7FEFC002802D0266007B0F0BD049777
:102CF00004A803A90126324605F0A8FFA8682968A0
:102D0000FDF7A0FA0290039902A806AA334605F03F
:102D10005DFF2049069D2846FDF7D4FC002804D01D
:102D2000BF200606266007B0F0BD1B492846FDF708
:102D3000ADFC002804D03F200606266007B0F0BD99
:102D400016492846FDF7BEFC002801D0002010E0FF
:102D500000212846FDF7B6FC002801D0022008E03B
:102D60000F492846FDF7AEFC002801D0042000E002
:102D7000062000957F21C9050191800009490918A5
:102D8000684605AA022305F0D5FE059E266007B019
:102D9000F0BDC046CDCC0C3F295C0FBFCDCC4C3E26
:102DA000CDCC4CBEF4930102F0B587B00C4606467C
:102DB0007F270088002801D0FD0503E0B0880028A7
:102DC0002ED0334DFDF7D1FC03907088FDF7CDFC7C
:102DD000049003A802A90126324605F037FF0299A4
:102DE00004A806AA334605F0F1FE2A49069E30469D
:102DF000FDF768FC002802D03F20010641E026498B
:102E00003046FDF743FC002802D0BF20010638E021
:102E100022493046FDF756FC002805D0002024E06A
:102E20000020206007B0F0BD1D493046FDF74AFC88
:102E3000002801D0022018E01A493046FDF742FC74
:102E4000002801D0042010E017493046FDF73AFC75
:102E5000002801D0062008E014493046FDF732FC76
:102E6000002801D0082000E00A200096F905019111
:102E700080000F490918684605AA022305F05AFE8A
:102E800005992846FDF7E6F9206007B0F0BDC04679
:102E9000000080BF000038433333733F0000C84256
:102EA00000007042000020420000A0410000C0402D
:102EB00014940102F0B59DB015460B917F2103914A
:102EC000C9051C9102911B9119A900248C801994A9
:102ED00018941794598C0691198C0F91DE8B998B4D
:102EE0000791997805911F882B21CA432799914210
:102EF00001DB7F0015E04022D243914211DC4922E0
:102F0000D243914202DB7908CF190AE05322D2431F
:102F10009142EEDA5D22D243914201DBBF0000E034
:102F2000FF000A971396269E597E00290BD0002198
:102F300032460F46D170917051701170121D7F1C76
:102F40005C7EA742F6D30C93119525991491229992
:102F50000D91159041088C4211D2FD4A2346A000E4
:102F600084583454270A451C7755250C871CF55581
:102F7000240EC01C34545B1C9CB2A142EFD8239891
:102F8000109001200990009030463146149A159F08
:102F90003B4605F0FFFB0D9800060890400E139D80
:102FA00000D186E068000490002F3FD00022104638
:102FB0001146144606E01C461146159F401C82B27D
:102FC000BA420ED283B2AB42F8D09200149B9A5E02
:102FD0000FB2BA42034600DC2346BA42EBDC0A4693
:102FE000E9E7002F25D0002210461146129206E094
:102FF00012931146159F401C82B2BA4214D283B27A
:10300000AB42F8D0A5B2AB420CD09200149B9A5EB2
:103010000FB2BA42034600DC129BBA42139DE7DCB2
:103020000A46E5E7139DE6E7129903E000242146EE
:1030300000E00021129110980183C4828582049FD0
:10304000F057FDF787FB7921C9050E91FDF702F9CD
:103050001099C86109980743F057FDF77BFB0E995B
:10306000FDF7F8F8109F38622004C40B3057FDF7C5
:1030700071FB0E99FDF7EEF87862601C3056FDF793
:1030800069FB0E9C2146FDF7E5F8B8621298000432
:10309000C70BF057FDF75EFB2146FDF7DBF8109CF0
:1030A000E062781C3056FDF755FB0E99FDF7D2F81B
:1030B0002063119805800C98407E410000278D42C6
:1030C00028463A46149E1ED30A9880B28AB29300CC
:1030D000F45E84420BDA491C8AB2AA42F6D9002770
:1030E00028463A4681B2691A012910D01BE0F0182F
:1030F000119B1980078808040FD0500040008019E8
:10310000001F0288084681B2691A01290BD1A80064
:10311000301811990D80078826E00020024681B200
:10312000691A0129F3D00A9989B2079B4B43BB4224
:103130001AD306998A4217D80599002914D0401C41
:1031400082B2891803E0401C82B291420CD983B24A
:10315000AB42F8D89200B35EBCB2A342F3DDB21822
:10316000119B18801788EEE712970B98058011982D
:1031700000882B1A002B16DD02210F9A1143032918
:1031800042D10E93411C421E10B281420EDA0E98BB
:10319000032824DB0C98808C012820D019A818A9BA
:1031A000FFF736FD1FE0002018902BE00026F443C7
:1031B000374608E0B8B2400019AD2B527F1C521CB4
:1031C00010B28142E3DB13B2A3423346F2DD159B1A
:1031D00098423346EEDA8000149B1B5AEAE719A89E
:1031E00018A9FFF7E1FD149E139D0F9A012A13D031
:1031F000032A11D0022A04D111980088281A022823
:103200000ADA0020179034E0022A01D1022BB8DA42
:1032100000201890012AEBD1681C691E0FB2B84239
:1032200008DA0C98808C01281DD119A817A9FFF77E
:10323000BBFD1CE00022D343144608E0A5B26D009C
:1032400019AF7E53641C491C0FB2B842E9DB0DB2C2
:103250009D421646F2DD159DAF421646EEDABD00E0
:10326000149E765BEAE719A817A9FFF7D1FC149E14
:10327000139D249F189C17992046FCF7E3FF0F9994
:10328000012900D8204638600D98002800D1CBE0F5
:1032900011990888109FB8860888281AB880129853
:1032A00080B2FDF762FA7921CC052146FCF7D2FF06
:1032B0002146FCF7CFFFB863119F3888002849D01A
:1032C00081008919091F0988129C0C1915998842D7
:1032D00003D280008019808804191598430053494F
:1032E00016AA304605F034FC169810994864FDF78C
:1032F00094FAA4B2A04201D14D480FE0001BFDF7A3
:1033000034FA1C901CA81BA9012205F09FFC204642
:10331000FDF72BFA01461B98FCF79CFF10990860FB
:103320003988491B4A1C92B2032A02D20021159FF8
:1033300017E009B20229159F12DB3F210906FDF7AC
:10334000C1F9002802990CD10998810709E0C0460B
:10335000402100400020129C15998842B9D3BCE757
:103360003449109801610898800E5DD0002F1CD060
:1033700000221146144610464B1B1DB2ED135B197B
:103380006B40139D1BB29200B25E53431818A418F1
:10339000491C8AB2BA42EFD3FDF7E7F90646204648
:1033A000FDF7E3F9002C03D100E000260398C005E7
:1033B0001C901CA81BA901252A4605F047FC1B9C54
:1033C00020463146FCF746FF014610988160002FE9
:1033D000119422D000242746264613951291B8B2A4
:1033E000FDF7C3F91299FCF72DFF0546A0001499CB
:1033F000085EFDF7AFF901461398C00785432846DC
:10340000FCF728FF01463046FCF7CBFE06467F1C42
:10341000BCB215988442E2D300E0002611983146F0
:10342000FCF718FF1099C8601DB0F0BD3CA4010264
:103430000000204100004040F0B58FB00692F74AEE
:1034400009AF70CA70C770CA70C70328079320D825
:103450008800F3A10858F649FCF7A3FE0446F54995
:10346000FCF79FFE0D90F4492046FCF79AFE0C9065
:10347000F2492046FCF795FE0B90F1492046FCF7F7
:1034800090FE0A90EF492046FCF78BFE0990EE492A
:1034900069E0042822D0062820D88800EBA108582B
:1034A000EE49FCF77EFE0446ED49FCF77AFE0D90EE
:1034B000EC492046FCF775FE0C90EB492046FCF7E2
:1034C00070FE0B90E9492046FCF76BFE0A90E84934
:1034D0002046FCF766FE0990FD4944E008380228C2
:1034E00021D88800FBA10858D149FCF75AFE0446B0
:1034F000FC49FCF756FE0D90FB492046FCF751FEB7
:103500000C90FF2081052046FCF74BFE0B90F749FD
:103510002046FCF746FE0A90CA492046FCF741FEC9
:103520000990FE491FE08800F1A10858F449FCF712
:1035300038FE0446F349FCF734FE0D90F24920466C
:10354000FCF72FFE0C90F1492046FCF72AFE0B9069
:10355000EF492046FCF725FE0A90EE492046FCF78D
:1035600020FE0990EC4900942046FCF71AFEEC4935
:1035700009680E90EB480468EB4801684808EB4F77
:1035800005463D400022002D08922DD0CA01120EA2
:1035900007D0280CE90D12D14000E649085AE64947
:1035A0000AE0C903090E0CD0280AE90B10D140002B
:1035B000E049085A8F2189004018E4300DE0DC49C9
:1035C0000AE081B27F2905D84800DA49085A04E0A8
:1035D000D94901E08F218900401800B2FDF7BAF8FF
:1035E000D649FCF737FE02460292039507252606C8
:1035F000D34B1A68002A089840D0791C8A420BD213
:103600001102090E13D0110C1F46D00D1FD1480016
:10361000C849085AC84907E01F46110E002A13D4AA
:103620004800C449085AC2494018E4301FE0110458
:103630001F46090E0ED0110AD00B12D14800BD4909
:10364000085A8F218900EFE7BE4808180FE0B848F4
:1036500008180CE091B27F2906D84800B549085AED
:1036600005E0B548081802E08F218900501800B223
:10367000FDF770F8B149FCF7EDFD3B460590159F4D
:103680002C40F50E5B69B0491940089810D0DA0259
:10369000D20E34D0C80B3E210140A648405AA6495C
:1036A0004018E43000B2FDF755F8A449FCF7D2FD0C
:1036B0000490149E6800A5A1085EFDF74BF8014632
:1036C000A00009AA1058FCF76CFD0146B8B2012809
:1036D000089F019102D1022C0AD9A74F052C24D1B1
:1036E000189808900C2D20D80B2D16D3A44918E05B
:1036F0000027022C089718D08120C70515E01A046E
:10370000120E00D1CAE0080AC90B00D0CDE040007B
:103710008849085A8F218900C2E7092D00D2C7E0E5
:1037200096490898FCF73DFD089001200021B5421C
:10373000034600D30B46052C00D308461799169A6A
:103740001A9C199D1843069B012B12D1079B402BF5
:1037500022D1002840D03846FCF723FD01460198CD
:10376000FCF71FFD01460098FCF76CFD059A0499D3
:103770008AE0079B402B1FD1002838D03846FCF741
:1037800010FD01460198FCF70CFD01460098FCF77E
:1037900059FD059A049977E0002833D03846FCF7A4
:1037A00000FD01460198FCF7FCFC01460098FCF77F
:1037B00049FD059A049967E000285BD03846FCF77C
:1037C000F0FC01460198FCF7ECFC01460098FCF780
:1037D00039FD059A049957E002981146FCF732FD2D
:1037E0000399002900D16748059A04994CE0029892
:1037F0001146FCF727FD0399002900D16148059A7D
:10380000049941E002981146FCF71CFD0399002938
:1038100000D15C48059A049936E0C0461CE20000DD
:10382000000068C1000088C166665EC1000084C1F6
:10383000000084410000B4410000484100002040E5
:103840000000F0C0000084C10000F841333323C100
:10385000000050C19A9929C19A9949C19A99494140
:103860003333CB4166667641CDCCAC40333393C025
:103870009A9949C102981146FCF7E4FC0399002982
:1038800000D14048059A049928601046FCF7DAFCFC
:103890000899FCF7D7FC20600FB0F0BD99B27F29E2
:1038A00011D848002349085AFCE623494018F9E694
:1038B000C12001060898FCF774FC0890062D00D979
:1038C00033E7002030E78F2189005818EAE6C04628
:1038D0003333F341000058C19A9961C19A9969C183
:1038E000000084C10000AC4100003841000008C164
:1038F000CDCC80C1CDCC88C133338FC1333397C198
:1039000033339741CDCC8C413333F3409A9919C06E
:10391000666646C1333397C1CDCCB4410000D44173
:103920000C0000405030004068400040FFFFFF00A6
:103930007C08000024E600005C050000919AF63C3B
:10394000642000409C0B0000FFFF1F00FAFFFCFFFB
:10395000FEFF000002000400060008000A000C0040
:103960000E00100012001400160018001A001C00AF
:103970001E00200022002400000080BF0000A0C024
:10398000000040C00000DCC2F0B5FFB0ECB017464C
:103990000E460D900021E991E891DC919991989162
:1039A000979196911491139112919AA8F49DF39C7A
:1039B000F29A002E00D1E6E10B938030F09B11804B
:1039C000099529602546DBAC218095AC21800C95BA
:1039D0002980DA917F24E405B994B894B794B69419
:1039E000B594B494B394B294B194B094AF94AE94AB
:1039F000AD94AC94AB94AA94A994A894A794A694DB
:103A0000A594A494A394A294A194A0949F949E940A
:103A10009D949C949B949A94046644668466C466C0
:103A2000046744678467C467046444648464C4644A
:103A3000046544658465C465046244628462C4624A
:103A4000046344638463C463046044608460C4604A
:103A5000046144618461C461B0090B250B2800D363
:103A6000AE011095012B0B9D00D070E12B89012B2D
:103A700000D06CE1298C00290E9200D18BE16B8C77
:103A8000002B00D1FAE1AA8C3021695C002900D119
:103A900088E10892109F5F431196304639460F9394
:103AA000FCF718FB0590FCF755FE01462046FCF795
:103AB0000EFC8321C905FCF7CDFB064696A8021D26
:103AC000119887420A9200D879E155A811909AA9D5
:103AD000069196AF15463A46059C234605F02AF80E
:103AE00015A80F9006992A46234605F023F80223CD
:103AF0000D93384631463A4605F068F8012308939D
:103B00000093E8AA10923846394604F035FEE8984A
:103B1000DD901198069D29463A46234605F00AF89D
:103B20000F9829460A9A234605F004F8384631468C
:103B30003A460D9B05F04AF8089B009338463946F3
:103B4000109A04F019FEE898DE9011982C46294648
:103B50003A46059D2B4604F0EDFF0F9821460A9A40
:103B60002C462B4604F0E6FF384631463A460D9B7C
:103B700005F02CF8089B009338463946109A04F05B
:103B8000FBFDE898DF901198069D29463A462346AA
:103B900004F0D0FF0F9829460A9A2346254604F0E0
:103BA000C9FF384631463A460D9B05F00FF8089B91
:103BB000009338463946109A04F0DEFDE898E0900C
:103BC0001198069C21463A462B4604F0B3FF0F9805
:103BD00021460A9A2C462B4604F0ACFF3846314663
:103BE0003A460D9B04F0F2FF089B00933846394695
:103BF000109A04F0C1FDE898E1901198069D2946BD
:103C00003A46234604F096FF0F9829460A9A23461F
:103C1000254604F08FFF384631463A460D9B04F0A6
:103C2000D5FF089B009338463946109A04F0A4FD4E
:103C3000E898E2901198069C21463A462B4604F0FB
:103C400079FF0F9821460A9A2B4604F073FF3846F5
:103C500031463A460D9B04F0B9FF089B0093384665
:103C60003946109A04F088FDE898E39011982146AF
:103C70003A462B4604F05EFF0F9821460A9A2B46DF
:103C80002C4604F057FF384631463A460D9B04F067
:103C90009DFF089B009338463946109A04F06CFD4E
:103CA000E898E4901198069D29463A46234604F088
:103CB00041FF0F9829460A9A2546234604F03AFF09
:103CC000384631463A460D9B04F080FF089B00932E
:103CD00038463946109A04F04FFDE898E59011985F
:103CE000069C21463A462B4604F024FF0F982146B5
:103CF0000A9A2B4604F01EFF384631463A460D9B81
:103D000004F064FF089B009338463946109A04F08B
:103D100033FDE898E690119821463A462B4604F088
:103D200009FF0F9821460A9A2B4604F003FF3846F4
:103D300031463A460D9B04F049FF089B00933846F4
:103D40003946109A04F018FDE898E7907AE0108858
:103D50000C9A108099919891DA9E08460F46099D19
:103D6000F59CFCF76FFA2860DC9827606060A6601D
:103D70000C34DDA80EC80EC42EC82EC42EC82EC406
:103D80007FB06CB0F0BDFF20108000212960208042
:103D90007FB06CB0F0BD002201233021695C0029A6
:103DA00000D076E6DDAA1ACF1AC23ACF3AC23ACF8D
:103DB0003AC20B213046FCF78DF9054642E000205F
:103DC0000690059D0796089F1190069801460D9C48
:103DD0000F9A4A43D219109B5A43119BD218D20012
:103DE000A35889002E4655AD6B503546121DA2587A
:103DF00015AB5A50401C01B28E42E9DC55A89AAE70
:103E000096AC314622462B4604F094FE15A8314666
:103E10000A9A2B4604F08EFE02232046079922467A
:103E200004F0D4FE01230093E8AA2046214604F0C2
:103E3000A3FC119B9800DDA9E89A0A505B1C0B2B90
:103E40001846C1D1F19EDDA89AA9DCAA0B2304F083
:103E500071FE09210E980F9101800B98C168DC9CBE
:103E60002046FCF7F7F90146A8B2E69F0F281BD8B9
:103E700008280DD30846FCF794F914E0FF201080C1
:103E80000021099A11600C9908807FB06CB0F0BDD8
:103E9000042803D381220846D10502E041220846C6
:103EA0001106FCF7D7F901462B20C04386420D9737
:103EB00004DB0846FCF775F9014603E04020C043E7
:103EC000864244DD0E9A0C9C0B98408A002811D043
:103ED0000B98038A95A80390DBA80290DAA80190BA
:103EE0000094DDA80D4602F073FD29462488DA9E71
:103EF000099D68E011910F98208000273D4610979A
:103F000005E00E9804887F1CB8B2A04211D8B8B260
:103F10008000DDA90C5820461199FCF7B7FB00285A
:103F2000EFD1002DEDD10C98078001250F9710944B
:103F3000E7E7DBA805800F9A90B2201A012811D17B
:103F40000C9804800D9FDA973E46099D3AE049207F
:103F5000C043864200DA8BE0FF2208469105FCF759
:103F600079F9A9E710200B990E5E012E00DA90E096
:103F7000551CABB21846A1B2AAB28A4217D805E0C6
:103F80000E990C88A1B2AAB28A4210D88000DDA98D
:103F90000C58204610991F46FCF76AFB3B46002848
:103FA00005D10C9805800B98068A0F95109430B2B5
:103FB000C1186D1CA8B28142E2DC109EDA960F9CFB
:103FC000099D0D9F11993046FCF781F9FCF70CFC17
:103FD000052800D3052095A90880A0B20E9909886C
:103FE000814218D9401C611E0CB2A04218DA12A8F6
:103FF00098A9FEF76DFE0E980188481C491E0CB268
:10400000A04221DA12A899A9FEF762FE9999989820
:10401000099D0D9FA4E600219891999108469FE67D
:104020000022134608E09CB2A40012AF3D515B1C75
:10403000491C0CB2A042DADB8DB20A2D1546F2D82B
:10404000A400DDAD2D59EEE70022134608E09CB236
:10405000A40012AF3D515B1C491C0CB2A042D1DB45
:104060008DB20A2D1546F2D8A400DDAD2D59EEE72C
:104070005320C043864200DB1BE70E460B98816944
:104080002046FCF7F5FA00280C9C08D10B98808B91
:1040900007E01446099D0D9F1199109E93E70B9818
:1040A000C08BFCF762FB01463046FCF7D3F8119059
:1040B00021E70000F0B58BB01C4609930E4603467D
:1040C00000200A9040480088224F05970AA90491D1
:1040D00003940292109C0194012500950B21414309
:1040E00089B230331C4A3046FFF74EFC38680790DF
:1040F00078680890B868069033480088334F009578
:1041000001940297324E30363249334A3346FEF735
:104110006BFB0698F86207983863089878630998EB
:1041200000882E4905912E4904912E49039102974A
:10413000019000962C4B284629462A46FEF74CFC57
:10414000432001060A98FCF785F8FCF74DFB0BB0FD
:10415000F0BDC04604A4010250C20102F0B589B00E
:104160000F9F0E9C002815D01098079016480088C5
:10417000164E01250095019102960893144B303399
:104180001449154AFEF730FB089BF7620798306325
:10419000746303E00D484763C462002518880F4923
:1041A00005910F4904910F4903910849029101902B
:1041B00007483030009001210B4B28460A46FEF795
:1041C0000BFC09B0F0BDC046ACA8010214B7010257
:1041D000689D0102889C0102ECB0010234A1010239
:1041E000A8A8010248A8010250A8010280B582B027
:1041F00001AB002018703121012200F057FB02B002
:1042000080BD000070B5421E0F2A23D8082808D8A8
:1042100001209040104A137F00290BD003431377ED
:104220000DE00938012282400B48437F002904D069
:10423000134303E08343137701E093434377064E30
:10424000747F357F402002212A462346FDF714FC67
:104250007477357770BDC0469495010280B51248D9
:1042600001681F220A40026003200840022812D180
:104270000E480268D30D02D0FF231B06D2180C4B48
:104280001A600C4A12680C4B1A6080680B4A108046
:10429000000C0B4A10801A488268002A02D08268FB
:1042A0000020904780BDC04674200040644000401C
:1042B00000B101027830004004B10102CC9D01023E
:1042C00008B7010280B50D48016889070FD505219F
:1042D00001600B48C178002908D00021C170C16875
:1042E000002903D0C26841680020904780BD05487E
:1042F00005A10B4A0BA307F035FDC0462C04004076
:10430000DC93010293F100005048595F54494D4538
:10431000525F49525148616E646C65720000000042
:104320008D0A0000556E6578706563746564206958
:104330006E746572727570740000000070B582B0A2
:104340000E484568056001A9002008700C4E05E084
:10435000401C01A90870C1B205290DD2C1B22A467C
:10436000CA40D107F4D0B268002AF1D001AC0021D4
:10437000204690472078EBE702B070BD3030014016
:10438000D095010270B50446401E012814D80320C0
:10439000084011D13F2040030818050B2819802838
:1043A0000AD8164E317801204840294603F03AFBDE
:1043B000641E6D1C002CF5D170BDC04680B5002078
:1043C000014603F053F8002800D080BD0B480121BE
:1043D000017080BD70B516460C460546FF22FBF7FE
:1043E000C7FE0548311805480278012050402A468A
:1043F000234603F0BFF970BD00E0070440A60102A8
:10440000012000037047012040037047F0B585B0DC
:1044100048484949016005F03BFA484DEA8A4A217B
:1044200047484252AC8A482144520021E983AB8874
:104430008362AE7A0671AE89C68104824282AA8DF9
:10444000028704938386EC8E01221D2C144600D82B
:104450000C463C490C703221695C41711002688045
:10446000288B394908806C8C0F20224602407D2120
:10447000C900260B4E43B6182205170F6422574376
:10448000F6192406270F0A246743F6192F4F3E809A
:10449000AE8C374607402B46350B4D43ED1937059B
:1044A0003F0F5743ED193606360F6643AD19284EB8
:1044B0003580DD8C2E4606402F0B4F43BE192F054D
:1044C0003F0F5743F6192D062D0F65437519214FE0
:1044D0003D801D8D28402E0B4E4330182905090FB5
:1044E000514340182906090F614340181A4E308085
:1044F00003241AA220462146049B08F08FFC0F4893
:104500004088C1B20091030A18A22046214608F053
:1045100085FC0E4803880E480088398832880A4D89
:104520002D8800AE27C619A22046214608F076FC49
:1045300005B0F0BDEC9501028951000042A60102D0
:1045400028990102FC960102DE960102D69601022C
:10455000D8960102DA960102DC960102C9E8B1B8E8
:1045600049443A202578202E0D0A0000B9CCBCFE23
:10457000B0E6B1BE3AB7C0B6AAC6F7B1EAC7A9203D
:104580005625642E25642E200D0A0000B7FECEF1BC
:10459000C6F7B5D8D6B73A2025642E25642E2564F3
:1045A0002E25643A25642E0D0A000000F0B583B074
:1045B00030480068C16B0901890F01D003B0F0BD1C
:1045C000C16BC06B2C4D05404800400F0826029679
:1045D00086400227384601F0F7FE01907043C10B78
:1045E0004A1B26485043FBF78BFD044607F0A6FA0A
:1045F000032123A238461F4F0091234608F00EFCEA
:10460000F88A002817D0019840012946FBF762FD7F
:1046100046431822324001200F2A014600D80021CB
:1046200073095B181B4CA3420DD8194DED1A6D058B
:104630000F2A0CD80CE038680021C160112001F06D
:10464000B3FE03B0F0BD5D1C6D050F2A00D95642C4
:104650002A0C029D2E4009018919A34202D8009814
:10466000000400E04004081880183968086303B0AB
:10467000F0BDC0466C940102FFFF1F0040420F00D6
:1046800052434F33324B2070706D2025640D0A0069
:10469000FF070000FE7F0000B0B582B01549086832
:1046A0008269D2070CD00122C2610D69002D07D0AA
:1046B00000686C46214607F01FF800212046A847F5
:1046C00002B0B0BDB0B582B00A490868026C92076A
:1046D0000ED5026C012313430364CD68002D07D06F
:1046E00000686C46214607F007F800212046A847DD
:1046F00002B0B0BD6C9401020648016803229143E8
:104700000160016801220A43026000F081F907F0AC
:1047100037FAC04628000040B0B500F0D6F800F0E7
:1047200093F801247D210422204600F0C7F864207C
:1047300000F0B6F8402507222046294600F0BEF8D2
:1047400041210022204600F0B9F83F2110222046E6
:1047500000F0B4F806210B22204600F0AFF8082143
:10476000C022204600F0AAF830212A22204600F07C
:10477000A5F8322120462A4600F0A0F83321204631
:10478000224600F09BF8B0BDF0B581B000290BD0F7
:1047900014460D4606460027B81980B2FDF78FFA79
:1047A000E0557F1CBD42F7D101B0F0BD80B50D4989
:1047B0000868002810D5224802680423032A01D083
:1047C0001A4300E01A460A601E490A68002A02D00D
:1047D00041680020904780BD03A00CA19E2211A338
:1047E00007F0C0FA2C100140696E636C7564652F88
:1047F000647269766572732F6D6B5F736C6565703B
:104800005F74696D65722E6300000000534C45456E
:10481000505F54494D45525F49525148616E646C36
:1048200065720000556E6578706563746564207309
:104830006C65657020696E746572727570740000C5
:104840000C90010210B70102B0B582B000242046DE
:1048500000F02AF801AD2C707F212046224600F09E
:104860002DF8642001F0CCFE012120460A462B469B
:1048700000F01CF82B78032003A2014608F0CEFAC2
:10488000204602B0B0BDC0465343374132325F5775
:10489000484F5F414D5F493A307825780D0A000056
:1048A00080B501F0A6FE80BD0120704780B50846A6
:1048B00011461A46FFF768FF012080BD80B5084603
:1048C0001146FDF748FA012080BD80B500204A213D
:1048D000A522FFF7F3FF80BDB0B5214C6078411CE5
:1048E00061703D2807D300206070204624300121EC
:1048F0001C4A01F013F907F0B7F81B4DA88F0028E8
:1049000016D01A49087840B2421E0A70002801DC0D
:10491000002100E001214900154A1170002804DD42
:104920000320144906F036FC02E0032006F024FCC4
:10493000FCF704FD0D48017849B2002906D4688FC0
:10494000A189814208D9401CA081B0BDFF2101701E
:10495000688FA1898142F6D80846401CA081B0BD6D
:1049600028990102DD59000042A601020D970102BB
:10497000E8B0010238950102F0B582B001930090D1
:104980000C784D782D022C198D78C97809024919B7
:1049900009040C198100134D6C509478D67817785F
:1049A0005078114B019A5A501A460002C01936022B
:1049B0003419240420186C18206307980478407870
:1049C0000A4D2D680A4E7550009B5B00094DEB188F
:1049D000000200195024185350180999016302B0BD
:1049E000F0BDC04604980102649801027897010264
:1049F000389D0102F095010280B504480168491C08
:104A000001600069002800D0804780BD7CC201029F
:104A100001480249016070473C9001020026B8033A
:104A200080B582B00E4908680022C2600192CA684F
:104A3000002A02D0016801A8904702B080BDC0469C
:104A400080B582B0064908690022C2600122019245
:104A5000CA69002A02D0016801A8904702B080BD4F
:104A6000D8920102F0B58BB0FD4C6079002857D088
:104A70000020607101273846394606F055F8F9489C
:104A8000F94904F07FFAF94D5B266E7039202870E1
:104A900050222A720220E871A871F5498888A8700E
:104AA000A38B2B71000AE870180A68712846093038
:104AB000891CFBF74BFB28463146FCF7EDFAA8555D
:104AC000000A29465B314870C320860106F028F8A9
:104AD0008319A3645D2128463A4609F003FB20644C
:104AE000A56C05F0B3FF401906F06EFD05460E46B5
:104AF000F948007B06F0F4FB81B2C90B401800B204
:104B0000C1174010F54A281810617141516106F033
:104B100007F8206304F0A6F90028FBD10BB0F0BD24
:104B200001200990014605F0FFFFE748E74904F03E
:104B300029FAE8484088E64DE871E9490988697131
:104B4000E84A12782A70E84A12782A716278EA7084
:104B5000000A2872080AA871501C6070A08AA17C03
:104B6000091ACAB2192A00D319212170A97249065B
:104B70000E0E4700DD48C11928460B303246FBF7C0
:104B8000E5FA70190B30DA49C9193246FBF7DEFA3B
:104B90002020687200200890A072E08A6870000AE5
:104BA000A870C320860105F0BBFF8319A364207899
:104BB00081000D312846099A09F094FA2064A56C09
:104BC00005F044FF401906F0FFFC05460E46E64896
:104BD000007B06F085FB81B2C90B401800B2C117FB
:104BE0004010BE4A2818106171411646516105F007
:104BF00097FF206304F036F90028FBD105F090FF01
:104C00006063A06CBB4D4119E1640120BA4A079072
:104C100009F01CFA206405F083FF21786943B74A44
:104C20008918206561650918481C00D00846A065F0
:104C300005F076FFA26DB24D5119E06521660FE0D7
:104C40000020E0720146AC4A09F000FA206405F049
:104C500067FFA06305F064FF2063A26DE06D51194A
:104C6000904202D3884200D8E6E005F059FFE065A3
:104C700005F056FF606304F0F5F800280AD0FCF751
:104C8000E3FF05F04DFFE065A16D8842F3D94919B6
:104C90008842F0D205F044FFA063E07A0228CFD02A
:104CA0000128DAD10027E77238463946924A09F0DE
:104CB000CDF92064934A507A212818D020281ED19B
:104CC000FBF732FA0A21FBF71BFA61667D20C00070
:104CD000401AFBF73FFD47210906FBF7BBFA8C4959
:104CE000FBF7F5FAFBF799FD06F02CFFB5E75079D5
:104CF0009179090208187A490988884205D0107804
:104D00000828AAD100F038FCA7E71078754909787F
:104D10008842F5D1A7665078917809020918A184D4
:104D20000AA804910180608A0028394649D06F4959
:104D300009880AAA12888A4215D006900799099014
:104D4000CBB2984212D95A006848865C82180998FA
:104D5000527812029219491C0AAE36889642EFD157
:104D600006935E4E39E00023069336E0C7285B4E7B
:104D7000069936D8A28A193293B2834221D203927D
:104D800041005B4A5218921E0693584B59188B1ECD
:104D90000021C943059101461E885E801688568011
:104DA00059484618761E367846540598460092199A
:104DB0009B19491E8EB206988642EDD80399474E3C
:104DC0000998099006918BB25900484A04985052AC
:104DD000474A57520998401C608205204A49C854E6
:104DE000069900200990E0662173A08AC9B2081ACA
:104DF000E084B369216F3269424F3E462236009605
:104E000001910292C0B239461A313A461E32FFF77A
:104E1000B3FD2521795C227B3C4B9954052903D1B4
:104E2000A273617B491C617396213846FBF7A7F991
:104E300009982083294E10E70125284601F0E0FB60
:104E4000284609F02DF930697169FCF74BF8608A42
:104E50000028089926D000212B4B244D0EE0C04697
:104E6000049701022DD0000095B900005CCF01022B
:104E700042A601025B1CAD1C401E13D01F787E1E93
:104E80001E70002FF6D02A8809928AB20F4621465A
:104E90001D4CA6540C4639465200144E099FB75279
:104EA000491CE7E7618288B260642178A28A5218BF
:104EB00091B28142089B194600D211461A2800D3AC
:104EC0000B46A3820BB0F0BD2DD0000095B90000B9
:104ED0005CCF010242A6010282900102C898010241
:104EE000509901022C9901023299010224C4010255
:104EF00094C20102200C010080841E008024010065
:104F00000026B80378B50102B4C501027CC60102CF
:104F100000007A4410B582B009F066F8124C60784F
:104F200008F05EFE11498A88684682800A884988AE
:104F300009048918009104F02DFD6078052804D03B
:104F400002220B49092805D003E00122084909285B
:104F500000D0891849792078621C08F005FF607A32
:104F600006F0D0F902B010BD8290010234E20000D8
:104F7000D09D0102F0B581B003F0B2FA164CE060AA
:104F8000A178002901D001B0F0BD21790029FAD122
:104F90000121217100281BD04D02281AA1688142ED
:104FA00016D00E4E2F46A068305C21698847A06855
:104FB000401CA060681EA168814201DD0020A06045
:104FC000E168A068022F03D3691A7F1E8842EAD1E4
:104FD0000020207101B0F0BDDC950102A8AE0102F5
:104FE00080B5002008F03CF980BD80B5012008F0B4
:104FF00037F980BDF0B589B00022D543032800D928
:10500000ABE00C46002900D1A7E00095216A0727F4
:10501000534DA9420EDC574DA9421ADD564A914222
:105020002FDC4B22D501A9423ED0120291424BD136
:10503000042246E04B4A914217DD4B4A91422ADC5A
:10504000E1221203914231D0494A91423CD10C22D3
:1050500037E04B252E01B14233D06A01914227D06F
:10506000AA01914230D102222BE0E1225502A9424D
:1050700020D09502A9421FD0D202914224D1092208
:105080001FE04B225202914218D0E12212029142BB
:105090001AD1062215E0E1225203914210D0334A80
:1050A000914211D10D220CE003220AE00A2208E00D
:1050B000012206E0072204E0082202E0052200E0C7
:1050C0000B22D1002D4A57587C2141432C4A505085
:1050D00056182068B0606068F060A1683161E268CD
:1050E00072610025059503230493039502950197AA
:1050F0000695079501231B020893012807D0002875
:105100000AD18818009A8018B161F06104E0304635
:1051100020300123FCF7FFF8206970636069B063F9
:10512000E069B067A069F063706801A908F0CAF986
:105130002068012806D830464030234610330ECB75
:10514000FCF70EF96068012807D1301D7036006841
:1051500001220C4B314608F089FA284609B0F0BD0F
:10516000FFC10100FF0F0E00FF1F1C0080841E0006
:1051700040420F007F250000FF95000060E2000024
:10518000B0A80102BDD80000F0B585B0F249097899
:10519000002956D0EF4FF98B002952D1EF4EB1685C
:1051A00008292ED88A0001A39A589746D1510000A9
:1051B0000352000003520000DD51000003520000C2
:1051C0000352000003520000E75100001352000098
:1051D000552833D10120B06005B0F0BD0721B16082
:1051E000707005B0F0BDF17872181073481CF07043
:1051F000C0B27178891E814223D10820B06005B009
:10520000F0BDAA2813D1012911D10220B06005B048
:10521000F0BD7278032A16D3931E00242146351957
:105220002D7B491989B2641C9C42F8DB0CE00229F1
:1052300004D1B0700320B06005B0F0BD00207070E4
:10524000B06005B0F0BD002108188118B0780918C9
:10525000C9B2FF2900D039E1302825D0032800D079
:1052600034E1C14800250570317BB47B707B012996
:1052700036D0022900D029E1381831460F312246B4
:10528000FAF764FF388AFB4CF94F01285BD1B84824
:105290000570B8480121017006F0C0FB4B2080006A
:1052A00001F0A7F93C6011E1F389B380347B0F2C46
:1052B00000D90BE1F089318A09040918083A757B95
:1052C000062C0491039536D1A0200190A448048DAA
:1052D0009C42029304463FD1283400230546C0E097
:1052E000A24A9471032111719170AA215170552124
:1052F000117040085071651DD5704000391817466F
:10530000D01D2246FAF722FF381DE11CEAB2D21C5A
:10531000037892B2D218401C491EF9D1E019D1434A
:10532000C171090A01720934002039462246034638
:1053300008F0E0FACAE08A4D298D994213D1294636
:1053400028310023ADE006F069FBBFF34F8F3C60CE
:10535000BFF34F8F00BFFDE7808D98420AD12546ED
:105360002C3401237DE0A88D98420AD129462C31A6
:10537000012396E0208E98420AD12546303402233C
:105380006FE0288E98420AD129463031022388E006
:10539000A08E98420AD125463434032361E0A88EBA
:1053A00098420AD12946343103237AE0208F98426B
:1053B0000AD125463834042353E0288F98420AD175
:1053C0002946383104236CE0A08F98420AD1254643
:1053D0003C34052345E0A88F98420BD129463C3147
:1053E00005235EE04020205A98420BD125464034E8
:1053F000062336E04020285A98420ED129464031F3
:1054000006234EE044202146205A029B98420DD1AB
:105410000C460D464434072323E019464420285AFD
:1054200098420DD12946443107233AE04820085AD2
:10543000029B98420CD10C460D464834082310E0DC
:105440004820285A884225D129464831082328E097
:105450004C20085A029B98423ED10C460D464C34D3
:1054600009230520E854E818039981720621017583
:105470000499080C60802180307828188277019880
:10548000385A642159436918502288523548029984
:1054900001801BE04C20285A884224D129464C31F7
:1054A00009230520E854E818039F87720475049FB8
:1054B000380C48800F803078281882776420584351
:1054C0002818503031461231FAF740FE0020F070B3
:1054D0007070B06005B0F0BD01983D5A3478092C69
:1054E00006D8641C05E0317809291CD8481C1BE04B
:1054F0000024E7B205200B46C855642078430818FD
:1055000050214552B8001818049D290C4185058585
:105510001448029901803470D819039981720621C8
:1055200001758277D2E700200290C0B205232B5488
:105530008300EB1804990F0C5F851985029931706F
:105540002918039B8B720C758A7764214143681874
:10555000B7E7C04642A601028494010258960102B0
:1055600036B10102EAB001023099010292990102BA
:105570009199010290990102B0B52F4D288B811E9F
:105580002E4C2046FBF788FD6883298B0919891E5C
:105590000A7849780902891880B2884200D0B0BDE3
:1055A000A088274909888142F9D16088A883617A57
:1055B000012922D0062904D00229F0D101206871E6
:1055C000B0BDA17AA971AA29E9D1E17A227B1202A0
:1055D00054182C84E3D0688401202872E871642177
:1055E0002046FAF777FD401C16490880032016A2D2
:1055F0000146234607F012FCB0BDA07AA87103282B
:10560000CDD3E17A227B12025118E983FE221040A9
:10561000154A135A8B42C2D01018018006F0FEF9C9
:10562000124800F0EDFFBFF34F8F114811490160A0
:10563000BFF34F8F00BFFDE70497010278B5010269
:10564000509901023CA60102BDF8C8EBC9FDBCB6E9
:10565000C4A3CABD2CBDD3CAD5CEC4BCFEB4F3D03E
:10566000A125640D0A00000042A6010260EA0000C4
:105670000CED00E00400FA0580B582B00020019036
:105680000448C268002A02D001A80021904702B055
:1056900080BDC04644950102F0B583B00024204689
:1056A000FEF78CFEFEF7AFFE274EB060FEF7A8FEB9
:1056B0007060264F0BE001A8C1888088084319D18B
:1056C00001A8408824180834B068844235D201AD5E
:1056D000082128462246FEF77DFE28880028EAD0C9
:1056E000B8422AD001AD0421284600F027FFA9883E
:1056F0008842E5D03460B06884420CD201AD02210A
:1057000028462246FEF766FE2888B84203D0A41C2D
:10571000B0688442F2D370682118491E40420840A4
:1057200030600DD00024254601202946FEF72AFED0
:1057300003CE4D19083E8542F6D3346003B0F0BD68
:105740000024346003B0F0BD80970102FFFF000029
:10575000F0B585B01F4604920646C8170C184440A1
:105760000A2C039114D301250A212046FAF7B2FC32
:105770006D1C632C0446F7D804998D4200D329464A
:105780000A9C002F09D00398002808D4002207E0C3
:10579000012504998D42F2D2F2E7002205E00122B0
:1057A000042323409B081343FA1A0223234004983E
:1057B0000028029412D1002B10D0F468002C62D47F
:1057C0000398002825D40298400734D57068B5683E
:1057D0006F1C87422FD830682B2423E0E407ECD1DC
:1057E000002A0AD1E9E7376820203855B560F0680B
:1057F000441CF460521E002CDFD49142DDD2776845
:10580000B468651CBD42EED9F468521E002CF4D574
:10581000D3E7404203907068B5686F1C87420AD88E
:1058200030682D244455B760F068441CF4600025AE
:10583000ED43A84227DB002B1CD00120029B18401F
:10584000049B184316D1002A03D113E0521E002CEA
:105850000ED491420CD27068B3685D1C8542F5D8B5
:1058600030683024C454B560F068441CF460EDE73F
:10587000002C08D40092029801900A223046039925
:10588000049B00F003F805B0F0BD0000F0B587B050
:105890001F4615460290012406919142009407D3B9
:1058A000012406982946FAF715FC641CA842F9D28F
:1058B0000D980C9ABC42039700D3039400990140C1
:1058C000002A009109D00029029C25D120218007BF
:1058D00005D40846002F11D004E0029C1CE03020C3
:1058E000002F0BD0084609E023685854A260E168F5
:1058F000491CE1603246721E00290DD40399914281
:105900000AD216466368A1684A1C9A42ECD9E1683B
:105910003246721E0029F1D5E068002859D405905E
:10592000012401E07F1E6C43022FFBD20698214622
:105930001646FAF7CFFB3246A842F4D202988068A6
:105940000490069F0195069738462146FAF7C2FB58
:10595000049D691C029F7A68914206D9069F059AA8
:10596000019D0592002A0ED516E01B4A125C3B6889
:105970005A55B960FA68521CFA600491069F019D5D
:105980000592002A08D460433F1A20462946FAF7B8
:10599000A1FBAC420446D6D200980028029C059B8D
:1059A000049D16D0002E14D0701C01E0002B10D4E2
:1059B000401E039981420CD2691C62689142F5D85D
:1059C000226820235355A160E268531CE3600D4612
:1059D000ECE707B0F0BDC0463CE50000F0B583B091
:1059E0000190204E0291002922D000271E4D0097E1
:1059F0000AE01F4941184A0F8918C910A9727F1C73
:105A0000B9B2029A914215D2019800884B24210123
:105A100000B200F031F8400061014018A88200B2E5
:105A2000B0420099EADB11498842E2DD6421E5E7F2
:105A30000D48808A01B201240020B142224600DBD9
:105A40000246094BDA72B142214600DA01460948A2
:105A5000007802F0FDFD05202146FEF7D3FB03B0E0
:105A6000F0BDC046E40C00002899010204100000BB
:105A70001CF3FFFFFA960102074A904201DD054A36
:105A8000801800B24143C817400D0818C00A00B280
:105A90007047C04600F0FFFFFF07000010B5007818
:105AA000012819D1AC480269012A04D1614A13685E
:105AB0000124A3431360032905D080214161C269F9
:105AC000002A05D107E001214161C269002A02D004
:105AD00001898069904710BDFF222E32024803A140
:105AE00007A306F03FF9C04608ED00006164635F5C
:105AF000646D615F63616C6C6261636B00000000E8
:105B0000556E657870656374656420646D612063AB
:105B100068616E6E656C0D0A00000000F0B58DB016
:105B20000D460124EFF31081214002D1EFF31083E1
:105B300072B6894E73690F2B06DD102B37D0402BC0
:105B40002FD0802B2DD005E0002B2AD0012B01D1A6
:105B500010237361B5813581B061F261002900D1F4
:105B600062B63179002929D00294304C05A90A4641
:105B700004950390E8CCE8C2E8CCE8C2029C204639
:105B800000F0AEFD2A4800902A4D294608312046F3
:105B9000039A049B00F014FE2C60002420460DB0F4
:105BA000F0BD0029FAD162B620460DB0F0BD022446
:105BB0000029F3D162B620460DB0F0BD317800293E
:105BC00007D01C48072181610460002420460DB0E5
:105BD000F0BD3269B3891749002B15D0B5693089FA
:105BE000012A02D0002A03D003E09FB2874200D1ED
:105BF0000C604F68FF07FCD08F6880C55B1E1F04D8
:105C0000EED10023B381B561012A02D10A68A24313
:105C10000A607461F2690024002ABFD0B369318937
:105C20008800181A904720460DB0F0BD7CE50000B2
:105C30009D5A000008D00140F0B581B0002856D030
:105C40000446424EF068800754D41325284600F0DD
:105C5000B3FB284605F042FD2768616801253846F8
:105C60002840CA07920F1018227C1207120E8018C3
:105C7000627C1207120D8018A27C1207120C801889
:105C8000627D13071B0AC0181209120680183060C3
:105C90007D2006020029304600D12D48E3681A0A0B
:105CA0007D2A1A4629D22B4EB3422AD200292BD064
:105CB000002A2946254E00D01146FAF70BFA401E5D
:105CC00080B2706024480761E27C0270237D03711A
:105CD000224F3E686902A468012C1BD02C02264387
:105CE0003E60002B1ED00121184A116329E00120DB
:105CF00001B0F0BD022001B0F0BD3246154EB342F6
:105D0000D4D333460029D3D11A46002A29460F4E50
:105D1000D2D1D2E73F242401A6437618F0363E6064
:105D2000002BE0D1002A0CD0FF2212020C4B1C6881
:105D300094430122D203A2181A60304A1160304AFB
:105D4000116001214161002001B0F0BD00D001408F
:105D50000026B80380841E00589501022C060040DE
:105D600008E400E070B5002801D0012070BD0C46A9
:105D70001625284600F020FB284605F0AFFC002C35
:105D800005D01B48183014222146FAF7DFF92821E4
:105D90001748415C002915D04168002916D4032218
:105DA0000B469343144A9C588D07ED0EFF26AE40D8
:105DB000B4439C501F220A40012191400F4A1160B8
:105DC0000F4A116001210161002070BD8A07D20EC7
:105DD000FF2393400F220A40083A03218A430549D2
:105DE00054589C43545001210161002070BDC046AD
:105DF000409001021CED00E000E400E080E200E0E1
:105E000000E100E05A21014A50527047689D0102AA
:105E100070B50A4E306002240025204629462A46E5
:105E200002F0EEFB012120462A4602F07FFC326898
:105E30000321204602F05CFB70BDC046309E01028B
:105E4000B0B59D4DA8600D24002120460A4602F001
:105E5000D7FB01210522204602F068FCAA68032135
:105E6000204602F045FBB0BD70B55621E548B4228E
:105E700042525C2100234352414AC287838739241E
:105E800044874049C18683863F4D45863F4D058600
:105E90003325C58583854485C18483847A244484DD
:105EA0000384C3830383C3820382394C44608360C9
:105EB000C360836503463E33364C250CDD829C82ED
:105EC000160C5E821A826422DA8157229A81672236
:105ED0005A815E221A81DD809C805E80090C0187D8
:105EE00001853D21490441834182090C81838182DE
:105EF00070BDC04670B55621C248B42242525C21E2
:105F0000002343521E4AC2878387392444871D4990
:105F1000C18683861C4D45861C4D05863325C58567
:105F200083854485C18483847A2444840384C38321
:105F30000383C3820382164C44608360C36083651D
:105F400003463E33134C250CDD829C82160C5E8288
:105F50001A826422DA8157229A8167225A815E224C
:105F60001A81DD809C805E80090C018701853D21BE
:105F7000490441834182090C8183818270BDC046FE
:105F80006C00630024002F00C7FF0000B7FF000073
:105F90004C3737376200640070B59B484C21016074
:105FA00001252C02601C00F087F9322000F028FB4C
:105FB00000F070F9284600F077F9284600F086F8DE
:105FC00000F062F90C4800F077F9002630463146BF
:105FD00000F082FA2846314600F07EFA204600F0B2
:105FE0006BF9022000F068F94834204605F032FED3
:105FF00005F090FE70BDC0460102000010B50446D9
:1060000006F06AFD2C48446010BDC04670B50524FA
:1060100004252046294602F061FB0620294602F0AD
:106020005DFB01263046294602F058FB0E2029462A
:1060300002F054FB00252846314602F04FFB0221B6
:1060400028462A4602F072FB0A20214602F046FB4F
:1060500070BD80B5042002F0BBFA80BD10B50120F0
:10606000114907F02FFAFAF783FE1048FFF7E4FD15
:106070000F4805F0FDF80F48002101600E4C226822
:106080001120022102F034FAA2680D20032102F04F
:106090002FFA042002F0ACFA05F03CFE60680721FC
:1060A00006F01AFD10BDC04688940102249001023A
:1060B0001C900102E4950102C896010202480168A1
:1060C00001229143016070475800004002490A686C
:1060D00002408242FBD1704704600040B0B5494D98
:1060E00028688107484C0ED528797F21084022680E
:1060F0008A431018206023680B4002200321434A82
:1061000006F08CFE286880040ED55E20285C7F2176
:10611000084062688A431018606063680B40022080
:1061200003213B4A06F07AFE172000F045F9394872
:10613000016802220A4301218A4302603648374936
:10614000016037480021C17181791F252940817183
:10615000817A427C837C1B029A18C37C1B04D21870
:10616000037D1B06D2182F4B9A4218D1427B837BAA
:106170001B029A18C37B1B04D218037C1B06D2187F
:10618000294B9A420BD1C27A037B491E122906D8A9
:1061900019028918254A914201D120210172017802
:1061A000CA0602D11022114301701C3C2068202134
:1061B000884320601E481F49016041680029FCD5C2
:1061C00003F048FB0446022003211BA2234606F0ED
:1061D00025FE0A20C441032C05D8022003211DA25C
:1061E00006F01CFEFEE71848C1680F229143C1600B
:1061F0000168164A0A4002601920000114494860EB
:106200000D60B0BDD09D01024800004050ED00007F
:106210003AED0000040200400C060040AF6B100A8B
:106220006B0001404D383650312E323607340000B5
:1062300000600040FE1C0080436869702049443AB9
:1062400020253038780D0A00C8600040FEFFC3FFEB
:106250000C0400404F6C642063686970206D6F64AB
:10626000656C206973206E6F7420737570706F7227
:1062700074656420627920746869732053444B21EB
:1062800021210D0A0000000080B5172000F08CF8D5
:10629000002080BD10B51724204600F08DF8204660
:1062A00005F01CFA002010BD0121C9070143014877
:1062B000016070470060004010B5C1B2000AC2B270
:1062C00002290CD0012913D0002930D1911E7F481A
:1062D00002291BD20121032A2AD0490429E07B4844
:1062E0004168002A1FD00246203A1143416010BD88
:1062F00076480168D31E022B10D3012A29D0002A28
:1063000041D1012292079143016010BD002A16D1AC
:106310000121490702688A43026010BD0123042A53
:106320001FD05A041EE0012292079143416010BD24
:106330000904194A7F32C36A13405918C1621749C8
:106340008A699207FCD50121490702680A43026065
:1063500010BD0522120791430246203A0A4302600B
:1063600010BD1A04836A0C4C1C40A21882620B4AAE
:10637000131F00241C600A4B0A4C1C600D235B0297
:1063800014681C431460054A93695B06FCD505221A
:1063900012071143016010BD80FFFCFF1402004092
:1063A00004010040FF0F00000121814047480268BE
:1063B0008A4302607047C046012181404348026819
:1063C0000A4302607047C04610B5052811D8C04680
:1063D0007844007940008744020E192434393B493F
:1063E0000A680868C0003CD53A4820390A425DD0A6
:1063F0003BE0002010BD35490A680868C00035D56B
:1064000034480B46203B1A4237D134E02F490A6802
:106410000868C00036D52F480B46203B1A424CD1A5
:1064200035E02A494C680120C0030A680B46203B2E
:106430001C421AD00C68E4003BD5264C1A423CD0D2
:106440003AE0224800680120C00310BD1F490A68D5
:106450000868C0001ED51F480B46203B1A4220D1B9
:106460001DE01B4820390A4220D010BD18480B46B9
:10647000203B1A4201D10120C00349688900890FDD
:10648000C84010BD12480B46203B1A4215D10120CE
:10649000C00312E00E480B46203B1A4201D10120F6
:1064A000C00349680903890FC84010BD0120C0031B
:1064B00010BD074C1A4200D020464A689200920F45
:1064C000D04049680901890FC84010BD2000004034
:1064D000006CDC020026B80304282CD8164AC046FB
:1064E0007844007940008744020A121A21000320F0
:1064F0000007136883438807800818181AE00320F0
:1065000080061368834388070009181812E00320E7
:106510008004136883438807000B18180AE0FF20E3
:106520000002136883430802181803E01068FF2371
:10653000984340181060704724000040B0B5002216
:1065400000290CD0074B047895B22D0A65406C00E9
:106550001C5B12026240491E401C0029F3D190B21C
:10656000B0BDC0463CE30000002841D000BF00BFE2
:1065700000BF00BF00BF00BF00BF00BF00BF00BF23
:1065800000BF00BF00BF00BF00BF00BF00BF00BF13
:1065900000BF00BF00BF00BF00BF00BF00BF00BF03
:1065A00000BF00BF00BF00BF00BF00BF00BF00BFF3
:1065B00000BF00BF00BF00BF00BF00BF00BF00BFE3
:1065C00000BF00BF00BF00BF00BF00BF00BF00BFD3
:1065D00000BF00BF00BF00BF00BF00BF00BF00BFC3
:1065E00000BF00BF00BF00BF00BF00BF401EBDD145
:1065F000704780B57D21C9004843FFF7B5FF80BDD6
:1066000000280AD030B407252C02CD256419604338
:1066100040091238001FFDD830BC7047F0B583B078
:106620001F4616460D460146E8680291F9F712FE2C
:1066300004460F2E11D8082E04D320462146F9F720
:10664000B0FD09E0042E02D38120C10501E0412004
:1066500001062046F9F7FEFD04460999089E2B2005
:10666000C043874205DB20460F462146F9F799FDD6
:106670000DE03F20C04387420BDA4920C0438742E8
:106680000CDBFF200F4681052046F9F7E3FD394674
:106690000446688A0880346003B0F0BD019153203D
:1066A000C043874206DB20462146F9F77AFD0446BF
:1066B000688A10E0A8690299F9F7F6FF002801D16D
:1066C000A88B00E0E88BFAF750F801462046F9F76E
:1066D000C1FD0446002001990880346003B0F0BD7C
:1066E000F0B581B005460120072D66D80C4600297B
:1066F00063D04A4F38680169C90736D1052630464C
:10670000FFF75AFE304604F0E9FF03CF0369012288
:1067100013430361002918D403200B4683438E489A
:106720001E588807C00EFF278740BE43402787407A
:10673000374389481F501F20084082408748026025
:1067400087480260354800680FE08A07D20EFF26AE
:1067500096400F230B40083B03218B437D495F5834
:10676000B743402696403E435E50690140180121E0
:1067700009024218E369DB069B0CA569ED00EDB246
:10678000EB18536062685207520B23685B075B0982
:106790009A18A3685B079B0CD218E3685B075B0D34
:1067A000D21823695B01DBB2D21863699B07DB0E49
:1067B000D218802313434350002001B0F0BDC046DF
:1067C000F0B581B0002A23D005460835134C266861
:1067D000F668EE40F50702D0022001B0F0BD069D3C
:1067E0008600A619B5604001246820180093012393
:1067F0001D02461977680724A7437760F16032616C
:106800000099B160415919434151002001B0F0BDD8
:1068100003A00AA174220DA305F0A4FA909201022C
:10682000696E636C7564652F647269766572732F27
:106830006D6B5F646D612E6300000000646D615FCD
:106840007472616E7366657200000000496E766155
:106850006C6964207472616E73666572206473740F
:1068600020616464720000000001584908584068C3
:106870007047C046F0B581B005460120012D4CD8C7
:106880000C46002949D0002D03D0012D04D10F2042
:1068900000E00E20FFF790FDA668012E04D0002E28
:1068A0004FD1E08900284CD12901294843580020C4
:1068B000D860F507AD0F27686668B607360F7619FA
:1068C0002569EA07920EB618022F04D0012F03D1D2
:1068D0000122164300E040361D4F9E60E2681A60B8
:1068E00079188D606269CA604968002917D403224B
:1068F0000B469343184A9C588D07ED0EFF26AE4079
:10690000B4438026AE4026439E501F220A400121F8
:106910009140124A1160124A116001B0F0BD8A071D
:10692000D20EFF2494400F230B40083B03218B43DE
:1069300008495D58A543802494402C435C5001B025
:10694000F0BD08A00FA1492212A305F00BFAC04622
:10695000D89201021CED00E000E400E080E200E0DB
:1069600000E100E0696E636C7564652F647269769E
:106970006572732F6D6B5F6475616C5F74696D65B3
:10698000722E63006475616C5F74696D65725F6F10
:1069900070656E00636F6E66696720697320696E4B
:1069A00076616C69640000000001084A10580160BB
:1069B000816880220A4382607047C0460001034913
:1069C000085881688022914381607047D892010203
:1069D000F0B58DB0019315460E460A90129800242A
:1069E00008900480149F3C801398099004601598C7
:1069F00004900480FF2081053046F9F72BFC0290BB
:106A0000304603963146F9F7CCFB2B463D460690BF
:106A1000274607950B9311E01180188880002858AD
:106A2000099908600120079D2880052004990880A5
:106A30007F1CBCB21888844200D9A0E028880028B6
:106A4000F6D1A0000A9D2E5830460699F9F71EFE91
:106A5000002817D030460399F9F718FE00280B9B41
:106A6000079DE5D1089A1780099D2E601888011BA3
:106A7000012934D11080198889000A9A5158296057
:106A8000059035E0089A1780099806600B9B1988D5
:106A9000081B0128C0D00C96019825187E1CB0B2A6
:106AA0008542BFD389B2B2B28A420ED880000A9919
:106AB0000C5820460C99F9F7DBFD0B9B002804D1FC
:106AC00009980460089806800C94761CB0B2854240
:106AD000A8D3198889B2B2B28A42E7D9F5E70C96F1
:106AE000019962187D1CA9B216468A4205972CD2DC
:106AF000059884B2A5000A9E7259002C104609D050
:106B0000A819001F016810460C92F9F74AFB0C9A6D
:106B1000062C07D80446A81941681046F9F741FB2E
:106B20000C902046079D0299F9F7BEFD00280B9BAB
:106B300007D10C980299F9F7A9FD0B9B002800D00A
:106B400076E701202880032070E780B2AAB2824253
:106B50000FD888000A990C5820460C99F9F788FD3F
:106B60000B9B002805D109980460089805800595BD
:106B70000C946D1CA9B28E42BAD31888E5E70DB00B
:106B8000F0BD0000F0B585B001273904494D6868B3
:106B900004918843686028684749014329603907A0
:106BA000464801604648039101600024204600F0F9
:106BB000BDFD4448017849B2002902D480220A432D
:106BC000027068690290A86901903F4803683F4ECF
:106BD0007360C36833603346143B1B68F36033460D
:106BE000103B1B68336133460C3B1B6873613346B3
:106BF000083B1B68B361331F1B68F3616C62FB05C4
:106C00002C460C3C20689843206078046A688243D4
:106C10006A6030BF6A6802436A6020681843206077
:106C20002B4C02980440002901D42648017007200B
:106C30006862002000F08CFD264803990160BFF3D4
:106C40004F8FBFF36F8F1D48016070681E49086049
:106C50003068C860002C08D08C622046019A104031
:106C6000086320469043C862CC611B4801688906CE
:106C7000FCD50A242046FFF7C3FCF80229688143AB
:106C800029602046FFF7BCFC38032968814329604E
:106C90002046FFF7B5FC2868B8432860284614381A
:106CA0000068C002FAD5686804990843686005B0B6
:106CB000F0BDC0462C000040011C000080E200E056
:106CC00000E100E067000140042000501C0100408A
:106CD000FFFF030080E100E02C0200400A490A683F
:106CE0000A4802400A60FD214900094A1268515CC5
:106CF000002908D007490A6C02400A6401200006F6
:106D00000A6882430A60704700040040FFFFFF7F6B
:106D1000EC9301022000004000207047F0B583B0E2
:106D20000D4604467C26464350488719F869396A5F
:106D3000F9F7D0F9A84200D892E001950294012118
:106D4000EFF31080084002D1EFF3108272B63C4698
:106D500010343B690025062B0CD80A469A40D3060E
:106D60005B0F06D161231A4275D00D46002803D06F
:106D700003E00225002800D162B6002D02D028468B
:106D800003B0F0BD00943C462034384880591021AF
:106D9000C1613E46143604F0B7FF05463868C06945
:106DA000C00605D504F0B0FF401B31888842F5D9F4
:106DB0000621029D284600F02FFF206801994143DB
:106DC000B869091838688160172179563C4617342C
:106DD000002909D5C16920220A43C2610121F9664F
:106DE000890502680A4302600521284600F014FF65
:106DF000207840B200250028C1D42B4800687D24AB
:106E0000E100F9F767F961014143029800F0D6FE0D
:106E100004F07AFF04463868C069C00705D004F062
:106E200073FF001B31888842F5D904F06DFF0446DA
:106E30003868C169890706D504F066FF001B3188F0
:106E40008842F5D938680121009A1160534981615F
:106E5000284603B0F0BD0321216000288CD08CE7C8
:106E6000034804A1084A09A304F07CFF009301022F
:106E700080ED0000666C6173685F626C6F636B5FCE
:106E800065726173650000005D020000626C6F63F3
:106E90006B20696478206973206F76657220726157
:106EA0006E67650D0A00000090C20102F0B583B064
:106EB00002907C214143934A5418E56EEAB2511E78
:106EC00002291FD229040126090E18D0019600922A
:106ED000022100F0A1FE2746143704F015FF0646F4
:106EE0002068C169890606D404F00EFF801B39882A
:106EF0008842F5D92068007DC007019E08D0304641
:106F000003B0F0BD032A36D100922804000E36D01B
:106F100020466C302D0C002101910160274614376A
:106F200004F0F2FE06462068C069C00705D004F0F0
:106F3000EBFE801B39888842F5D904F0E5FE064651
:106F40002068C169890706D504F0DEFE801B3988F8
:106F50008842F5D9206811498161E9B201200029F0
:106F600011D003290099019E00D006202061226FD4
:106F7000002A0ED1C3E70026304603B0F0BD01263B
:106F8000304603B0F0BD0099019E2061226F002AB7
:106F9000B5D002A89047304603B0F0BD000093EB97
:106FA00070B5002801D0012070BD7825CD4E705DF0
:106FB00000280ED000240921204600F02DFE0F20CD
:106FC000FFF71EFB1520FFF7EFF9745534612046DB
:106FD00070BD042070BDC046F0B581B00C4600788D
:106FE000484EF16881422CD1032C54D1706EB16EA1
:106FF000884261D900240621204600F00DFE306849
:10700000F16D81602046214600F006FE3546603570
:107010002CCDF0683168B48C414F00975B1BA342C4
:1070200000D81C46A3081431FFF7CAFBB06E001944
:10703000B066306E00193066F06D0019F06501B071
:10704000F0BDB168814255D1032C45D1F08CF16D72
:107050000918F165316E09183166B16E0818B0660D
:10706000716E814238D900240621204600F0D4FDFB
:107070003068F16D81600121204600F0CDFD316E58
:10708000B068F38C3268264C009414329B08FFF7EA
:1070900097FB01B0F0BD30681021C16104F034FEEF
:1070A00005463068C069C00616D504F02DFE401BA9
:1070B000B18A8842F5D90FE030681021C16104F02F
:1070C00023FE05463068C069C00605D504F01CFEE5
:1070D000401BB18A8842F5D90120C1073268136884
:1070E0008B431360F16E22040A4300021043F066E2
:1070F00001B0F0BD4D200201034804A1844B04F00F
:1071000031FEC0460093010280ED0000666C6173A1
:10711000685F646D615F63616C6C6261636B0000EA
:10712000D96F0000F0B581B000786E4DAA68824238
:1071300000D0D0E001263002032942D16A6DAA6650
:10714000AB6DAC6AA418EB652C66AB6C5B1CAB64D6
:107150006B6E934235D95E30FFF752FA686CA96CBA
:1071600002293AD3814238D1E88C696D08186865E4
:107170000020062100F050FD2868E96D81602F6D28
:1071800004F0C2FD04462868C069C00705D004F0B9
:10719000BBFD001BA98A8842F5D904F0B5FD044661
:1071A0002A68D069800706D504F0AEFD001BA98AC5
:1071B0008842F5D92A687420285C012841D0F1045E
:1071C00040E0F2072B681C6894431C60EA6E0904D7
:1071D00011430143E96601B0F0BD0229FBD38142AE
:1071E000F9D2E88C696D09186965A96D0818A86558
:1071F0000020062100F010FD2868E96D8160EF8C09
:1072000004F082FD04462868C069C00705D004F078
:107210007BFD001BA98A8842F5D904F075FD044660
:107220002A68D069800706D504F06EFD001BA98A84
:107230008842F5D92A687420285C012822D0F104FC
:1072400021E03105334B3B405918012802D0192069
:10725000400601E00720C00608182F49401850607A
:10726000002F0DD004F050FD04462A68D069800735
:1072700006D404F049FD001BA98A8842F5D92A6882
:107280002B6D1FE03105234B3B40C918012802D06C
:107290001920400601E00720C00608181E494018C2
:1072A0005060002F0DD004F02FFD04462A68D069ED
:1072B000800706D404F028FD001BA98A8842F5D96E
:1072C0002A68EB8C296EA868144C00941432FFF7DE
:1072D00077FA01B0F0BD044804A10C4A0C4B04F04D
:1072E00041FDC0460093010280ED0000666C6173B1
:1072F000685F646D615F77726974655F6E627974EF
:1073000065735F63616C6C6261636B0072040000A3
:1073100067ED0000FF3F0000008080002571000045
:10732000F0B587B004460126880E14D01546002A11
:1073300011D00F468120C004401B88420BD37C2013
:107340006043F04908180590818C38460691F8F79B
:10735000C1FE002902D0304607B0F0BD284606998C
:10736000F8F7B8FE0029F6D1059880693E1A304634
:107370000699F8F7AFFE0746039670190190069E2E
:107380003146F8F7A7FE0546C01B04900598006A31
:1073900002903146F8F79EFE049981420FD20026F2
:1073A000BD42D8D92046394600F03CFB2046FFF7C5
:1073B0007DFD0028FAD17F1CAF42F3D3CBE70090CC
:1073C0000398029D2946F8F785FE06462846704335
:1073D0000399081A019800D0761C2946009D754330
:1073E000F8F778FE0590029941430198401A0390FE
:1073F0000699F8F76FFE0490AF420BD2204639464B
:1074000000F010FB2046FFF751FD0028FAD17F1C49
:10741000AF42F3D305988642069D009F0CD22046CA
:107420003146FFF77BFC2046FFF740FD0028FAD1EC
:10743000761C05988642F2D30398A84203D2002610
:10744000304607B0F0BD059847430025E9192046AE
:1074500000F0E8FA2046FFF729FD0028FAD16D1C5C
:10746000002604988542F1D375E7C046F0B585B093
:10747000002803D00124204605B0F0BD7822A14F9A
:10748000B85C002803D00024204605B0F0BD04926B
:10749000002905D0384614300CC90CC01CC91CC0CA
:1074A0000020F86615242046FEF786FF204604F0EB
:1074B00015F938681021C16104F026FC04463868CB
:1074C000C169C90607D504F01FFC001BB98A8842B0
:1074D000F5D9386800E0B98ABA7D1207120B521844
:1074E000F97DCB07DB08D2188B07DB0F5B05D218C1
:1074F000CB06DB0FDB05D2184B07DB0FDB06D21800
:107500008B06DB0F5B07D2180907C90F89071143E8
:10751000016000240A21204600F07EFB3220FFF7A4
:107520006FF80821204600F077FB04F0EDFB0546DC
:107530003868C169890606D404F0E6FB401BB98AA5
:107540008842F5D93868017D0A46C23A5342534110
:1075500074257B550904027D12025118007D0B1819
:107560000220032668A2314605F058FC785D012808
:10757000039619D1F87D029000260621304600F0CE
:107580004BFB0721304600F047FB01210298814365
:10759000785D012847D13868890101750675752124
:1075A000795C012938D048E00020032100F034FB49
:1075B00004F0AAFB06463868C169890606D404F0BF
:1075C000A3FB801BB98A8842F5D93868007D46083C
:1075D0000122F87D014631431640C90701D03040F1
:1075E00036D00295002506212846019200F014FBB2
:1075F00007210095284600F00FFB019846400298AD
:10760000385C012813D13868B10101750099017502
:107610007521795C012910D114307621795C4A42B8
:107620004A41510008E038680675490003E03868AF
:1076300000990175710014300170374800687D2190
:10764000C900F8F747FD28214143002000F0B6FAB1
:107650007720385C012803D102200021FEF73CFF8F
:1076600004F052FB06463868C069C00705D004F034
:107670004BFB801BB98A8842F5D904F045FB0646CE
:107680003868C169890706D504F03EFB801BB98ABA
:107690008842F5D93868E2498161172038560028B8
:1076A00029D57868002816D40146039A91431C4ACC
:1076B0008B588507ED0EFF26AE40B3438026AE40C3
:1076C0001E438E501F21014001208840154908604B
:1076D000154908600FE08107C90EFF228A400F2379
:1076E0000340083B039883430C481D589543802270
:1076F0008A402A431A500120049978543861204660
:1077000005B0F0BD009301026A656465635F69645A
:107710002025780D0A00000090C201021CED00E057
:1077200000E400E080E200E000E100E080B57C21C0
:107730004143A64842187823D25C002A05D040581D
:10774000024941600F20FEF75BFF80BD008020B939
:1077500080B57C2141439D4842187823D25C002AA1
:1077600005D04058024941601E20FEF749FF80BD08
:10777000008020ABF0B593B07C270A904743934834
:10778000C619980704D0F07D4024044000D017E1CA
:107790000125880E2ED0002B2CD08120C004C01AC9
:1077A000884227D309920122EFF31084144002D1BA
:1077B000EFF3108072B63046103005903069002526
:1077C00006280891069310D8079414468440E106D1
:1077D000490F04D161210C4203D0154604E0022573
:1077E00002E00221059B1960079C002C00D162B6C3
:1077F000002D02D0284613B0F0BD3446173473482C
:10780000C05910210491C1613746143704F07CFA45
:1078100005463068C069C00605D504F075FA401BFE
:1078200039888842F5D92078400665D40297B78C0C
:10783000069C20463946F8F74DFC079039464143EF
:10784000601A039035462435A74200D894E0039887
:1078500000281CD006210A9C204600F0DDF928886B
:1078600007994843089940183168886000272046E6
:10787000039C394600F0D0F9079B099A28885843A1
:10788000C0193168097D11547F1CA742F6D33068B6
:107890000499C16104F038FA0446029D3068C06959
:1078A000C00605D504F030FA001B29888842F5D9B6
:1078B00004F02AFA04463068C069C00705D004F015
:1078C00023FA001B29888842F5D904F01DFA0446E2
:1078D0003068C169890706D504F016FA001B2988AB
:1078E0008842F5D930680121059A1160B249816159
:1078F0000025284613B0F0BD03200025089FF7653A
:107900000999316606997166B566F0660120C0076F
:1079100031680A6802430A6006210A9C204600F08A
:107920007BF9306887602046294600F075F93A4FA8
:107930000BAA0A921BCF1BC21BCF1BC2B48CF068D0
:107940000A99FEF7CDFEF0683168344A0092069A33
:10795000944200D31446A3081431099AFEF730FF6D
:10796000B06E0019B066306E00193066F06D001907
:10797000F065284613B0F0BD002404E0641C0798AD
:10798000844200D363E706210A9800F045F928886D
:107990006043089940183168886000270A98394682
:1079A00000F03AF928880028099AE7D060431018B7
:1079B0003168097DC1557F1C28888742F6D3DDE7F1
:1079C000034804A1064A07A304F0CCF9009301027E
:1079D00080ED0000666C6173685F72656164000031
:1079E000C603000054686520444D412072656164FF
:1079F000206C656E6774682073686F756C642062B4
:107A00006520746865206D756C7469706C65206F95
:107A10006620340D0A000000DCE50000D96F00008C
:107A2000000093EBF0B583B00D4604467C26464338
:107A300051488719F869B98CF8F74CFBA84200D86F
:107A400094E0019502940121EFF31080084002D1E7
:107A5000EFF3108272B63C4610343B690025062BCA
:107A60000CD80A469A40D3065B0F06D161231A420E
:107A700077D00D46002803D003E00225002800D16E
:107A800062B6002D02D0284603B0F0BD00943C46FB
:107A90002434394880591021C1613E46143604F01F
:107AA00033F905463868C069C00605D504F02CF9DD
:107AB000401B31888842F5D90621029D284600F0F6
:107AC000ABF8208801994143B8690918386881608A
:107AD000172179563C461734002909D5C16920225F
:107AE0000A43C2610121F966890502680A430260FE
:107AF0000421284600F090F8207840B22C4600255A
:107B00000028C0D42B4800687D21C900F8F7E2FAAC
:107B100020492D314143204600F050F804F0F4F89C
:107B200004463868C069C00705D004F0EDF8001BB2
:107B300031888842F5D904F0E7F804463868C1690D
:107B4000890706D504F0E0F8001B31888842F5D992
:107B500038680121009A116017498161284603B0F5
:107B6000F0BD0321216000288AD08AE7034804A1E0
:107B7000084A09A304F0F6F80093010280ED000022
:107B8000666C6173685F736563746F725F65726161
:107B9000736500002B020000736563746F722069C7
:107BA0006478206973206F7665722072616E6765F4
:107BB0000D0A000090C20102000093EBF0B583B003
:107BC00001917C220290424353498C18254614357A
:107BD00004F09AF806460221029800F01DF804F01D
:107BE00093F807462068C169890606D404F08CF82A
:107BF000C01B29888842F5D92068007DC00708D0BD
:107C00006420FEF7FDFC04F07FF8801B0199884298
:107C1000E1D903B0F0BDC046F0B585B0049104468B
:107C20007C2060433C490F183D46143504F06CF845
:107C300006463868C069C00705D004F065F8801BA7
:107C400029888842F5D904F05FF806463868C0698B
:107C5000800705D504F058F8801B29888842F5D99B
:107C60001421049B5943DC2060432C4A10180390D4
:107C700002914018018A8268C47C7426BE5D012E80
:107C80000DD10191012B02990CD0012B0DD075263D
:107C9000BE5D012E0ED0019E072B0ED10EE00E46CA
:107CA00002990BE00222012BF1D138247526BE5D2A
:107CB000012EF0D10326072B00D0019E184B334034
:107CC00024069207D20A1219D218039B5958C907E1
:107CD000490C52184168CB071B0CD218837C5B07F8
:107CE0005B0BD218C0684007000A10183A68506051
:107CF000002E0ED001290CD104F006F80446386895
:107D0000C069800705D403F0FFFF001B2988884263
:107D1000F5D905B0F0BDC0460093010224E700008C
:107D2000FF3F0000F0B59DB00D460126890E2FD013
:107D3000002B2DD011928121C9041093C91AA94298
:107D400026D30121EFF310840C4002D1EFF310820F
:107D500072B67C220F904243E74814928718384647
:107D600010303B690026062B0DD80A469A40D306F0
:107D70005B0F07D161231A4200D16FE30E46002C3E
:107D800003D003E00226002C00D162B6002E02D000
:107D900030461DB0F0BD0290BD650021139179659C
:107DA0001098401E12904019B964B9690D916E1A6D
:107DB0001199B962FD6238637E63F98C0E91304689
:107DC000F8F788F90446B863129830180E9E3146C9
:107DD000F8F780F9109B011B4A1CF86339647A6438
:107DE000139A0029194608D0704359190D9BC91AD6
:107DF0000A1A7443581B80190119384648300E90EE
:107E0000384644300D90384640300B903846263086
:107E10000590384658301390384654301290F96423
:107E20003A651498B44908581021C1613846143095
:107E300014903846503004903D464C3503F064FFB2
:107E400004463868C069C00606D503F05DFF001B14
:107E5000149909888842F4D9F87D40060C9500D51C
:107E600074E201230E9803600D98016800290F98B1
:107E700000D1CDE23A4674320A92DA0407921A052A
:107E800009921922520606920722D206089216E09B
:107E90009A4800687D21C900F8F71CF91099414300
:107EA0000F9C2046FFF78AFE20460C9D0E9A116813
:107EB0004B1C13600D9909688B4200D9A8E20B9AFC
:107EC0001268012A55D0002A00D0A8E02E68129925
:107ED0000C6813990D6806211091FFF79DFE386814
:107EE00085601198051903F00FFF04463868C069D2
:107EF000C00706D003F008FF001B149909888842C8
:107F0000F4D903F001FF04463868C169890707D531
:107F100003F0FAFE001B149909888842F4D93868E6
:107F20000A990A78012A089900D00699012A099A23
:107F300000D0079A3346724C234013430B437149D8
:107F40000B434360002EA3D003F0DEFE04463868E6
:107F5000C069800706D403F0D7FE001B1499098876
:107F60008842F4D93868297801756D1C761EFAD1DB
:107F70008EE7012B00D0C7E02E6812990C68139988
:107F80000D6806211091FFF747FE3868856011984B
:107F9000051903F0B9FE04463868C069C00706D069
:107FA00003F0B2FE001B149909888842F4D903F04B
:107FB000ABFE04463868C169890707D503F0A4FE03
:107FC000001B149909888842F4D938680A990A78FC
:107FD000012A089900D00699012A099A00D0079A27
:107FE0003346474C234013430B4346490B434360FE
:107FF000002E69D003F088FE04463868C069800707
:1080000006D403F081FE001B149909888842F4D934
:108010003868297801756D1C761EFAD154E0012B61
:1080200000D0C9E02E6812990C6813990D680621DA
:108030001091FFF7F1FD386885601198051903F07C
:1080400063FE04463868C069C00706D003F05CFED2
:10805000001B149909888842F4D903F055FE0446A0
:108060003868C169890707D503F04EFE001B1499D3
:1080700009888842F4D938680A990A78012A089947
:1080800000D00699012A099A00D0079A33461C4C61
:10809000234013430B431B490B434360002E13D073
:1080A00003F032FE04463868C069800706D403F046
:1080B0002BFE001B149909888842F4D93868297866
:1080C00001756D1C761EFAD10C4800687D21C9002F
:1080D000F8F700F8109941430F9C2046FFF76EFD1A
:1080E00020460C9D2A68139B196889181960129BF9
:1080F000196889181960D9E60093010290C201023B
:10810000FF3F0000008080008B4200D0CEE6049943
:108110000E6812990C6813990D6806211091FFF7EB
:108120007BFD386885601198051903F0EDFD044664
:108130003868C069C00706D003F0E6FD001B14993B
:1081400009888842F4D903F0DFFD04463868C16924
:10815000890707D503F0D8FD001B149909888842C8
:10816000F4D938680A990A78012A089900D0069942
:10817000012A099A00D0079A3346D44C234013436E
:108180000B43D3490B434360002E00D180E603F03C
:10819000BBFD04463868C069800706D403F0B4FD0F
:1081A000001B149909888842F4D938682978017528
:1081B0006D1C761EFAD16BE6129A1268119CA618F5
:1081C000139A15688B425FD104990C6806210391BC
:1081D000FFF722FD3868856003F096FD0546386894
:1081E000C069C00706D003F08FFD401B14990988B1
:1081F0008842F4D903F088FD10900C9D3868C1695D
:10820000890708D503F080FD1099401A1499098850
:108210008842F3D938680A990A78012A089900D067
:1082200006991091012A099A00D0079A2346A74976
:108230000B40134310990B43A5490B434360002C9B
:1082400014D003F061FD10903868C069800707D42E
:1082500003F05AFD1099401A149909888842F3D9FD
:10826000386831780175761C641EFAD19A48006826
:108270007D21C900F7F72EFF039941430F9C20464B
:10828000FFF79CFC204611E605990C880621039116
:10829000FFF7C2FC3868856003F036FD0546386894
:1082A000C069C00706D003F02FFD401B1499098850
:1082B0008842F4D903F028FD10900C9D3868C169FC
:1082C000890708D503F020FD1099401A14990988F0
:1082D0008842F3D938680A990A78012A089900D0A7
:1082E00006991091012A099A00D0079A23467749E6
:1082F0000B40134310990B4375490B434360002C0B
:1083000014D003F001FD10903868C069800707D4CD
:1083100003F0FAFC1099401A149909888842F3D99D
:10832000386831780175761C641EFAD16A48006895
:108330007D21C900F7F7CEFE039941430F9C2046EB
:10834000FFF73CFC204605990A88CCE65E4815A953
:108350000A4678C878C278C878C20125E8073A6822
:10836000136803431360B868FEF7BAF902200026C9
:10837000139C2168BA6AF9653A6610997966BE66F7
:10838000F8660C980068129A1168091811600E9B23
:1083900019684A1C1A60226810182060002900D051
:1083A000F6E410953846603013903C465C3438460D
:1083B0000830129006210F98FFF72EFC38682168CC
:1083C00081600C980068119003F09EFC04463868A8
:1083D000C069C00706D003F097FC001B14990988F8
:1083E0008842F4D903F090FC0446109D3A68D069A5
:1083F000800707D503F088FC001B14990988884280
:10840000F4D93A687420385C01282DD0E9042CE0B6
:1084100003F07AFC04463868C069C00706D003F050
:1084200073FC001B149909888842F4D903F06CFC92
:1084300004463868C169890707D503F065FC001B4D
:10844000149909888842F4D938680121029A116088
:1084500022498161002630461DB0F0BD0421016033
:10846000002C00D191E491E42905119C174B234085
:10847000591801280C9D02D01920400601E0072060
:10848000C0060818124940185060002C0ED003F0A6
:108490003BFC04463A68D069800707D403F034FCFB
:1084A000001B149909888842F4D93A682B681398FC
:1084B000016812980068074C00941432FEF780F9A6
:1084C00030461DB0F0BDC0469CE50000FF3F0000F7
:1084D000008080002571000090C20102000093EB33
:1084E0003120C00001490968085870479092010284
:1084F000F0B5032920D8C0467944097949008F4452
:1085000001080F15012181404F4B1B685963D96247
:1085100012E0012181404C4B1B681963D9620BE0CA
:1085200001218140484B1B68596304E001218140CF
:10853000454B1B681963996283004349CB18DA6085
:108540008A68002A29D14A68002A16D403231446CF
:108550009C43174BE5589607F60EFF27B740BD43DF
:108560008027B7402F43E7501F23134001229A4032
:10857000104B1A60104B1A600FE09307DB0EFF25BB
:108580009D400F241440083C03229443074AA658F8
:10859000AE4380259D403543A550012282400868A6
:1085A0000262886810438860F0BDC0461CED00E0A0
:1085B00000E400E080E200E000E100E010B501240A
:1085C0002046FDF7F9FE204603F088F8002010BD94
:1085D000012181401C48006842688A43426070471C
:1085E000194909680968C140012008407047C04620
:1085F000012181401448006842680A434260704784
:10860000012907D0002910D1012181400F480268BB
:108610000A430FE0012181400B4800684368002AAB
:108620000DD00B4343600161704701218140074831
:1086300002688A43026004480068416170478B43C6
:10864000436001617047C046809301020801004009
:1086500080B5114A1170114A10708001C90101439F
:108660000F480078400108430E4909780901014389
:108670000D480078C00008430C490978890001437F
:108680000B480078400008430A4909780143C8B202
:10869000F9F73AFA80BDC046849C0102FA960102BD
:1086A000D4930102F2CF0102A9A80102859C010224
:1086B00076B50102AAA8010210B50548046805486C
:1086C000006860430449F7F71BFD201A10BDC0463F
:1086D000740000400CB7010240420F00124A072804
:1086E00009D880000F2383408140194010689843C7
:1086F0000843106070470F280AD8800020380F23E5
:108700008340814019405068984308435060704747
:10871000800040380F23834081401940906898437F
:10872000084390607047C04634000040F0B54307EE
:10873000DC0E0726A640C3089D000E4BEF187D688F
:10874000B5433E1D002908D0356001228240012931
:108750000CD1186810431860F0BD012181401868E1
:1087600088431860A24015433560F0BD18689043F7
:108770001860F0BD0C01004010B582B014460A46E6
:1087800001460498009301900820234600F092F8D7
:1087900002B010BDB0B584B014460A460146089830
:1087A00002250095019302900720234600F052F91C
:1087B00004B0B0BD70B500285BD031490A783149AA
:1087C000002A03D14A68012313434B60428803887F
:1087D0001B049A180B46183B1A60828883891B0475
:1087E0009B180C460C3C23600B46083B84681C60BD
:1087F000446903232340057CAD00EB188569AD0770
:108800002D0D5B19457C2D035B19C569AE07B60AB2
:108810009B19867CB6059B190E1F3360036A122BC9
:1088200004D107240C60541EA2410AE0032C05D198
:10883000012D03D807220A60012202E006220A6005
:108840000122114C002525700F2464012034C57CC1
:108850006D0225401B069B0BD218C3791B07DB0E4C
:10886000D21880790007C00D10184019143908601B
:1088700070BD064806A1862209A303F073FAC0461C
:10888000A0AE010218100050A2AE010250F000008C
:108890006C73705F656E67696E655F72756E000000
:1088A000506172616D65746572206973206E756CBC
:1088B0006C000000F0B58BB0109E34043ED00D4625
:1088C000D64C2140012701977F06B9423CD1114681
:1088D0002140B9423FD11C40BC4243D1119902AC66
:1088E0000027E781E780668027802782A774E174EC
:1088F0009908A181A908A1800A900997089707976C
:10890000900880B204902046FFF754FFAA480078F0
:10891000002801D00BB0F0BDAB480168C90708D1F1
:108920000168C90705D10168C90702D10168C907F3
:10893000F3D07F48019901700BB0F0BDB8480D49E4
:10894000AF22C14B03F00EFA0095B5480949B02299
:10895000754B03F007FA0092B1480649B122724BF9
:1089600003F000FA0093AE480249B2226E4B03F0C6
:10897000F9F9C04626F00000F0B58DB00392139EC1
:10898000340446D00A46A54C2140012502956F06C5
:10899000B94244D103992140B94247D11C40BC425D
:1089A0004CD11499129D04ACE1742949218200270D
:1089B000E781E780668027809908A1819108A180DE
:1089C0000B95012D01D16121CF43A7740C9002209A
:1089D0000A9009900398800880B206902046FFF71D
:1089E000E9FE75480078002801D00DB0F0BD76484A
:1089F0000168C90708D10168C90705D10168C9071D
:108A000002D10168C907F3D04948029901700DB03D
:108A1000F0BD83480D49FB228B4B03F0A3F9009274
:108A20007F480A49FC22404B03F09CF903980090D0
:108A30007B480649FD223C4B03F094F900937848AB
:108A40000249FE22384B03F08DF9C04633F0000096
:108A50008E8E0000F0B58BB0119E340447D00D46C9
:108A60006E4C2140012701977F06B94245D111463E
:108A70002140B94248D11C40BC424CD11299109FB0
:108A800002ACE174294921820021E181E180668004
:108A900021809908A181A908A1800997012F01D0FF
:108AA000712100E06121C943A1740A90032008905C
:108AB0000790900880B204902046FFF77BFE3E4866
:108AC0000078002801D00BB0F0BD3F480168C9070D
:108AD00008D10168C90705D10168C90702D1016839
:108AE000C907F3D01248019901700BB0F0BD4C4892
:108AF0000C49D522544B03F035F9009548480949F3
:108B0000D622094B03F02EF9009245480549D72299
:108B1000054B03F027F9009341480249D822024B44
:108B200003F020F942F0000070F00000868600009B
:108B3000A2AE010210B582B014460A4601460020DA
:108B40000093019004202346FFF7B4FE02B010BD4D
:108B500010B584B014460A460146002000900193E7
:108B6000029004202346FFF707FF04B010BD000069
:108B700070B50D46064604242046FDF71DFC204630
:108B800002F0ACFD0B4805600B480670002E0ED0BD
:108B90000A48016880220A437F218A43026001203B
:108BA000000307490860074908600748046000207F
:108BB00070BDC046A4AE0102A0AE01020CE400E00C
:108BC00080E200E000E100E01C100050B0B582B08F
:108BD000144602461148204001256D06A8420DD1D9
:108BE000180413D01748016000200093019006205C
:108BF00011462346FFF75EFE02B0B0BD0094FF228F
:108C00008C320748074908A303F0ACF8FF208C30EA
:108C1000421C034803490C4B03F0A4F80300FCFF7B
:108C200050F0000018F00000447374206164647216
:108C300065737320257820697320696E76616C698D
:108C400064000000081000508EF0000080B582B073
:108C50000B46014600200092019003200A46FFF7D0
:108C600029FE02B080BD0000002801D0042100E0F0
:108C70000221C64A5172411E8841800103490A6897
:108C800040239A43101808607047C04650A0005017
:108C9000F0B583B002912E49CD7A0E7B77198742C9
:108CA0004FD908990191182545434126F604BF0084
:108CB000BE19745B34490C4057033C199B07D90C0F
:108CC0006418324B1B681B7A745375196C88032621
:108CD000B60326409B079B0C9B193F2404401819A0
:108CE000029CA3061B0DC0186880012A184E13D8D9
:108CF000707B14224243307B5023434324011B19D1
:108D00009A18F37AC0181C234343D01880081E4ACF
:108D1000104007430F432F800198686001F000FF67
:108D2000A860E8681A4908403030E86028690840BF
:108D30002721715C4018286100F052FE686103B081
:108D4000F0BDFF228832034803A108A303F00AF80C
:108D5000ACB00102DFF000006D61635F63735F63BD
:108D60006F6E737472756374000000004353206962
:108D70006E646578206973206F7665722072616E0B
:108D800067650D0A00000000FF070000EC93010278
:108D90000000F0FF2820F04900220A547047C04626
:108DA000F0B581B0009314460D46074606263046BE
:108DB000FDF702FB304602F091FC26211D48475486
:108DC0000021017041708171017181704171C17028
:108DD000C17102224272C162016341638163047303
:108DE0004273C572009A561C134A168001724120C4
:108DF000C00401214903F7F7C2F95020604329015B
:108E0000081861198A00801818224A438018B2B2E3
:108E10004A438018094940180949884204D200F0A1
:108E2000B7F8002001B0F0BD064807A19A2209A3B7
:108E300002F098FFACB00102A8B0010228000802BD
:108E400001200802DFF000006D61635F696E6974E4
:108E500000000000454D206F766572666C6F770DDF
:108E60000A000000BC48C179002901D001207047E8
:108E7000007A411E88417047F0B583B002912A49BB
:108E80004B7B834248D9CB7A0C7BE31818245C4394
:108E90009B00E3184124E4041A19142401900546A8
:108EA00065430026565100925519EE882E4F0B4609
:108EB0007A1C32402D4E3688497A711A2C4E0E405B
:108EC000B618EE803740997BEF80AA88294F17406B
:108ED0004A424A4191007918274A8918A980274FA8
:108EE0000F402D1D029801280AD125490E40092165
:108EF000C902711869800121C9037918298000E02D
:108F00002F800198444300980019074A918C4182B0
:108F1000118C018203B0F0BD3520C200034804A1CA
:108F200009A302F01FFFC046ACB00102DFF0000051
:108F30006D61635F6C696E6B5F646573635F636FC4
:108F40006E737472756374004C696E6B2064657324
:108F50006320696E646578206973206F766572207E
:108F600072616E67650D0A00FFFBFFFFA8B001028A
:108F7000FF03000003D0FFFFE80F0000EF1F000019
:108F8000FF830000D54A506391637047ACB0010283
:108F9000F0B581B04348CC21016003214160CF4945
:108FA0000A7BD304404C1B19CC7AA218541E1C43D4
:108FB0001823534392009A184B7B14255D43521992
:108FC000920122430124630613434361002282621B
:108FD000C262026342638263C26342650267334BCB
:108FE0001A605A609A60324B1A601A619A61DC61A9
:108FF000304C1C62304C251D1D6325460C3D5D63C5
:109000002546283D9D632D4EDE631C645C642C4D1B
:109010002F461C379F642746143FDF64103C1C65B5
:10902000284C5C65284C9C650C369E67274CA563D4
:109030004035E563DA651A665A669A66DA661A6733
:10904000234DDD6702258561224DC561C325AD0332
:10905000CD620A63D2435A601F4A1368FF25AB43AF
:1090600026254D5DAD072D0EEB1813601B4A10230E
:1090700013601B4A1360272260238B5419498160B7
:10908000C160016121607D210901016641661649C7
:10909000C164164941641649016400F091FC01B0B5
:1090A000F0BDC04604A000500000F8FF94A000509E
:1090B00034A10050FF185A00300400400410004052
:1090C0001C2000405430004060400040B8A10050D7
:1090D00014001400FF3F3FFF04E400E080E200E0E2
:1090E00000E100E0DC05DC053F0270020133D0073F
:1090F000D007D00770B5182002F0F0FA192002F05E
:10910000EDFA0624204602F0E9FA2046FDF754F96C
:10911000D54C002525706570A5712571A570657108
:10912000E570607B14214143207B50224243E37A67
:109130001E0192195118C0181C224243891841205F
:10914000C004F7F71CF8E5712572FFF721FF70BD29
:109150002921C54A50547047ACB00102F0B58BB01C
:10916000079208910146C04FB8780991FFF784FE35
:1091700078793A7B79790691824200D89FE0FB7A30
:109180009A181823534392004124E1040491521881
:10919000D2187B7B14214B43D218502460431558BE
:1091A00001230A93DB022E469E4316504E4B2B4062
:1091B00005937D7B03914D433E7B7443F97A0B010C
:1091C0001B195B1971181C24029461435918A74B91
:1091D0001B88069C5C430919C904490D059BC918E5
:1091E000115010180799416038787979089A0092DF
:1091F0000322099BFFF74CFDF87A397B0918387870
:10920000814263D983000993049AD45C0894F721BE
:109210002140D154D1184D788E7836027619CB780A
:109220001B04F31807900A9886051E43330CCB7075
:10923000FB7A387BBC784D709E4D3540039E66436B
:10924000C018029B4343981940029B4B03405C1992
:10925000200A8870200CC870F023089D2B401B1D2D
:109260003D7B0895FE7A099D5355C8700620079AE4
:1092700050438019089A801848701F22D202224059
:109280000243100A88707879401C7871387B7979AC
:10929000814201D3002179713978491C3970F97AFA
:1092A00008183978884201D80020387028200A9997
:1092B0003954387A401C3872387A0BB0F0BDA72088
:1092C0004200D1480649074B02F04CFDA72042005E
:1092D0007A32CD487249734B02F044FDACB00102C2
:1092E000FFF00000A8F0000000F0FFFF03200006E0
:1092F00005490A6882430A600A6802430A60034813
:10930000012101607047C0461C0000401CA00050B5
:1093100080B50120FDF752FB80BD0000F0B587B09D
:1093200006930646504C607A504B1B88181A0C9DC9
:10933000A84200DC89E00F460592012E06D156486E
:109340000021C1620169554A89180160A07831463F
:10935000FFF792FDE078E178069A2B4600F0AEF830
:109360002078E1780097002206923346FFF790FCC0
:10937000E07A217B0818217888426ED94120C20406
:1093800004918800815C0391F7250D400292855479
:109390004549455C4549465C360276194449475C77
:1093A0003F04F6190127BF0537433E0C4654E67AC1
:1093B000217BA3783C4A85543E4D3D4014275F43B2
:1093C00089191C234B43D91949023B4B0B405D19AA
:1093D000290A364BC1542E0C35494654F0270399BF
:1093E0000F400599002900D13F1D217BE37A029AA5
:1093F00087542F4A86540622049E7243D21851186D
:10940000294A81541F22D20215400D43290A274AB6
:109410008154E078401CE070E07AE178814201D329
:109420000699E1702178491C2170217B0818217868
:10943000884201D806982070E079401CE071A07A3B
:10944000401CA072E07907B0F0BD3920C20016328E
:10945000074808A109A302F085FC3920C20004488E
:109460000F49104B02F07EFCACB00102A8B0010223
:10947000DFF000006D61635F747800004D414320B0
:109480005458206C656E206973206F766572207267
:10949000616E67650D0A00000804004090D003006B
:1094A00015F10000C6F000000100080202000802E9
:1094B00003000802FF07C0FF00F83F00F0B589B0C5
:1094C0000893019204914F4DEF7A874200D891E0C2
:1094D000297B502632464A434124E3040693D2189E
:1094E000CC19A10051181822059254430A19697B1E
:1094F0001423079359435318029000011958044646
:109500000390504A0A40A97AC90251180898820566
:10951000D2088A181A514C4911402A7B00965643AA
:10952000384CE57A2C0106982418A719354E5419A1
:10953000A5007D19059844432819747B079D6C4349
:109540000519049FD2194148048854432A19089CDC
:10955000D204520D51181D460398195000F04AFAD2
:109560000146707A001902043E460CD080B2C00059
:10957000002900D1801E029FA5214900F6F7AAFD0F
:109580001F21014001E00021029F38012818427983
:1095900083791B029A18C3791B04D2182C4B1340F1
:1095A000437109045918090CC171002C20D01548C9
:1095B00035460646007B009B4343F17A0A01069F2D
:1095C0003A43D21841188B00D218059B4B43D1184F
:1095D000727B079B5343C91840191C4A12884243A7
:1095E00088180199884203D001992246F6F7AEFD0A
:1095F00009B0F0BDFF225C32034804A109A302F0C8
:10960000B1FBC046ACB00102DFF000006D61635FEA
:1096100074785F646573635F636F6E737472756390
:10962000740000005458204445534320696E64651B
:1096300078206973206F7665722072616E67650DA0
:109640000A000000FF0700E000F8FFFFA8B00102D9
:10965000EFFFE0000168044A1160416851608168D1
:109660009160C068D060704780A0005082B0FCF765
:1096700093FC052000252946FFF730F806202946EF
:10968000FFF72CF80A202946FFF728F80920294679
:10969000FFF724F80124204603F0EAFC284603F0F3
:1096A000E7FCFCF7B3FC07212846FCF7A7FC01F018
:1096B00095FF01F08DFFFAF7A9FE5648016856485C
:1096C0000068890308D4032109070840210788425C
:1096D00002D0FCF7C9FB06E0FBF7DEFFFCF70AFC53
:1096E0000020FDF75DFCFCF7F9FC0025284604F09E
:1096F00025FD032049A2014603F090FB4D4E301D8D
:1097000001F0B6FDFEF75AFFF8F7C6FA30460C3006
:10971000FCF792FAF7F786FEFAF7FEFF0C20FEF749
:1097200057FF62024449454B2846009203F09EFFD2
:1097300001F07CFC424A2046214602F0D3F9E003C6
:1097400002F000FA3F48FCF763FB21464F4C2046ED
:1097500024303D4A0191FCF7E1F93C48FCF770FBED
:10976000FBF7D8FB09E00027384601F00FFC38462C
:109770003149009A314B03F079FF607A002802D01A
:109780006572FBF7A9F83078002809D035700727F3
:109790003846FEF72DFFFBF765F93846FEF718FF50
:1097A000FBF7E8FB02273846FEF71AFFA0713846A0
:1097B000FEF716FF7178002807D000290BD1E5715C
:1097C000019870701E20B07004E0012903D1019847
:1097D000B07075702572F8F711FBE0790028CCD0D5
:1097E00070781B4909780143C7D102F015FFEFF3E8
:1097F0001080C007B7D1EFF3108072B6002738464B
:1098000001F0C4FB38460C49009A0C4B03F02EFFC4
:1098100062B6B2E7180000403000014055574220C0
:1098200073696D706C65206578616D706C650D0A8B
:109830000000000018900102A8AE0102A5D80000A7
:10984000B9BA000039E10000DD5900007D98000040
:10985000E8B00102014800687047C0460C000040B3
:1098600081B080B581B0039303AB009302F050FF49
:1098700001B080BC02BC01B00847000080B50348BD
:1098800000218181FAF7B2FC80BDC046289901020F
:10989000F0B581B0002630463146FDF7E7FD0125E1
:1098A0006C022649264F30463A462346FDF762FFB2
:1098B0003988244881423ED064217E5262217E5202
:1098C00060217E524422BE52FD87BD8778227A876E
:1098D00002223A874322FA86BE83FE811A4ABA815F
:1098E0007E810A223A81C822FA80184ABA803880DA
:1098F000FE8306203885F984FF2012307884873073
:10990000B88450203E523A83EFF3108072B630464E
:109910003146FDF7ABFD00280CD12A030026304666
:10992000064D2946FDF7FCFC054A304629462346EC
:10993000FEF7F8F962B601B0F0BDC04600E00204DF
:1099400042A60102AA550000E1FF00003412000007
:109950000020704710B50024002809D0002905D048
:1099600003464A0003481946F6F7F0FB204610BDAF
:10997000E04310BDF8920102014600200A2901DAF5
:10998000C0437047014A11807047C0467C93010272
:109990000020704780B50188064A11808178064A08
:1099A0001170C178054A11700079FCF72BFA00207C
:1099B00080BDC046D6930102D8930102FCB00102DB
:1099C000044805490160152109044160034981608B
:1099D0007047C0469C30004041000800340007003A
:1099E0000748006840697047FD2040000449096845
:1099F000085C7047024800686221405C7047C046BE
:109A0000EC93010210B5064804680648006864211A
:109A1000F6F776FB0221C9434143081910BDC04641
:109A200000B1010204B101020A491A220A600A497E
:109A300048704878FF210902084A13688B43800365
:109A400080B2C018106006482021016005480160FE
:109A50000020704770200040DC93010204E400E025
:109A600080E200E000E100E0F0B5A9B016460F4644
:109A70000546C648002B024600D01A463921CC00C4
:109A80003D21C900511811918242189206D001203F
:109A90004202BE491898F6F759FB189A612011192D
:109AA00013910E21119C0A91A170002F0D9501D0E8
:109AB0000A2100E00921592317938300E1707842BD
:109AC000784113990870307810901070F17AE17431
:109AD00071785170B7789770F178D17035791571C8
:109AE00074795471B1799171F179D171317A1172BE
:109AF000717A5172B17A91727E1EF0B20021032800
:109B0000169106D870B28000A1A210586A00805A3F
:109B10001690179882001898C0181490F81E022802
:109B200004D3012E084604D89D4800E09D4803193F
:109B300018781290189DA818179028463030159064
:109B40002C4656346D2080002950974A974B149E1E
:109B500033627262B362F2623176F182139B5970A2
:109B600009229A70281841608160C16001611098D3
:109B700080008F490858F6F7B1FE012F10900F9121
:109B800004D0022F05D17F217E2004E07C217B20A0
:109B900001E05B215A20159DA984207003200C90C0
:109BA000A080012666701F200B90A8821820A87440
:109BB0000A46083A179BDA76169B129AD2184A433D
:109BC0009100189A9163B702791E8B420E9109D9C0
:109BD00078486080342068847748288277481399D1
:109BE000088339E07F2B10DD802B18D031028B42A7
:109BF0001BD071028B4227D16E49618068846F4807
:109C000013990883CF20C00025E0202B17D0402BCC
:109C10001AD1684860800420688469481BE0654860
:109C2000608006206884674815E0624860801020E4
:109C30006884624813990883C520C0000BE062481D
:109C400060800220688404E0042068848120400051
:109C50006080FF2002302882104600F005FF129835
:109C6000102806D0402808D108201499C87607206B
:109C700000E004201799887002E017980C99817011
:109C80001898169A8078C11E02290CD3022811D088
:109C900001280CD12672BA4200D900266672BA4257
:109CA00013D8F44812E00D20000211990880012019
:109CB000800201E00C9800022081BA4201D8EE48EF
:109CC00000E0FA20179988600EE0FA201799886062
:109CD000139800780028119901D0E8484880E84896
:109CE000139A1083E7480880A88CF6F759FD0026E0
:109CF000E54B3246F6F7DCFB02460B46E3493046BD
:109D0000F6F73EFCE24B3246F6F7D2FBF6F79AFD49
:109D10000746E080DF493046109A0F9BF6F730FC8B
:109D2000DD4B3246F6F7C4FBF6F78CFD7843404234
:109D3000800B608116990E98814208D90C20149FDF
:109D4000B872D648179988831220189A0EE0480AEC
:109D5000189A149F01D00D2003E0080A00D1DBE21D
:109D60000A98B872CE48179988831220F872D07872
:109D7000052844D878440079400087440227402CC5
:109D80003339C848B881C8482FE0C04690900102D6
:109D90004CE500004CE500005CE500005CE50000DF
:109DA0003AE2000041E20000307500001027000098
:109DB000FCE2000005020000FF06000004080000AD
:109DC0000A0400003604000003020000B748F881CE
:109DD000B748388013E0B748F881B7483882B748A9
:109DE00038600CE0B448B881B5481799C88306E0DC
:109DF000B4487882B448B8800B9800069064AE48A6
:109E00003881A748F880B14802882A84B048007891
:109E1000E874B0480078119F7875387D1390002859
:109E20005ED0AD490A681023DA413A600A794B796D
:109E3000CF8867801B029A186A840A7A4B7A8F7AD5
:109E4000C87A0D7B65701B029A183B04D218000675
:109E50001018179FF860487B8A7BCB7B3B771202F8
:109E600010186081087C7877487C149A9072887CFE
:109E7000D072C87C159B1874087D5874487D119069
:109E80009874C87D0A7E120212181A84887DD874CC
:109E900018464B7EC375887ECD7E2D022818B8806B
:109EA000087F4D7F2D022818F880887FB877C87FFB
:109EB000F8772020085C149D28732120085C6873C3
:109EC0002A20085C2A314D782D0228188D782D041F
:109ED0004019C9780906401818998864119801E05A
:109EE000EB7DA87C7D498B700A8080001F38C8827A
:109EF000C883139800281FD022227748825C03462B
:109F000022335B781B029A180A842422825C03465F
:109F100024335B781B029A18CA842622825C03468B
:109F200026335B781B029A188A832822825C2830A9
:109F300040780002801888846948032569A2294670
:109F400002F06CFF189F387814907B78B8780F90E7
:109F5000FA78B8791390F8791190387A1090787A65
:109F6000B97A0890099100930F980190029216987F
:109F700003901298049013980590119806901098E9
:109F80000790FAA2F8482946149B02F047FF3D4685
:109F9000643580212846F6F7F2F8B878C11E022908
:109FA0000ED3012800D18FE1022800D0ABE1169139
:109FB000149078787F225043F7494018F74907E01A
:109FC0001691149078785B225043F1494018F1497A
:109FD00041182846F6F7BAF80D9D1898C6870E3432
:109FE000324602E0641C0F2A0ADA21780029F9D0EF
:109FF000491C8907C90F91400E43C687521CF1E7DF
:10A000001699022907D31499491E012900D97DE127
:10A010004279D24901E04279CF4989180C78002D64
:10A0200000D177E1C1790E91032900D94AE1427943
:10A03000062A00D979E14921890041181191E430BB
:10A0400010900E98401E129019A800190F9000232E
:10A050001392149403E01898290600D15AE1052AB6
:10A060005AD8C0467A44127952009744455C7285AA
:10A0700098ABC04688130000E20400000C08000002
:10A08000060A0000040F00000000104130C1BD416D
:10A09000000070400000F0400000D041120C0000B1
:10A0A000140B000012120000140E00000E16000027
:10A0B000130D0000121600000E120000140B0E0A01
:10A0C00012080000101600000E0B0000D6930102CB
:10A0D000D8930102FCB0010208B1010244940102CC
:10A0E000010800004361736520706172616D6574E1
:10A0F0006572733A200D0A001693DFB2002F04D068
:10A1000019A801223946F6F733F8002C00D191E066
:10A1100019A8C019BB498AE0E8B2022867D0002715
:10A12000022867D06BE00E98022872D1E8B20228AC
:10A1300000D103461693DFB2002F04D019A80122E4
:10A140003946F6F715F8002C74D019A8C019ACA13F
:10A150006DE0E8B2022800D104231693DFB2002F8D
:10A1600004D019A801223946F6F702F8002C61D074
:10A1700019A8C0199FA15AE0E8B2022800D106230D
:10A180001693DFB2002F04D019A801223946F5F743
:10A19000EFFF002C4ED019A8C01992A147E0E8B2F9
:10A1A000022800D10C231693DFB2002F04D019A887
:10A1B00001223946F5F7DCFF002C3BD019A8C01965
:10A1C000874934E0E8B2811E4A424A41970002289A
:10A1D00004D119A801223946F5F7CAFF002C16D080
:10A1E00019A8C0197CA12246F5F7B0FF0FE0062799
:10A1F000022804D119A801223946F5F7B9FF002C2D
:10A2000005D019A8C01980492246F5F79FFF169777
:10A2100010E01693DFB2002F04D019A801223946AE
:10A22000F5F7A6FF002C05D019A8C01973492246DE
:10A23000F5F78CFF3C193F2C05D80F98C019402129
:10A24000091BF5F79CFF12980228189801D20020EC
:10A2500002E0C078411E884115990870611E2E46A3
:10A26000E8B202280CD1179A517019A9119AB8C9ED
:10A27000B8C2B8C9B8C2B8C9B8C2B8C9B8C20DE086
:10A28000179A117019A9109AB8C9B8C2B8C9B8C23A
:10A29000B8C9B8C2B8C9B8C2C10709D18007354624
:10A2A000149C139A169B00D4D5E602208543D2E66F
:10A2B000FE20354605401898149C139A169B2906D3
:10A2C00028D0CCE637A231E01691149078780B991B
:10A2D0004143334808181F386F21C9430D9D7A1830
:10A2E0000378D427D3554378D827D3558378DC27F0
:10A2F000D355002900D170E6C378E027D35510313B
:10A30000001D189FEBE70120404A10E00024002DBB
:10A3100000D087E629B0F0BD80290ED30F20B87297
:10A32000104817998883102020E525A201200146B6
:10A3300002F074FD189829B0F0BD1020402904D314
:10A34000B8720849179B998310E5B87204481799A9
:10A35000888314200AE5C04641E200003AE200008A
:10A36000150F0000140B00000108000025642025D3
:10A37000642025642025642025642025642025642C
:10A380002025642025642025642025640D0A000012
:10A390009BFA00001DF7FFFFB3F1000089FBFFFFF0
:10A3A000A3F900007472785F6D6F6465207061724C
:10A3B000616D65746572206572726F720D0A0000BE
:10A3C0004E73666420706172616D6574657220659C
:10A3D00072726F720D0A0000FFFFFFFF01FF0000A5
:10A3E000FCE50000FFFFFFFFFF0101FFFF01FF0190
:10A3F000FFFF01FFFFFFFF01FFFF01FF00E800007B
:10A40000FFFF01FF1CE600006CE5000051F10000B9
:10A41000002800D101481D49086070479090010252
:10A4200010B5002801D0044601E018480468204611
:10A4300000F006FC204600F021F80B4841780B4A5A
:10A440001A23136041704078FF210902084A1368FB
:10A450008B438007000CC018106006482021016063
:10A460000548016010BDC046DC9301027020004029
:10A4700004E400E080E200E000E100E0F0B586B036
:10A48000002805D10148006802E0C046EC930102B3
:10A490003121C900049141188A791F231A40CD79CE
:10A4A000ED06AD0DAA180D7AED066D0C52194D7A18
:10A4B000ED062D0B52198D7AED06ED095219CD7A64
:10A4C000ED06AD0852194D7CED075219BD4C2260C6
:10A4D0000A7B1A404E7BF606B60DB2188E7BF60646
:10A4E000760C9219CE7BF606360B92190E79F6068B
:10A4F000F60992194E79F606B608921962604A6A10
:10A50000B14D2A40A2608A6A2A40E2602D22D20020
:10A5100087183A7E1A4003937E7EF606B60DB2186F
:10A52000BE7EF606760C9219FE7EF606360B921962
:10A530003E7FF606F60992197E7FF606B608921956
:10A540000E7CF60792192261BA7F1A400597FE7FAA
:10A55000F606B60DB218049BC35CDB065B0CD21882
:10A560004B78DB061B0BD2188B78DB06DB09D21885
:10A57000CB78DB069B08D2186261CA692A40A261C7
:10A580000A6A2A40E2618A7C01252A40CB7CDB07EB
:10A590009B0F9A180B7DDB075B0FD2184B7D9B0737
:10A5A000DB0ED2188B7DDB079B0ED218CB7D1B07F1
:10A5B0009B0D9A180B7E1B079B0CD2184B7E5B06DB
:10A5C000DB0A13438A7E520612091A43CB7E5B07CD
:10A5D0005B0813432362CA6A62620A6BA2624A6B17
:10A5E000E2628A6B22633922D200835C1E462E40CF
:10A5F00066635E425E41B304AE04744F3C68B4438C
:10A60000E3183B6083185A782A409C782407E40EAC
:10A61000A2188C8F6401A2186D4C1440C98FC90513
:10A62000490A0919DA78D207120A89181A79120721
:10A63000120989185A79D207D2088918FB4EB163DA
:10A640009968F163997904952940DA79D207920FD4
:10A6500051181A7B5207D20E89185A7BD206920DD6
:10A6600051189A7B5207D20C8918DA7BD206920BCA
:10A6700089181A7CD206520A89185A7C5207920904
:10A680000A43997CC906490851183164D97C039A58
:10A6900011401A7DD206920D51185A7DD206520CE5
:10A6A00089189A7DD206120B8918DA7DD206D20952
:10A6B00089187164197E0F2421405A7E12015118A5
:10A6C0009A7E12038918DA7E1207120A51181A7F2D
:10A6D0001207120989185A7F12078918B164997FE5
:10A6E00001942140DA7F1207120E51183D22D20048
:10A6F000835C5B075B0D5918841862781207520C53
:10A700008918A278D206120B8918E278D206D209EB
:10A710008918F164217907220A406179C9008918F2
:10A72000A2795206920B5118E2799207120B8918FE
:10A73000227AD2078A18BF490A60627AA37A1B027A
:10A740009A18E37A1B04D2184A60E289BA4B134084
:10A750000394228AD2049209D2188A6003463033C5
:10A76000598CB64A114002939A8CD205D20A5118DC
:10A770005622825C12068918B14D29600146563175
:10A780004A788C782402A2188C8864056409A2187F
:10A79000CC78240712196A60CA880C7AA407A40B23
:10A7A000A2184C7A6407E40A1219AA604989E96080
:10A7B000492189004118FF22663282180092103523
:10A7C000002207E000300040FFFFFF0004040040CB
:10A7D000FF3F000084186427E65D03273E406523A1
:10A7E000E35C9B071B0F9B196626A65DB607B60E9A
:10A7F000F3186726A65DB601F318DBB26826A65DDE
:10A80000B607B60DF3186926A65DB607360DF31820
:10A810006A26A65DB607B60CF3186B26A65DB607CA
:10A82000360CF3186C26A65DB607B60BF3186D262A
:10A83000A65DB607360BF3186E26A65DB607B60AF8
:10A84000F3186F26A65DB607360AF3187026A65DC4
:10A85000B607B609F3187126A65DB6073609F318D0
:10A860007226A65DB607B608F3187326A45DA40782
:10A87000E31808C51032802AACD1019AD243704E39
:10A88000B4180B783B404D78AD072D0FEB188D7841
:10A89000AD07AD0EEB18CD78AD01EB18DBB20D793D
:10A8A000AD07AD0DEB184D79AD072D0DEB188D797A
:10A8B000AD07AD0CEB18CD79AD072D0CEB180D7A6B
:10A8C000AD07AD0BEB184D7AAD072D0BEB188D7A5C
:10A8D000AD07AD0AEB18CD7AAD072D0AEB180D7B4D
:10A8E000AD07AD09EB184D7BAD072D09EB188D7B3E
:10A8F000AD07AD08EB18CD7BAD07EB18A3641031A5
:10A90000121DBDD1009B19785A785207520D51186B
:10A910009A78D207120D8918B164059B1968F16401
:10A92000D97D5A681202511831659968454A0A4022
:10A93000998A490589187165D9683D4C2140B165EE
:10A9400019692140F165029E3178049D2940827881
:10A950005207120F5118C2799207920E8918427A43
:10A960009207920D5118827A9207120D8918C27AB5
:10A97000D207920C89189A7DD207520C89187278E6
:10A980009207D20B8918B2781207D20A8918F27886
:10A990001207D2098A182C490A60327C737C1B0783
:10A9A0001B0D9A18B37C9B069B0BD218F37C1B07DC
:10A9B0009B0AD218337DDB065B09D218737DDB0757
:10A9C0001B09D2184A60B27D2A40C38F5B009A18D7
:10A9D0008A60826CCA60C26C22400A61F27D7F2369
:10A9E0001340328C5204520AD2184A6102698A61B9
:10A9F0004269CA6182690A62C2694A62026A8A62FB
:10AA0000426ACA62826A0A63C26A4A63039A927C91
:10AA1000D201121D0A64027A3A40CA65808F074A41
:10AA200010400866002006B0F0BDC046003000406F
:10AA3000FFFFFF009C300040FF1F0000FF030000ED
:10AA400000400040FFFF1F00002000400448006855
:10AA5000806B800803490968490040180930704735
:10AA6000EC9301021004004010B52D21C9004118DB
:10AA7000027A032A04D10079002807D0082006E0D2
:10AA80008378DA1E022A05D2032412E0142088609B
:10AA90001C203DE0012B02D1C8228A6012E004791B
:10AAA000042C01D3462404E0032C01D1322400E01D
:10AAB00014248C605B1E022B04D3022A10D242792C
:10AAC000154B01E04279154B9B181B78402B04D0A5
:10AAD000102B06D11423442405E02A233E2402E04F
:10AAE0004279342348244B800C80022A06D0062A5F
:10AAF00008D0052A08D118224C2301E01422502343
:10AB00000B8000E01C224A80C078042803D1142066
:10AB100048806420088010BD41E200003AE2000055
:10AB2000424800687047C04610B53F4A10709170A7
:10AB30003E49002813D0506808610420486190788D
:10AB4000FF2212023A4B1C689443800380B2001922
:10AB5000186001204007054A1060364A1060002046
:10AB60000860354901220A6010BDC04680E200E05D
:10AB70003148002101602D48016802688A420BD0EB
:10AB8000016802688A4207D0016802688A4203D0DD
:10AB9000016802688A42EFD17047C046F0B581B0C3
:10ABA00021480178214D002911D08178FF2212021D
:10ABB0001F4B1C689443890389B20919196001214C
:10ABC00049071C4A11604068286104206861012718
:10ABD000EFF310803840009002D1EFF3108072B68E
:10ABE000154807602E682868B04208D12868B0422E
:10ABF00005D12868B04202D12868B042F3D0FDF7F1
:10AC00005BFD0446F5F7B1FD0C49F5F723FBF5F7BD
:10AC100004FE3018B84328600098002800D162B6BE
:10AC2000204601B0F0BDC046DC930102180400408C
:10AC30001CE400E000E100E07000004080096E4587
:10AC4000F0B591B0002801D1C04800688778F91E9E
:10AC5000022913D3012F21D0022F3CD11021CA4346
:10AC600044782146193991423DD800970125B94AC7
:10AC700028462946234602F0D1F853E10821CA4369
:10AC8000447821462139914218D800970125B14ACC
:10AC900028462946234602F0C1F843E10821CA4369
:10ACA000447821460939914234D800970125A94AB0
:10ACB00028462946234602F0B1F833E1032F3CD061
:10ACC000042F43D1C3780125042B00D02DE1064683
:10ACD0002A02042343E00125A6A2284629463B4632
:10ACE00002F09CF81EE1C3780125052B0AD8064620
:10ACF0002A02284698401B21084230D10021052B0A
:10AD000008462ED002200090914A2846294602F09B
:10AD100085F807E10646C3780021022B1ED3032BDA
:10AD20001CD0042B08460A461BD001250095884AF2
:10AD30002846294602F072F8F4E0C3780125032B77
:10AD400000D0FAE006462A02032308E0012583A288
:10AD5000284629463B4602F061F8E3E00A46012115
:10AD600048020F91592189007518FD214900711879
:10AD70000291314662313F05D219641E1F272740D8
:10AD80005C013C191443044332795207D20C22432C
:10AD90002B789B065B0BD218B379DB071B0B134395
:10ADA0006D4D2B60F279032310931A40737A9B0741
:10ADB0009B0E9A18B37A5B07DB0D9A18F37ADB07C0
:10ADC0009B0DD218337BDB075B0DD218737B1B07FF
:10ADD0005B0CD218AA603269EA6072692A61B269B2
:10ADE0006A61F269AA61326AEA61726A2A62B26AC7
:10ADF0006A620F980870F06AA8623F20C4432C353D
:10AE00003046E4300F903046E5300E903046E63064
:10AE10000D903046E7300C903046E8300B903046CD
:10AE2000E9300A903046EA3009903046EB3008901D
:10AE30003046EC3007903046ED3006903046EE302C
:10AE400005903046EF3004903046F030039037469E
:10AE5000F1373046F230F3360F990A194021525C2F
:10AE6000109B1A400E9B1B195B5C9B071B0F9A18CB
:10AE70000D9B1B195B5C9B079B0E9A180C9B1B1967
:10AE80005B5C9B019A18D2B20B9B1B195B5C9B0706
:10AE90009B0D9A180A9B1B195B5C9B071B0D9A184C
:10AEA000099B1B195B5C9B079B0C9A18089B1B1941
:10AEB0005B5C9B071B0C9A18079B1B195B5C9B0731
:10AEC0009B0B9A18069B1B195B5C9B071B0B9A1824
:10AED000059B1B195B5C9B079B0A9A18049B1B191B
:10AEE0005B5C9B071B0A9A18039B1B195B5C9B0707
:10AEF0009B099A183B195B5C9B071B099A1803195D
:10AF00005B5C9B079B089A183319595C8907891861
:10AF100002C51034A0D102980078042101430E48E4
:10AF2000C1630025284611B0F0BD04200090084AF6
:10AF30002846294601F072FFF4E703200090044AF6
:10AF40002846294601F06AFFECE7C046EC9301026F
:10AF500026F100006CF1000000100040556E6465A1
:10AF600066696E6564206D65616E205052462025CD
:10AF7000640D0A00496E76616C6964206D65616ECE
:10AF8000205052462025640D0A000000B0B584B060
:10AF90000446FBF75EF81F48016800914168019183
:10AFA00081680291C0680390FFF7E2FD00F0FCFDAC
:10AFB0001948016804220A430260184D6868A021FC
:10AFC000002C01D1884300E008436860FF20023074
:10AFD000FBF772F9FBF7D6FD0020FFF721FAFEF729
:10AFE00089F86846FEF736FB0D480168C907FCD0B2
:10AFF000012080022968814329600A48FBF75CF937
:10B00000FFF7CCFD4B49086000F0ECFDFBF726F89C
:10B0100004B0B0BD80A0005010ED00E02C00004056
:10B020002C020040010200007047704780B50E49B5
:10B030000E480246083A1268920000D46031426815
:10B040000A4342600A490A6808239A430A60091FB2
:10B05000012252040A600321890402688A430260C3
:10B06000FBF72CF880BDC04620000080280000407F
:10B0700004020040B0B5032000072D490A6882434E
:10B08000012568071018086000242046FFF7CDFF4F
:10B090002046FFF7C9FFEFF31080284002D1EFF3FD
:10B0A000108172B68021C943224A53680B40536015
:10B0B00093680B409360D3680B40D36013690B40D7
:10B0C000136153690B405361002800D162B6B0BDD3
:10B0D00070B50C4603210907154A13680B4313602A
:10B0E0000122EFF31081114002D1EFF3108272B60A
:10B0F0008025EA430F4B5E6816405E609E682E43D3
:10B100009E60DD681540DD601D6915401D615D694B
:10B1100015405D61002900D162B6002802D00120EF
:10B12000FFF783FF002C02D00120FFF77DFF70BDE9
:10B1300000040040789501020D4A002907D001293A
:10B140000BD10121814010688843106007E0012184
:10B15000814010680843106001E001218140101F08
:10B1600002680A430121C907114301607047C046C4
:10B170004400004070470000042801D901207047B6
:10B1800003498140524802688A43026000207047A8
:10B1900000000108F0B581B004460120042C62D8FB
:10B1A0000D4600295FD0287900072968C907C90919
:10B1B0000F186879FF2670436421F4F78BFF0006AF
:10B1C000000C3918A000294FC219243A1160032C31
:10B1D00031D801A108588746E9B10000F9B1000053
:10B1E00011B2000021B20000A87946432D20C10011
:10B1F0003046F4F76FFF07E0A87946432D20C100E1
:10B200003046F4F767FF000439680143396012E003
:10B21000A87946432D20C1003046F4F75BFF07E0D4
:10B22000A87946432D20C1003046F4F753FF0004AF
:10B2300079680143796001210B46A340381F0268F9
:10B24000EE79002E01D01A4300E09A430B04A3408C
:10B250002D7A002D01D01A4300E09A43C906A1407F
:10B2600011430160002001B0F0BDC0462430014010
:10B27000B0B5044612252846FBF79EF8284600F094
:10B280002DFA002C07D0227810490A7060780871D6
:10B2900063688B6002E00D4908790A7801210B038D
:10B2A0001207120DD2180A4B1A6000280BD0094859
:10B2B0000268802313437F229343036008040649F6
:10B2C0000860064908600020B0BDC046D095010264
:10B2D0002030014010E400E080E200E000E100E006
:10B2E000032804D840000649085A00B270470020DD
:10B2F00000B27047032802D84000014A115270473B
:10B300006EB501029E4908707047C04670B58AB09C
:10B310000C460546FF20FC30A8490E68315C5920D8
:10B320008000335CB278307808AE069609AE059698
:10B330000C4E04962126760603960B4E02960126A5
:10B3400001960E2600965B1CDBB2F8F775F809989B
:10B35000F5F74AFA28700898F5F746FA20700AB00F
:10B3600070BDC0460000204100000443F0B58BB022
:10B370000446457C824800788249002822D000207B
:10B380000880814A1080814B01269E761E830A9098
:10B390007F4800787F4E36786DB205957E4D0495D6
:10B3A0007E4D03950AAD02957D4D01950096F7F708
:10B3B00081FD0A9D112020567A497B4A00F0E4FB6A
:10B3C000064626E000260E806F4A16806F4B01204D
:10B3D0009876188309966E4800786E4F3F786DB264
:10B3E00005956D4D04956D4D039509AD02956C4D18
:10B3F00001950097F7F75EFD099D112021567F20EA
:10B40000C005009001900296664A674B3046F8F7F7
:10B41000A5FE432001062846F4F71CFFF5F7E4F9E2
:10B42000089062480078002824D0512080006049AC
:10B430004A7D42438D185F480068A8642F46403714
:10B4400050480078B87450480078F874554800782F
:10B45000387555480078787557480078F875504821
:10B460000069F5F7C1F9B87552484069E8644C487D
:10B4700000686864FF20FE3050490968085C392282
:10B48000D2008918022812D303D04E480078012830
:10B490000DD14B480660434800883A4A1080424824
:10B4A0000088394A108009200790089605E0444832
:10B4B000089A02603548C08B07900B780022002B59
:10B4C00001D0114600E0D1430125002B01D0042317
:10B4D00000E0EB43A67AAD1BEE175B19714165687E
:10B4E000AE0F277AAD00ED195641677A3F1FF81766
:10B4F000ED1970414000EE0F80196D00EB184841C6
:10B500008001990E4118980127239B02C31A91418B
:10B510001D4805881B480088854201D00798421BBA
:10B5200010202056C001194D2D8C032D07D1E46841
:10B53000E5176D0A6419E4150519EC170FE0E468C6
:10B54000E5176D0A6519EC17ED15C6174519744115
:10B5500097B2002F00D03446002F00D00546581B6C
:10B56000A141130409D012B2D2015242D31780185C
:10B570005941089BDA17C01A91410BB0F0BDC04683
:10B580007E9301024CA801024AA8010244940102E0
:10B59000819001028090010234A00102349E0102D8
:10B5A00050A801029AA8010298A8010200A4010271
:10B5B00038A101026420004048A80102EC93010276
:10B5C00044A80102A8A80102C10D400280307047C2
:10B5D0000120C0071B4908607047C04610B51948D4
:10B5E0000068C10710D1810711D4410712D40107A7
:10B5F00013D4C10614D4810615D4410616D4802173
:10B60000084016D031A215E001240FA213E0022455
:10B6100011A210E0032414A20DE0042416A20AE0F3
:10B62000052419A207E006241CA204E0072421A295
:10B6300001E0254A04090220032101F0EFFB204626
:10B6400010BDC0465C00004052657365742062798D
:10B6500020504F520D0A00005265736574206279C4
:10B6600020424F520D0A00005265736574206279C2
:10B670002050494E0D0A00005265736574206279AE
:10B68000205744540D0A0000526573657420627996
:10B69000204C4F434B55500D0A0000005265736516
:10B6A00074206279205357205265626F6F740D0ABF
:10B6B000000000005265736574206279205359536D
:10B6C0005245510D0A000000DEED00005265736521
:10B6D0007420627920445644440D0A0001218140BF
:10B6E000044A1F2802D0106888431060106808437D
:10B6F000106070471C000040F0B583B00291044612
:10B700009949F4F7E7FC0546984901942046F4F777
:10B71000E1FC974946189749714300956F1896497F
:10B72000441864212046F4F7D5FC3818A108471ABC
:10B7300092492046F4F7E4FC381891494518914F96
:10B7400005D464213046F4F7C5FC0C4614E0A6B2DB
:10B7500064213046F4F7BEFCB7204000A20701D1B7
:10B76000002907D1884B73430422D341874A93426F
:10B7700000D3401E0C4645190098474302980680A6
:10B78000192001013046F4F7A5FC2A461F3A284645
:10B7900000DB1046019BFF18B30705D1002C03D036
:10B7A0001F2D05DA0120C5E01F2D0BDA0120C1E0B5
:10B7B00005461D3D034600DB2B461C2808DC022005
:10B7C0001546B7E000290CD01C21451A0CD50CE019
:10B7D00019461F39184600DB08461F2B1DDA0320C7
:10B7E000A8E01D21451A00D42846002D08D40146A2
:10B7F0001F39024600DB0A461F2804DA032099E0BD
:10B800000220154696E015461E3D104600DB2846F0
:10B810001E2A0CDA04200D468CE005461E3D024629
:10B8200000DB2A461E280BDA04200D4682E0014682
:10B830001F39024600DB0A461F280ADA052079E094
:10B8400011461F39104600DB08461F2A0BDA052077
:10B8500070E015461E3D104600DB28461E2A0CDA15
:10B8600006200D4666E005461E3D024600DB2A46E0
:10B870001E280BDA06200D465CE001461F39024601
:10B8800000DB0A461F280ADA072053E011461F3959
:10B89000104600DB08461F2A0BDA07204AE015464F
:10B8A0001F3D134600DB2B461F2A0CDA08200D46ED
:10B8B00040E005461F3D024600DB2A461F280BDA02
:10B8C00008200D4636E019461E39184600DB0846AA
:10B8D0001E2B0ADA09202DE011461E39104600DB26
:10B8E00008461E2A0BDA092024E01F28054601DB42
:10B8F00005461F3D1F280CDA0A200D461AE01F28B6
:10B90000054601DB05461F3D1F2806DA0A200D46C5
:10B9100010E01E2D05DB0C2004E01E2D06DB0C20A4
:10B9200005E00B201E2D05DB1E3D03E00B201E2D28
:10B9300000DB1E3D029EB070681CF070E12001012A
:10B940003846F4F7C7FB3071C0B211494143CC19F6
:10B950003C212046F4F7BEFB70713B21C9434143B3
:10B960000819B07103B0F0BD805101008033E101CE
:10B97000B207000093FEFFFFB107000070FEFFFF5B
:10B98000A7FA0A0080AEFEFF295C8FC20BD7A30086
:10B99000F0F1FFFFF0B581B00446FFF76BFBA08A22
:10B9A000424EB085B18D002909D0F0850220F07299
:10B9B00000203083FFF7B4F8706301B0F0BDE08A77
:10B9C0003083A169328B1248F4F7C0FB2046FFF7A1
:10B9D000CDFC05460C460F48007BFFF781FC81B289
:10B9E000C90B401800B2C11740100B4F281AB8619C
:10B9F0008C41FC61FFF794F830637868401C7860F4
:10BA0000FEF700F870670120F07201B0F0BDC0468B
:10BA100078B5010282900102C8980102F0B581B0A8
:10BA2000EFF3108072B600200146FBF71FFD0446BD
:10BA3000002803D062B6204601B0F0BD01273A03CA
:10BA40000025074E28463146FBF76AFC7B02054A73
:10BA500028463146FCF766F962B6204601B0F0BDD3
:10BA600000E0020442A60102F0B51048418A022912
:10BA700011D30F4A931C012404E09B1C641C8C42CC
:10BA800035460CD2EEB27600965B1F88B74226464A
:10BA9000F3D32E46F1E70022002905D002E0F2B2EE
:10BAA000002901D00349895C4172F0BD049701026D
:10BAB00094C201027CC6010210B5084901204872F7
:10BAC0000A7A531C0B72064A9478DBB2A34202D165
:10BAD000C87100230B72107010BDC0462899010276
:10BAE0001890010270B514460D4606461120FAF76B
:10BAF00063FC2248042101600C4804601E48056074
:10BB00008660002E0DD0FF20000609490A68824396
:10BB10000120C00710180860064808210160064887
:10BB200001601A200221FFF707FB70BD10B7010268
:10BB300000E400E080E200E000E100E00C49086081
:10BB40007047C04610B5044609480068604309497B
:10BB5000F4F7D6FA00190849486008480022026044
:10BB600002460C3A4B6813600968016010BDC0467C
:10BB70000CB7010240420F000C9001022C10014052
:10BB800000480047C100000080B582B013460A4655
:10BB900000900348011D0348F8F78CFA02B080BDFD
:10BBA0004CB70102689D01023B4800210160816899
:10BBB0004068401C534A13685B0104D400290246C4
:10BBC00009D00A4607E04D490B685B1C0B60012158
:10BBD00049061160024649494860801ACA688018BF
:10BBE000C860704770B5454E71682748821C914205
:10BBF0002AD2491E284A516028490B680340032075
:10BC000084071B190B60002191601060FCF754FD44
:10BC1000054674682146F4F75DFAF1684919224631
:10BC20004243891AF160A14204D3091B401CA1427E
:10BC3000FBD2F160316809183160002803D0306907
:10BC4000002800D0804770BD10481149E622114BF2
:10BC500000F088F810B50C498A1C90420DD2401EA5
:10BC60000D4A50600D4803680B4003218C071B19D7
:10BC7000036000209060116010BD04480449E62272
:10BC8000044B00F06FF8C046FFFFFF00B5ED000069
:10BC9000CFED00009BED000010E000E020ED00E0A3
:10BCA000B0B50120EFF31081014002D1EFF3108213
:10BCB00072B6124A1368124C2268646885061148ED
:10BCC00000682840850E5D192923DB006B43002C9A
:10BCD0001D4606D1002809D11E20684300290AD03C
:10BCE000B0BD121BD218551C0028F5D01D461E20D1
:10BCF00068430029F4D162B6B0BDC0467CC20102DF
:10BD000014E000E004ED00E080B50020FAF7ACFD9F
:10BD1000404280BDB0B586B0104869460A4638C872
:10BD200038C238C838C200242046FAF7A3FD039968
:10BD30002046FAF739FE0198012803D0082400288C
:10BD400004D102E00424002800D104460220FAF7BE
:10BD50003BFBE0400249086006B0B0BD48E200008D
:10BD600090C2010290B01C4605AB07C3EFF31080F0
:10BD7000C00702D1EFF3108072B6EFF310800B9082
:10BD800068460E907046089010AB0F93CF4F3E1D43
:10BD900001200490C50230462946224600F0B8FC36
:10BDA00000213154EFF303800990EFF308800C90E9
:10BDB000EFF309800D90EFF314800A9000F02CFC53
:10BDC0003868012833D80028C14F00D0C14F2A203D
:10BDD000C1497A69920703D50A783A60401E491C26
:10BDE0000028F6D1B948041D2046F4F7D3F90028FD
:10BDF00007D079698907FAD521783960401E641C1B
:10BE0000F5E70220B5497A69920703D50A783A60C6
:10BE1000401E491C0028F6D12A20AF497A699207B2
:10BE200003D50A783A60401E491C0028F6D1FFF776
:10BE300037FF0346AA4A30462946FDF711FD04465E
:10BE40003018291B089F3B1F049A9343A5A2FDF7B6
:10BE500007FD9E490968012966D8001900299C4CF4
:10BE600000D09C4C00280AD09849091D62699207AD
:10BE700003D50A782260401E491C0028F6D10A200A
:10BE80009F496269920703D50A782260401E491CC7
:10BE90000028F6D10598F4F77DF9002809D06169EA
:10BEA0008907FAD5059A11782160401E521C059227
:10BEB000F3E7022089496269920703D50A78226074
:10BEC000401E491C0028F6D10A208EA16269920703
:10BED00003D50A782260401E491C0028F6D1069836
:10BEE000F4F758F9002809D061698907FAD5069A4C
:10BEF00011782160401E521C0692F3E70220774918
:10BF00006269920703D50A782260401E491C002806
:10BF1000F6D10A207EA16269920703D50A782260D1
:10BF2000401E491C0028F6D17CA230462946079BBA
:10BF3000FDF796FC6549096801290E9B1BD800296D
:10BF4000634900D0634900280AD0604A121D4C6939
:10BF5000A40703D514780C60401E521C0028F6D1AB
:10BF600002205E4A4C69A40703D514780C60401E79
:10BF7000521C0028F6D16AA230462946FDF770FC13
:10BF800004463018291B694A3B46FDF769FC4F49B6
:10BF90000968012911D8001900294D4900D04D49DF
:10BFA00000280AD0494A121D4B699B0703D5137814
:10BFB0000B60401E521C0028F6D15D4A30462946CF
:10BFC000099F3B46FDF74CFC0446F800C00FB90042
:10BFD000C90F7A00D20F0092019102903019291BEB
:10BFE000FB0F544AFDF73CFC04193019291B3F2371
:10BFF0003B40514AFDF734FC34490968012911D806
:10C0000020180029324900D0324900280AD02F4A8E
:10C01000121D4B699B0703D513780B60401E521C01
:10C020000028F6D1454A304629460B9BFDF718FCFF
:10C0300004463018291B424A0A9BFDF711FC23498C
:10C040000968012911D800190029214900D0214986
:10C0500000280AD01D4A121D4B699B0703D513788F
:10C060000B60401E521C0028F6D1364A3046294645
:10C070000C9BFDF7F5FB04463018291B324A0D9B3B
:10C08000FDF7EEFB114909680129114A0DD8001985
:10C09000002908D00F4A06E05169890703D5317895
:10C0A0001160401E761C0028F6D128490E98091A06
:10C0B000A94200D32946890800F03AFE24480068C6
:10C0C000002800D0804700F045F8C04648C701026C
:10C0D0000090014000A001400FEE000090F1000030
:10C0E000F8ED00000D0A23232320415353455254F9
:10C0F000204020307825303858202323230D0A0093
:10C10000D2EE000046554E4354494F4E3A200000AF
:10C110004C494E45202020203A2000002564000094
:10C120000D0A53503D253038580D0A0097EE000097
:10C13000ADEE0000B9EE0000A1EE000056EE0000EA
:10C1400065EE000074EE00007FEE000000F80202D1
:10C1500044C70102F7480068012811D8002801D01F
:10C160000B4800E0FC480C210A4A01E0002907D0F6
:10C1700043699B07FAD513780360491E521CF5E703
:10C180001E20FFF7ABFA00BF00BF00BF00BFFAE7F9
:10C1900000A0014002EE00008AB00646E448B06606
:10C1A00000F03AFAFFF77CFD0346E248041D012047
:10C1B0000590C502E04A20462946FDF751FB074697
:10C1C00008942018DB4C0995E91BF36C3F2206927A
:10C1D0001340DAA2FDF744FB2168012910D8C019E9
:10C1E0000029DD4900D0DD49002809D0221D4B6916
:10C1F0009B0703D513780B60401E521C0028F6D114
:10C20000F36BD7A2089C2046099D2946FDF728FB21
:10C210000746291A2018336C069A134007D1D8A272
:10C22000FDF71EFBC34C2168012907D917E0CEA2F8
:10C23000FDF716FBBF4C2168012910D8C019002951
:10C24000C54900D0C549002809D0221D4B699B076C
:10C2500003D513780B60401E521C0028F6D100272E
:10C26000CBA5B80030580090089809992A463B465B
:10C27000FDF7F6FA216801290FD80029B64900D048
:10C28000B649002809D0221D4B699B0703D51378B6
:10C290000B60401E521C0028F6D17F1C0D2FE0D1F0
:10C2A000736BBFA2089C2046099D2946FDF7D8FA6A
:10C2B000074620189F4CE91BB36BBC4AFDF7D0FA28
:10C2C0002168012910D8C0190029A34900D0A34929
:10C2D000002809D0221D4B699B0703D513780B60FA
:10C2E000401E521C0028F6D1336CB14A089C2046EF
:10C2F000099D2946FDF7B4FA0746326CD000C00FFD
:10C300009100C90F5300DB0F009301910290E019D7
:10C31000E91BD30FA74AFDF7A3FA3246C619A019A5
:10C32000A91B1546136C069A1340A34AFDF798FA09
:10C3300080490968012911D880190029864900D04F
:10C34000864900280AD07B4A121D4B699B0703D5FA
:10C3500013780B60401E521C0028F6D12E466B6CE1
:10C36000964A089C2046099D2946FDF779FA07461A
:10C370002018E91B0796B36C914AFDF771FA6D4AD4
:10C380001168012910D8C0190029734900D07349D8
:10C39000002809D0121D4B699B0703D513780B6049
:10C3A000401E521C0028F6D10798426E04236021DB
:10C3B0005C2004931A400B4600D003460693002AE3
:10C3C00000D00846079E33587E4A089C2046099DA7
:10C3D0002946FDF745FA074606983358E019E91B48
:10C3E000794AFDF73DFAC619A019A91B079A536EA1
:10C3F00076A2FDF735FA4F490968022911D2801952
:10C400000029554900D0554900280AD0494A121D33
:10C410004B699B0703D513780B60401E521C002804
:10C42000F6D10798C36C06466DA2089C2046099D6C
:10C430002946FDF715FA07462018E91B336D6B4AAC
:10C44000FDF70EFAC619A019A91B079F7B6D68A2FC
:10C45000FDF706FA8619A019A91BBB6D67A2FDF7A7
:10C46000FFF9344909680129059C11D88019002970
:10C47000394900D0394900280AD02E4A121D4B698B
:10C480009B0703D513780B60401E521C0028F6D181
:10C490000798476B5D4A974237D2032087430026AF
:10C4A000059CB00039580246049B1A43BA58082329
:10C4B0000343FB580C2505437D59009101920293DB
:10C4C00003953B1808980999514AFDF7C9F919498C
:10C4D000096801290FD800291F4900D01F490028E9
:10C4E00009D0089A4B699B0703D513780B60401E4F
:10C4F000521C0028F6D11B2E444A06D80798406BE0
:10C50000361DB10040189042CBD30798406B111AEA
:10C51000099A914201D8890800E0610200F008FC04
:10C520003C480068002800D08047FFF713FEC04653
:10C5300022224B4D48C70102F8ED00000D0A0D0AFA
:10C5400023232320455843455054494F4E2025640A
:10C55000202323230D0A00000090014000A0014089
:10C5600050433D25303858002C2045786365707461
:10C57000696F6E4E756D6265723D25640D0A00002F
:10C580002C205468726561644D6F64650D0A00006B
:10C5900052252D32643D253038580D0A0000000028
:10C5A00053503D253038580D0A00000097EE00002A
:10C5B000ADEE0000B9EE0000A1EE000056EE000066
:10C5C00065EE000074EE00007FEE00004558435F0A
:10C5D00052455455524E3D253038580D0A00000042
:10C5E000494353523D253038580D0A008AEE000069
:10C5F0005343523D253038580D0A00004343523D05
:10C60000253038580D0A0D0A0000000000F802021B
:10C610003AEE000044C70102F0B583B0344D2C68F7
:10C62000012C06D8601E8441204601F0C9FA00287A
:10C63000FAD10120EFF310810140019102D1EFF313
:10C64000108072B62B48285A2B49695A814245D02E
:10C650002A68002A01D02A4E00E0284E1F23DB0260
:10C660000293284C022A27D205E01046214AA852FC
:10C6700082B2914232D087B2B9420A4600D8621CD7
:10C68000131A21482B5218040DD0E819001D9FB22F
:10C6900001E0002F07D073699B07FAD50378336058
:10C6A0007F1E401CF5E7A242DFD902981018DDE793
:10C6B000304683B299420CD0024680B281420E4687
:10C6C00000D8661CA642F3D90298301883B299426A
:10C6D000F2D108496852B01A0B4968520B48002140
:10C6E00029540198002800D162B603B0F0BDC046BD
:10C6F00048C701020A080000080800000090014035
:10C7000000A00140FF0700000C0800000F08000017
:10C71000F0B58DB00793174600240C9409AA13C2F4
:10C7200015E006986849F3F795FDF4F75DF8C11731
:10C73000401848406549F3F7CDFC009509A806224A
:10C740003346F9F705F8BDE0002C00D5BEE1387896
:10C750007F1C25280DD0002800D1B7E10B9A511C71
:10C760000A9B9942F0D8099B9854641C0C940B9135
:10C77000EAE708940025397823390D2914D80120D7
:10C780007944097949008F44090F0F0F0F0F0F0FDC
:10C790000B0F060F0F0D05437F1CECE70820FAE78F
:10C7A0000420F8E70220F6E7387801463039002403
:10C7B000092902D9264639460BE000260A21714391
:10C7C0000E18303E791C78780246303A0A2A0F4615
:10C7D000F4D32E2817D14A1C48780146303909294C
:10C7E00005D911464F1C2538532811D96AE0002479
:10C7F0000A2161430C18303C511C50780246303AF3
:10C800000A2A0A46F4D34F1C2538532800D959E088
:10C810004000C0467844808840008744A000530010
:10C820005300530053005300530053005300530070
:10C830005300530053005300530053005300530060
:10C840005300530053005300530053005300530050
:10C850005300530053005300530053005300600033
:10C860005300530053005300530053005300530030
:10C870005300530053005300530053005300530020
:10C8800053009800530053005300530053005300CB
:10C890005300530053005300AD00B6005300600036
:10C8A00053005900530053005300590053005300E4
:10C8B0005300DE0053005300BD005300D30053006B
:10C8C000530098000C9C3FE70024744940420F003D
:10C8D000791C38780F4625385328F3D898E70799FC
:10C8E000C91D07208143086807914968F4F70AF8D1
:10C8F00000210690F3F7D8FE00280BD10B99481CB5
:10C900000A9A904206D8099A2D2353540899491C33
:10C910000C910B900798083007900698F3F764FF86
:10C920000095C2178118514009A822463346F8F7EE
:10C930000FFF0B98411C0A9A914200D9F1E6099A1F
:10C940002E2313540B910C98401C0C90E9E6079889
:10C9500002C807900096019509A8102239E00B98AB
:10C96000411C0A9A9142ADD8099A252313540B9180
:10C970000C98401C0C90A5E70B9A511C079C201D9D
:10C980000A9B994239D907909CE7079802C80790FB
:10C99000009509A82246D3E6079901C9079109998C
:10C9A0000A9A089E02E0401C002E8BD40378002BCC
:10C9B00088D00B9D6C1C9442F5D84B55761C0C9678
:10C9C0000B94F0E7079802C807900096019509A814
:10C9D0000A222346F8F75AFF74E7079B10CB102C66
:10C9E000079308D300202146401C0A09FF2911465D
:10C9F000FAD806280AD8082009E02368099CA3541D
:10CA0000089A521C0C920B9107905BE7401C069011
:10CA100009230C980B9D099905910A9E04940DE039
:10CA2000202104463046059E715506462046049C4A
:10CA3000401C15460146089100290AD45B1E069940
:10CA4000994206D26A1CB242EAD908990891002993
:10CA5000F4D50C900B950898002800D532E70126F4
:10CA6000082501E06D1E3601022DFBD2204631461D
:10CA7000F3F730FB0F28F6D80C980590099803902F
:10CA80000A9806900B9D20463146F3F723FB691C5C
:10CA9000069A914204D90899089100290CD511E011
:10CAA0000C4A125C039B5A55089A521C0D4605927B
:10CAB00011460891002905D47043241A3009102E1C
:10CAC0000646E0D205980C900B95FBE620460DB08B
:10CAD000F0BDC0463CE5000070B588B000220328D8
:10CAE00003D9D243104608B070BD7F4CC34D2A51C4
:10CAF0000F4B104EEE5081231E010123AB552860D1
:10CB00002C1962600128EDD8079300220692059245
:10CB1000049203230393029201920091411E8841E3
:10CB2000694600F0CFFC0246104608B070BDC04612
:10CB300004080000FFC0FFC0F0B583B00C4600231E
:10CB4000D943012C56DB074602910126EFF31085ED
:10CB5000354002D1EFF3108072B65849584A505C04
:10CB6000002800D0A3E056545E48115A5E48105A7F
:10CB70000196F202161A814240D832465218A24259
:10CB800040DB00930295A642354600DB25464C4922
:10CB90000818001D39462A46F3F7D8FAA642484E2F
:10CBA00004DA7919621B301DF3F7D0FA4E48305A77
:10CBB000001981B24D4A914201D94D494018029D58
:10CBC000009B4949705230464A4E805D002865D12D
:10CBD000EFF310850198054002D1EFF3108072B693
:10CBE000374A4048115A4048105A884232D1424888
:10CBF00013524FE00C46204603B0F0BD424252189B
:10CC0000A242BEDA3B4A2E4EB25C002A0CD03A4A0F
:10CC1000B25A51188AB2354CA242284C029F01D90F
:10CC2000334A8918304A02E0244C2F4A029F335578
:10CC3000B152421A89B2884202D22C488018421C52
:10CC400093B22F4801212FA200F0E8F83C46002DB6
:10CC5000D1D128E0019F9755884201D82348401C34
:10CC6000421A90B2800A01D0019882022248144FE1
:10CC70003A52386801280DD8431E9841104B591874
:10CC8000091D92B21D4B00F035FE009B002801D01B
:10CC90000B488355002D029D00D162B60748084914
:10CCA0000B54002DA7D162B6204603B0F0BD212061
:10CCB0000201044804A108A3FFF754F80E0800007D
:10CCC00048C701024EEF000074726163655F6F75C3
:10CCD0007470757400000000545241434520425561
:10CCE000535900000A08000008080000FF07000070
:10CCF00000F8FFFF0F0800000C08000049CF0000FB
:10CD000002FF00000D0A5472616365206275666659
:10CD100065722069732066756C6C2C20646973637E
:10CD2000617264732025752062797465730D0A0041
:10CD3000F0B587B00546002606960596049603963C
:10CD40000296800701D007B0F0BD019102A814211E
:10CD500026A2FCF785FD29490968012911D8002977
:10CD6000274900D0274900280BD002AA01E000285B
:10CD700007D04B699B07FAD513780B60401E521CF5
:10CD8000F5E701990029DED0204C3746B8002B5832
:10CD9000D80724D0581EA04204D31B4818181C4A98
:10CDA00090421CD802A814211AA2FCF759FD13497D
:10CDB0000968012911D80029114900D0114900281A
:10CDC0000BD002AA01E0002807D04B699B07FAD5D7
:10CDD00013780B60401E521CF5E7761C01997F1CEE
:10CDE0008F42B0D2322ED1D3ADE7C0460D0A426198
:10CDF000636B74726163653A200D0A0048C70102D3
:10CE00000090014000A00140FFFFFFFCFFFF020077
:10CE1000FEFF0100253038580D0A000081B0F0B542
:10CE2000C4B00E4607464993812000012F49085C93
:10CE3000002845D002920120050204A82946F3F7F4
:10CE40009EF9FCB20021C8430C2C3AD8721E032A6A
:10CE500037D82748005DB042084632D3F80535D5AB
:10CE60000021B8050DD404A801904018691AA20049
:10CE700022A39B582E4AFCF7F3FC0198F3F78AF99A
:10CE8000014678050ED404AF7818691AB20029A3B8
:10CE9000D218121F1368264AFCF7E2FC3846F3F753
:10CEA00079F90146029A04AE70180C46691A49AB2A
:10CEB0000393FFF72DFC01193046FFF73DFE00E01C
:10CEC000002044B0F0BC02BC01B00847FEF7E8FE09
:10CED000034604A8019007A22946FCF7C1FC01986B
:10CEE000F3F758F90146B805BDD5CAE748C70102AE
:10CEF00073FD000025313075207C2000F2EE00002B
:10CF000048EF000042EF000021EF0000ECEE0000CF
:10CF10000DEF00003BEF000034EF00002FEF0000AA
:10CF2000E5EE0000F8EE000008EF0000DDEE000086
:10CF300069EF000027EF000013EF00001AEF000078
:10CF4000FEEE000000000000F0B581B00B460120AD
:10CF5000EFF31084044002D1EFF3108172B6990F01
:10CF600007D0022001212DA2FFF758FF002C3DD150
:10CF700041E02249224D00276F54224AAB5A224AEF
:10CF8000AE5AF3189EB2F60A01D0204E9B19AB524E
:10CF9000EFF31086064002D1EFF3108372B6AA5A5F
:10CFA0001C4BEB5A934202D116482F521AE0685498
:10CFB000934201D8164B5B1C9B1A99B2890A00D088
:10CFC000830210482B52286801280BD8411E884143
:10CFD000A918091D9AB2104B00F08CFC002801D052
:10CFE00006482F54002E03D0002C04D001B0F0BD11
:10CFF00062B6002CFAD162B601B0F0BD0F08000095
:10D0000048C701020C0800000A08000000F8FFFFF2
:10D01000FF0700000808000049CF000055415254A6
:10D02000204572726F722025780D0A00B0B5044653
:10D03000FEF720F8A08A002800D0B0BD0A4D28686D
:10D04000401C2860FDF76CFD084CE063A06F0028D1
:10D0500005D0FDF765FDE8600020A067B0BD206B3E
:10D06000A8600120A067B0BDC89801020497010222
:10D0700070B5012801D9012070BD48224243734B8D
:10D080009C58A5691F218D43A5610625A5600F2524
:10D0900025629C18A27C002A05D1627C002A02D15C
:10D0A000227C002A14D06368002B11D4251D0B406C
:10D0B000012216469E400C4B1E60BFF34F8FBFF3FC
:10D0C0006F8F2B68002B03D40B409A4007490A60EE
:10D0D000002803D0012804D1092000E00820F9F736
:10D0E00063F90020A06170BD80E100E080E200E013
:10D0F000F0B585B00D460278E348C368934219D075
:10D10000446D944216D08368934203D0016D9142DE
:10D1100000D07FE09B1A591E8B410493482159434C
:10D12000032D46D14418E16900294ED01C3400205B
:10D1300020606DE09B1A5A1E93410493032D1AD16F
:10D14000039548225A438418A26B0121EFF31085FE
:10D150000D4002D1EFF3108772B6A7691026B743CE
:10D16000A761A669002E01D118342160002D00D1DD
:10D1700062B6039D0CE04821594342189169183268
:10D18000302902D0116810294CD180211160002271
:10D190004821594340180021816301628162243093
:10D1A00000210160002A33D004A82946904705B029
:10D1B000F0BD421891691832302902D01168202937
:10D1C00039D180211160002216E00395E26B01261F
:10D1D000EFF31085354002D1EFF3108172B6A169EB
:10D1E0002027B943A161A169002901D11834266023
:10D1F000002D00D162B6039D4821594340180021FB
:10D20000C163C1624163303000210160002ACBD18B
:10D2100005B0F0BD00920E4A2E329C480D490E4BCF
:10D22000FEF7A0FD10680093019098480949084A4C
:10D230000A4BFEF797FD106800930190044A2432D0
:10D2400092480449054BFEF78DFDC046A8940102A3
:10D25000C2020000CDEF0000A2EF000086EF000048
:10D26000F0B585B0049048210A464243864B9C584D
:10D27000E6690F2535409A18167C002E31D04F20D4
:10D2800040026169014200D185E0A0690421884320
:10D29000A06102202062012081076918D161D36B4F
:10D2A000EFF31084044002D1EFF3108572B6956954
:10D2B0002026B54395619569002D00D173E0104695
:10D2C0003C30002C00D162B600240460D462546368
:10D2D000303200201060002B63D004A8984705B0BE
:10D2E000F0BD0C2D5DD8C0467D442D796D00AF4456
:10D2F00067586B580658A1635858585806009569E6
:10D30000202D04D0154618352D68302D49D1156BC8
:10D31000566B3432AE4217D26669360714D564684C
:10D3200015686E1C166048431818C06A4455049866
:10D330000C4644431A19156B566B3432AE4203D275
:10D340001C5966693607EAD41268AA4229D14143BA
:10D35000585882690524A24382615A18D36B01216F
:10D36000EFF31080084002D1EFF3108472B6946995
:10D370002025AC4394619469002C02D114461834E2
:10D38000216014463C34002800D162B6002121609F
:10D39000D16251639CE70C2D00D176E7012D00D1BD
:10D3A00073E705B0F0BD15461835286010463C30CF
:10D3B000002C00D187E787E70420206205B0F0BD8C
:10D3C0000120206205B0F0BD0825256216461836FA
:10D3D0009569102D02D03568302D4BD10396566AD1
:10D3E00015462835976AB74228D1A069022188439B
:10D3F000A061936B0121EFF31080084002D1EFF39D
:10D40000108472B6039E34681027BC4334603468BD
:10D41000002C00D1316014463834002800D162B6A7
:10D420000021216029601162243200201060002B4D
:10D43000B7D052E70220206205B0F0BD2A68B242A0
:10D44000AFD262699207ACD52A68561C2E60484359
:10D450001818006A805C206004980A4642439D18B0
:10D46000AC6A6E6AB4429CD228359C5862699207B5
:10D47000EAD496E7316800900191044804A1094A72
:10D4800009A3FEF76FFCC046A89401026CEF0000F0
:10D49000756172745F6972715F68616E646C6572E8
:10D4A000000000004E0300005561727420256420C6
:10D4B000737461746520676F65732077726F6E6730
:10D4C00020256400F0B585B00E460546022804D339
:10D4D000002E02D1012005B0F0BD002D03D0012D9A
:10D4E00008D1092400E008242046F8F765FF20460B
:10D4F000FEF7F4F848216943E74A505883691F242E
:10D500000294A3438361062383600F230193036284
:10D5100057180023BB62BB63FB633B627B62FB6209
:10D520003B63317F3974727F7A74B27FBA7404932B
:10D530007B637368B268F468920022435B1E032B1E
:10D540000ED8C0467B441B795B009F44010503074E
:10D55000082304E0282302E0182300E038231A43BC
:10D56000C260C907090F72699201D2B28918B26903
:10D570009207920E8918491C8160796131690129ED
:10D5800001D122210161012D5CD831680E2959D2C7
:10D590003846123003900324002D01D0204600E0CD
:10D5A00004204C432D490E19B178F8F795FF3968DE
:10D5B000CA68802510462843C8602848005D7378F3
:10D5C0001B021818C862AA43CA60F9F719F8039831
:10D5D0000078002809D1384611300078002804D19D
:10D5E000384610300078002827D07868002815D4F5
:10D5F000032102468A431B4953588407E40EFF2641
:10D60000A640B343A5401D43555002990140012057
:10D610008840A2490860144908600EE08107C90EDD
:10D62000FF228A40019C0440083C032084430C48AC
:10D63000235893438D401D4325500120B861049821
:10D6400005B0F0BD02480349EB22034BFEF78AFB0D
:10D650006CEF0000DFEF0000BCEF0000D0E2000044
:10D660001CED00E000E400E000E100E0F0B58FB068
:10D670000E900125002900D14BE0039304910592FF
:10D68000002A00D145E00121EFF3108201910A4008
:10D6900002D1EFF3108172B64827029747437E49C3
:10D6A000CE19B5690023302D23D831461831C04634
:10D6B0007D442D796D00AF4420242626262626267B
:10D6C00026262626262626265E26262626262626C2
:10D6D00026262626262626261826262626262626F8
:10D6E000262626262626262618000223002A0CD0C7
:10D6F0000CE0402D01D0802D05D10123002A04D05B
:10D7000004E020240C60002A00D162B61D46002BE4
:10D7100002D028460FB0F0BD002575630399F16370
:10D720000499F162059931635B4CE35959691322FD
:10D73000D202114205D0062199600F211962716948
:10D740009960317C00290CD0F56109950895079501
:10D7500006950D950B9502210A91012810D01720EE
:10D760000FE0717C9A6900292CD0952002439A61C0
:10D7700028460FB0F0BD30240C60002AC5D0C5E7A4
:10D780001920049F0C907068002805D41F210840C0
:10D79000019981404148016014209861B06806A950
:10D7A000F8F79EFF0E98029941436018806861580F
:10D7B0003B4A0092091D3A46059BF9F701F82846B5
:10D7C0000FB0F0BD3436110602D580218A439A612C
:10D7D00031680025059A91422DD205955D694F214A
:10D7E0004A0215421BD1E90502D4029CFB4F0AE014
:10D7F000596833685C1C3460029C6043F74F3818EA
:10D80000C06AC1540E98214641437E18736B346B35
:10D81000A34238D234367B585D691542E3D00221E9
:10D820001962019EB10729433546EC4CEFF3108293
:10D83000324006D008E02946019EEFF310823240C4
:10D8400002D1EFF3108372B6029B4343E018836961
:10D850002024A34383618369002B05D0002A08D0CC
:10D86000C26B002A0AD154E7034618331E60002A0F
:10D87000F6D162B6C26B002A00D14AE70EA89047E3
:10D8800028460FB0F0BD2946059D019E3C46EFF3AA
:10D8900010823240D5D0D7E7A894010280E200E0A0
:10D8A000F1D0000080B5012042020249024BFFF78F
:10D8B000DDFE80BDA8AE0102A5D80000B0B582B0E3
:10D8C00079208400094D285D01A908706520800039
:10D8D0002818F3F701FD2F20C0002858291901222C
:10D8E000034BFFF7C3FE02B0B0BDC046B0A80102B3
:10D8F000BDD80000F0B591B010900126002900D1EC
:10D900009BE003930591002A00D196E00790012146
:10D91000EFF310800291084002D1EFF3108172B64C
:10D9200004924823069307994B43AC49C9188D6963
:10D930000026302D6ED80C461834AD00374602A6AE
:10D9400075593E46AF46C0461DDA000025DA000094
:10D9500029DA000029DA000029DA000029DA0000BB
:10D9600029DA000029DA000029DA000029DA0000AB
:10D9700029DA000029DA000029DA000029DA00009B
:10D9800029DA000029DA00000DDA000029DA0000A7
:10D9900029DA000029DA000029DA000029DA00007B
:10D9A00029DA000029DA000029DA000029DA00006B
:10D9B00029DA000029DA000029DA000029DA00005B
:10D9C00029DA000029DA0000BBDA000029DA0000B9
:10D9D00029DA000029DA000029DA000029DA00003B
:10D9E00029DA000029DA000029DA000029DA00002B
:10D9F00029DA000029DA000029DA000029DA00001B
:10DA000029DA000029DA00000DDA000002260028D9
:10DA10000CD00CE0402D01D0802D05D1012600282E
:10DA200004D004E010252560002800D162B6002E45
:10DA3000069D6A4F049C079802D0304611B0F0BD95
:10DA400000268E62039A8A63059A0A624C620A7CF7
:10DA5000002A0BD00C960B960A96099608960E96FD
:10DA600002220D9201282DD018202CE08A7C28312A
:10DA7000002A3BD00A68A24216D22B464343FA58EA
:10DA80005469A40710D50868441C0C60F918096A89
:10DA9000085C10601098294641437A1811462831D5
:10DAA000936A526A9342E8D3454378598169822246
:10DAB0000A438261304611B0F0BD30252560002850
:10DAC000B4D0B4E71A200F90C86808A9F8F708FE88
:10DAD000109845437A597819C068384900910599DA
:10DAE0002346F8F76DFE304611B0F0BDFB589A6939
:10DAF000140602D58024A2439A610A68002604987D
:10DB000082422ED25D694F225202154207980AD0F6
:10DB100002211962029EB10729431FE028315D6985
:10DB200015423E46F4D137465C69A40702D40699F3
:10DB30002A4E0AE00C68661C0E6006994843274E80
:10DB40003018006A005D18601098414373587118CE
:10DB50008C6A4E6AB442E1D329463E46069D1F4F69
:10DB600001E0314607985A6A002AFCD1EFF310828F
:10DB7000029B1A4002D1EFF3108372B64543781925
:10DB800083691024A34383618369002B05D0002A95
:10DB900009D0826B002A0BD14FE703461833029C51
:10DBA0001C60002AF5D162B6826B002A00D144E7DE
:10DBB00010A89047304611B0F0BDC046F1D000002B
:10DBC00048214143054842189269D20601D40020F9
:10DBD000704740584169012008407047A8940102ED
:10DBE000F0B587B001460127022505283A4600D046
:10DBF0002A4600200929014600D01146C900374AAB
:10DC000054180E210591615EFDF774FB1026A15F8B
:10DC10003846FDF76FFB1227E15F2846FDF76AFBE8
:10DC200006951425615F03200490FDF763FB0598BA
:10DC3000235EA05FE15F625F00AD07C528A2069F7B
:10DC40003846049D2946FFF7E9F820462630042689
:10DC50003146FBF77FFE2620235E2820205E2A2106
:10DC6000615E2C22A25E00900191029224A23846AD
:10DC70002946FFF7D3F827463E3738463146FBF7AB
:10DC800087FE3E20235E06983C5EB95F0622BA5EA0
:10DC900000940191029221A207462E462946FFF7E1
:10DCA000BDF856240D4D285FFBF766FE2B5F2C4612
:10DCB00021A2384631463546FFF7B0F82646583699
:10DCC0003046FBF745FE5820235EF05F00901FA210
:10DCD00038462946FFF7A2F807B0F0BDD09D0102F3
:10DCE000546F4620616E742064656C6179732025E1
:10DCF000642025642025642025640D0A00000000AE
:10DD000050446F412064656C61797320256420253F
:10DD1000642025642025640D0A00000050446F41F2
:10DD2000206761696E7320256420256420256420A6
:10DD300025640D0A0000000050446F4120616E749C
:10DD40002073706163652025640D0A0050446F41A3
:10DD500020616E676C65206F66667365747320253D
:10DD6000642025640D0A0000F0B587B015467A4B93
:10DD70001A680F24A2432F783A431A60774C23463F
:10DD80002C3B774A1A60049003462246283A1268D0
:10DD90001207FAD5734E092F029306D9754A3260DD
:10DDA00072600C2F09D175480FE0042F07D9704A13
:10DDB0003260704A7260092F06D3714805E06A48E4
:10DDC00030607060694800E06B486E4A1060EB7A22
:10DDD000FF2B039102D10020B0620AE003210B4027
:10DDE0006948C05C40220243B2620220674AFFF7E2
:10DDF00015F8029F0021384605952A460B46FBF789
:10DE000033FE06460225032161A2284601913346CE
:10DE1000FFF704F806963046FCF7FAFA0121049859
:10DE2000009108402CD13D4033D1604900283AD1BF
:10DE3000002D1ED06548A062E062206360636448E4
:10DE4000606264480860152085046E1C8E608D60D9
:10DE5000642420460F46F8F7D3FB3E603D60204621
:10DE6000F8F7CEFB281D386003215BA24E48FEF771
:10DE7000D5FF0598007BFAF7F7FE069807B0F0BDCE
:10DE80002E4605460698FCF7DBFE284635463D4003
:10DE9000CBD02E4605460698FCF7F0FA28463546C4
:10DEA00042490028C4D0424808614248486142487B
:10DEB00088611520C8614148016840220A43026018
:10DEC00007210803274B5A69824300984003101822
:10DED00058610522039842432A4803689818334E34
:10DEE000766B47780F40995C0907490EC919CA0338
:10DEF000334B33409A18C9015118324A89182B4ABA
:10DF000051632A49896B3822914382785207920ED5
:10DF1000891804220A4325498A63124B1969027938
:10DF2000019E3240C0784007C00E80181F229143E6
:10DF30000818186155204003411C216020606420AE
:10DF4000F8F75EFB204A18483146039BFEF766FF50
:10DF50001649002D8DD06DE7040400402C60004070
:10DF600000040080000600400F040F0471E9000067
:10DF70000304030400040004A2EA000040E80000D7
:10DF8000D3EB0000F093010204ED00000BF0000061
:10DF900050485920706172616D73207365747320ED
:10DFA000253038780D0A000002080000906000401B
:10DFB00012A83E009DD79B5AD579BD493402004036
:10DFC0003F0080FF40400000EDEF0000200882008D
:10DFD00002D50F00020255007577625F72785F69A3
:10DFE0006E69740D0A000000F0B581B01820FDF7CD
:10DFF00075FB1920FDF772FB002420462146F7F738
:10E00000B1FE20462146FAF7B3FD012603257F2302
:10E01000304629462A46FAF7C3FE3046FBF798F801
:10E0200002273846FBF700FD30463146FCF77CFD01
:10E0300003A238462946FEF7F1FE204601B0F0BDA6
:10E040007577625F6F70656E0D0A0000F0B581B084
:10E05000164600910446002001273946FDF738F89E
:10E06000EFF310853D4002D1EFF3108072B6272008
:10E07000400170430A21F2F72DF80246002C02D02D
:10E080000020009901E002200021FBF767F8044618
:10E09000FBF72CF9002D00D162B6204601B0F0BD8F
:10E0A00070B504460E4D29680F2001400629FAD0AC
:10E0B00029680140072912D10120EFF3108606409C
:10E0C00002D1EFF3108072B6FCF72AFDFA30A86097
:10E0D000002C01D0FAF75EFE002E00D162B670BDB2
:10E0E00000040040F0B581B01D460E460446022AE9
:10E0F00009D1012738463946FCF7EAFF009600228D
:10E10000384629460FE0174601200021FCF7E0FFC2
:10E11000012F04D1009600202946024603E0009614
:10E12000022000210A462346FBF7F8F80446FBF7D5
:10E13000DDF8204601B0F0BD7047000070B5002842
:10E1400001D0012070BD0325A9020F4802680F4BC2
:10E15000535000249460012253030D4E3360BFF3EB
:10E160004F8FBFF36F8F0B4E336003685A5084722A
:10E1700004811020F8F718F9022007A22946FEF7BB
:10E180004DFE204670BDC0464495010251E5CC1AB3
:10E1900080E100E080E200E057445420636C6F733C
:10E1A000650D0A000146012000290CD106490A7AB2
:10E1B000002A08D003208202096804488850002001
:10E1C000C86001238B5070474495010251E5CC1A79
:10E1D0002021020C01D010211046020A01D0104665
:10E1E0000839020901D01046091F820801D01046E3
:10E1F000891E420801D0881E7047081A704702E045
:10E2000008C8121F08C1002AFAD1704770470020C1
:10E2100001E001C1121F002AFBD17047000084C138
:10E22000000008C10000C03F000038410000AC41C0
:10E230000000D44128000400000008400800000845
:10E24000100804081020000000000000000000007A
:10E2500001000000FFFFFFFF0000000000000000C1
:10E2600000000000B0040000010000006009000090
:10E2700002000000C0120000030000008025000022
:10E2800004000000004B00000500000000960000A4
:10E290000600000000E100000700000000C20100CD
:10E2A00008000000008403000900000000080700C7
:10E2B0000A00000000100E000B00000000201C00EF
:10E2C0000C00000040420F000D00000080841E0082
:10E2D00059062014032145012882003241003219D9
:10E2E00000411300390300B506002D03002D020084
:10E2F0002201002201003E01002000008009EE4DB5
:10E300005048504F80096E4F58E5854F80096E4F39
:10E31000B867C14F5048D04FB867C14FE828DF4FAA
:10E320008009EE4F18EAFC4F8009EE4F58E5055082
:10E33000A4550D50F0C51450A4550D5000002110E7
:10E34000422063308440A550C660E770088129915F
:10E350004AA16BB18CC1ADD1CEE1EFF13112100207
:10E3600073325222B5529442F772D66239931883AF
:10E370007BB35AA3BDD39CC3FFF3DEE362244334D3
:10E3800020040114E664C774A44485546AA54BB5FF
:10E3900028850995EEE5CFF5ACC58DD553367226A7
:10E3A00011163006D776F6669556B4465BB77AA74F
:10E3B00019973887DFF7FEE79DD7BCC7C448E558F3
:10E3C0008668A7784008611802282338CCC9EDD99F
:10E3D0008EE9AFF9488969990AA92BB9F55AD44A47
:10E3E000B77A966A711A500A333A122AFDDBDCCBEF
:10E3F000BFFB9EEB799B588B3BBB1AABA66C877C13
:10E40000E44CC55C222C033C600C411CAEED8FFD3E
:10E41000ECCDCDDD2AAD0BBD688D499D977EB66EE6
:10E42000D55EF44E133E322E511E700E9FFFBEEF8E
:10E43000DDDFFCCF1BBF3AAF599F788F8891A98150
:10E44000CAB1EBA10CD12DC14EF16FE18010A1003A
:10E45000C230E3200450254046706760B98398932A
:10E46000FBA3DAB33DC31CD37FE35EF3B10290128A
:10E47000F322D2323542145277625672EAB5CBA5F6
:10E48000A89589856EF54FE52CD50DC5E234C324DA
:10E49000A01481046674476424540544DBA7FAB7CA
:10E4A0009987B8975FE77EF71DC73CD7D326F2362A
:10E4B0009106B01657667676154634564CD96DC916
:10E4C0000EF92FE9C899E9898AB9ABA9445865487A
:10E4D00006782768C018E1088238A3287DCB5CDB6A
:10E4E0003FEB1EFBF98BD89BBBAB9ABB754A545ACA
:10E4F000376A167AF10AD01AB32A923A2EFD0FED36
:10E500006CDD4DCDAABD8BADE89DC98D267C076C19
:10E51000645C454CA23C832CE01CC10C1FEF3EFF09
:10E520005DCF7CDF9BAFBABFD98FF89F176E367E69
:10E53000554E745E932EB23ED10EF01E3031323302
:10E54000343536373839414243444546100040009F
:10E5500080000001000200040008001010001800F4
:10E56000200030004000600080000001FFFFFFFF3E
:10E5700001FF01FFFF0101FFFF0100000200000099
:10E580000100000002000000020000000200000084
:10E59000000000001B000000000000000000000060
:10E5A000000000000000000000000000000000006B
:10E5B0000200000000000000140000000200000043
:10E5C0000700000002000000020000000000000040
:10E5D0000200000000000000140000000200000023
:10E5E0000100000002000000020000000200000024
:10E5F000000000001400000000000000FFFFFFFF0B
:10E60000FFFFFF01FFFF01FFFF01FF01FF01FFFF10
:10E61000FF0101FFFFFF01FF0101FFFF000100FFFC
:10E62000010000FF000064009E00C800E800020135
:10E6300019012C013D014C015A01660172017D0155
:10E64000870190019901A101A901B001B701BE01A3
:10E65000C401CA01D001D601DB01E101E601EB01F1
:10E66000EF01F401F801FD010102050209020D02AA
:10E670001102140218021B021F02220225022802A4
:10E680002B022E023102340237023A023D023F02CF
:10E690004202450247024A024C024F025102530213
:10E6A000560258025A025C025F026102630265026E
:10E6B000670269026B026D026F02710273027502DA
:10E6C000760278027A027C027E027F028102830255
:10E6D00084028602880289028B028C028E028F02DB
:10E6E0009102920294029502970298029A029B026A
:10E6F0009D029E029F02A102A202A302A502A602FF
:10E70000A702A902AA02AB02AD02AE02AF02B0029A
:10E71000B102B302B402B502B602B702B902BA023C
:10E72000BB02BC020000000000000000020000006C
:10E7300004000000001003EB0000000001000000D6
:10E740000100000004000000000100320000000091
:10E7500000000000000000000100000001000005B2
:10E7600000000000000000000000000001000000A8
:10E770000100003500000000010000000000000062
:10E780000400000000000020000000000100000064
:10E790000000000004000000000000D8000000009D
:10E7A0000100000000000000010000000000000661
:10E7B0000000000001000000000000000100000057
:10E7C0000200000100000000000000000000000046
:10E7D000010000000300009F000000000100000095
:10E7E0000000000001000000000000B9000000006F
:10E7F000010000000000000001000000000000AB6C
:10E80000000100FF010000FF000100FF010000FF08
:10E81000FF00000100FF00010001000000FF00FFF9
:10E8200000FF00000100FFFF00FF010000000001E9
:10E83000010000FFFFFF01FF0101000000000101D6
:10E8400000030201000005020100000103010000B5
:10E8500003030100010003010001020301000200A3
:10E860000301000202030100030203010003040389
:10E870000100040203010000000302000003030280
:10E88000000006030200010003020001030302006E
:10E890000106030200020103020002040302000257
:10E8A0000703020003030302000001070300000640
:10E8B000070300010004030001000703000104072F
:10E8C0000300010707030002000703000204070317
:10E8D0000002070703000302070300030607030003
:10E8E00004020703000406070300050104030005F2
:10E8F00002070300050607030006000703000604DD
:10E9000007030006070703000703070300070707BD
:10E9100003000802070300080607030009020703B3
:10E920000009060703000A020703000A070703009D
:10E930000B050703000C030703000C070703000D7A
:10E94000070703000E070703000E060704000E0763
:10E950000704030E070704030E070704030E070747
:10E9600004030E070704030E070704030E0707043A
:10E97000030007000202010000020200040102027B
:10E98000000701020202020002020101010202016B
:10E99000060102020305000202040200020202064E
:10E9A0000102020300010202030501020205030045
:10E9B000020204050102020204020202020702022C
:10E9C000020503010202050601020206000102021D
:10E9D000060301020202050302020206030202010B
:10E9E00006040202010607020202030402020203F5
:10E9F00007020202060702020302070202030507DA
:10EA000002020307070202040704020205010402CE
:10EA100002050107020205030702020506070202BA
:10EA200006020702020605070202070107020207A3
:10EA30000407020208010402020802070202080594
:10EA4000070202090304020209040702020A00077E
:10EA500002020A020702020A050702020A07070267
:10EA6000020B030702020B060702020C0107020257
:10EA70000C040702020D010702020E000702020E3B
:10EA8000040702020F010702020F050702020E042B
:10EA90000703030F030703030F070703030F07070A
:10EAA0000303000000020200000002020000000256
:10EAB0000200000002020000000202000000020248
:10EAC000000100020200040002020007000202012D
:10EAD0000100020201040002020107000202020317
:10EAE0000002020104010202010601020203050004
:10EAF00002020204010202030101020203030102F5
:10EB000002040101020204040102020206020202DE
:10EB100003020202020106030202020203020201D0
:10EB200002070202010407020203030302020204B5
:10EB300004020202050702020301070202030504A0
:10EB4000020204010702020403070202050603028F
:10EB5000020500070202050207020205040702027D
:10EB60000600070202060207020206050702020665
:10EB7000070702020704070202070704020208024D
:10EB80000702020805070202090107020209040739
:10EB900002020A000702020A030702020A0607022B
:10EBA000020B020702020B050702020C0107020218
:10EBB0000C050702020D020702020C010703030CF9
:10EBC000060703030D020703030E020703030E07E4
:10EBD0000703030000000202000000020200000020
:10EBE0000202000000020200030002020100000213
:10EBF00002010200020200050102020202000202FA
:10EC000003010002020201010202020401020201E8
:10EC100002020202010402020203040102020202D1
:10EC200002020202050202020002070202000407B9
:10EC300002020006070202010207020201040702A3
:10EC4000020106070202020307020202050702028E
:10EC5000030207020203040702020402070202047D
:10EC60000407020204060702020501070202050367
:10EC70000702020505070202060207020206040750
:10EC80000202060607020207040702020801070241
:10EC90000209000702020901070202090307020232
:10ECA0000A000702020A020702020B000702020B17
:10ECB000020702020C000702020B060702020C0404
:10ECC0000702020C060702020D030702030C0007ED
:10ECD00003030C020703030C050703030C070703D8
:10ECE000030D050703030D070703030D07070303C0
:10ECF0000D070703030D070703030D070703030DA4
:10ED0000070703030E0D0B07696E636C7564652FAF
:10ED1000647269766572732F6D6B5F6164632E63D5
:10ED200000696E636C7564652F64726976657273D1
:10ED30002F6D6B5F6165732E630033324B206C6FF8
:10ED40006164206361702076616C2025640D0A0087
:10ED50005854414C206C6F6164206361702076616F
:10ED60006C2025640D0A00556E65787065637465C6
:10ED70006420646D61206368616E6E656C0D0A00CD
:10ED8000696E636C7564652F647269766572732F42
:10ED90006D6B5F666C6173682E630052656C6F61AA
:10EDA000642076616C756520696D706F737369623C
:10EDB0006C650D0A00696E636C7564652F64726919
:10EDC000766572732F6D6B5F6D6973632E6300736D
:10EDD00079735F7469636B5F7374617274005265F9
:10EDE00073657420627920756E6B6E6F776E207319
:10EDF0006F757263650D0A0025313064207C200D2B
:10EE00000A00437261736865642121210D0A002D97
:10EE10002D2D2D2D2D2D2D2D2D2D2D2D2D2D2D2D22
:10EE20002D2D2D2D2D2D2D2D2D2D2D2D2D2D2D2D12
:10EE30002D2D2D2D2D2D2D0D0A00253038583A2041
:10EE4000253038582025303858202530385820258E
:10EE50003038580D0A005052494D41534B3D253032
:10EE600038580D0A00434F4E54524F4C3D25303810
:10EE7000580D0A004D53503D253038580D0A0050AA
:10EE800053503D253038580D0A0041495243523DF8
:10EE9000253038580D0A004C523D253038580D0A9F
:10EEA00000495053523D253038580D0A00785053D0
:10EEB000523D253038580D0A004E3D25642C205A0D
:10EEC0003D25642C20433D25642C20563D25640DB2
:10EED0000A0046494C45202020203A20005B53433D
:10EEE0005030335D005B464952415D005B555742EF
:10EEF0005D005B4D41435D005B4343435D005B56FA
:10EF00004552424F53455D005B53455D005B5543A1
:10EF1000495D005B5741524E5D005B494E464F5D77
:10EF2000005B4150505D005B4552524F525D005BAB
:10EF30004F535D005B424F4F545D005B544553544B
:10EF40005D005B4452565D005B5048595D00696E40
:10EF5000636C7564652F647269766572732F6D6B6F
:10EF60005F74726163652E6300257300696E636C64
:10EF70007564652F647269766572732F6D6B5F754A
:10EF80006172742E6300556E657870656374656494
:10EF90002075617274202564207374617465202566
:10EFA0006400556E657870656374656420646D6196
:10EFB000206368616E6E656C20256400506172612B
:10EFC0006D74657220696E76616C6964007561723A
:10EFD000745F646D615F63616C6C6261636B00752B
:10EFE0006172745F626175645F73657400757762E6
:10EFF0005F74785F696E69742C20706F776572201A
:10F000006C6576656C2025640D0A004F70656E2076
:10F01000414E5425640D0A006C73705F7363616C1C
:10F02000655F663332006C73705F675F6F705F6639
:10F030003332006C73705F675F6F705F696E74313D
:10F0400036006C73705F675F6F705F696E74380055
:10F050002E2E2F2E2E2F2E2E2F2E2E2F2E2E2F6495
:10F060007269766572732F6D6B5F6C73702E6300BF
:10F070004F706572616E64206164647265737320A1
:10F08000257820697320696E76616C6964004E652D
:10F090006564206174206C65617374206F6E6520F7
:10F0A0006F706572616E640052582044455343206E
:10F0B000696E646578206973206F7665722072616D
:10F0C0006E67650D0A00455420696E646578206995
:10F0D00073206F7665722072616E67650D0A002E6F
:10F0E0002E2F2E2E2F2E2E2F2E2E2F2E2E2F6472C1
:10F0F00069766572732F6D6B5F6D61632E63006D52
:10F1000061635F72785F646573635F636F6E73746E
:10F1100072756374006D61635F65745F636F6E73B6
:10F12000747275637400556E646566696E656420FB
:10F13000626974207261746520256420666F722094
:10F140006D65616E20505246206F662025640D0A61
:10F15000004D45414E2050524620706172616D65F0
:10F16000746572206572726F720D0A00436F646578
:10F170002069647820256420616E64206D65616E6D
:10F180002050524620256420636F6E666C6963745C
:10F190000D0A002E2E2F2E2E2F2E2E2F2E2E2F2EFE
:10F1A0002E2F647269766572732F6D6B5F7068794C
:10F1B0002E630001000001000000FF00FFFF0000BF
:10F1C000FFFF01000100010000FF01FF010100013C
:10F1D000000000000101FF000000010000FF00002E
:10F1E000FFFF00FF01000100FFFF00FF0101010020
:10F1F000010100000001FF00010000FF000101FF0C
:10F20000000101010000FF01000001000100FF00FA
:10F210000101FF01FFFF01000000000000010000EC
:10F22000000000FF0100000000FF00FF000000FFE1
:10F23000FF01010100000100FF01000001000001C9
:10F24000000000000000FF000000FF0000FFFF00C2
:10F250000000FF0001FF0100FF0001FF00FF0100AF
:10F260000000000001FF0000010100FF000100009C
:10F27000FFFF0100000101FF010001FF000100008C
:10F280000000FF00FF00FF00FF0101FF010001007F
:10F2900000010001000000FF010001010100000069
:10F2A000FFFFFFFF0101010000000001010100FF5D
:10F2B000FFFF01FF00000000010000FFFF00000051
:10F2C0000000FF000100010001FF0001000001003B
:10F2D000000100FF0000FF0101010000010000002B
:10F2E000FF01000100FF000000000101010101FF1A
:10F2F000010001FFFF0001FF000101FFFF00FF000F
:10F3000000000100FF010000010001FFFFFFFF00FE
:10F310000000FF000000000000FF01000001FF00EE
:10F3200001010000000101FF00000101FF00FF00DA
:10F33000FF01000101000000000000FF000100FFCC
:10F340000100FFFFFF01FF01010000FF01000101BB
:10F35000000100010001000000FF0000FF0000FFAD
:10F3600001000001FF0101000000FF01FF00FF019B
:10F370000100FF000101010100FF0000FF00010189
:10F38000000001000100000101FF00000100000079
:10F3900001FF000000FF00FFFF0100000000FF0070
:10F3A000000000FFFF0001000000000001FFFF015E
:10F3B000000000FFFF00000000FFFF010100FF014F
:10F3C00001010100FF000101000100FF0000FF0139
:10F3D00000010100000101FF0001010001FF010027
:10F3E000FF0000010000FF00FFFF000000FF01FF21
:10F3F00000000100000000FF000101FF000000000C
:10F400000001FF00FF000000000000FF0000FF01FE
:10F41000FF0101FF01000000FF00010001000101E8
:10F4200001FF0000FFFF00000100010000000100DB
:10F430000000010100FF000100FF000001FF00FFCC
:10F440000100FF000001000100000000010001FFB9
:10F45000000000000101000001000101010101FFA5
:10F460000100FF0001FF00FFFF01000101FFFF009D
:10F470000000FFFFFF000100000001000100FF018C
:10F48000FF00000000000001FF01FF00FFFF00007F
:10F490000101000000FF00000100000101FF000069
:10F4A000FFFF0101FF0000FF00000000000001FF5E
:10F4B00000000100FF000000FF010100000000FF4C
:10F4C000FFFF0101000000010001FF00FF0100003B
:10F4D000FF01000000FFFF00FF0000FFFF00FFFF33
:10F4E000010101FF0100FF0101000001FF01010016
:10F4F0000100000000000100FF00010101FF000009
:10F5000001000001000000FF00000000010000FFFA
:10F51000FF010001010001000100FF0000FF00FFEA
:10F5200001FF0001000101000000000001010000D6
:10F5300000000100000001000001FFFF0001FF01C9
:10F540000100FF000000FFFF000001FF00010000BC
:10F550000101000000010101000001000100FF00A5
:10F56000FF01FF00FF000100000100000100010198
:10F57000FFFFFFFF0100000101FFFF010001FF008D
:10F58000FFFF01000000000000FF00FF000000007E
:10F59000FF0100FFFF000001000000000001FF016B
:10F5A00001000000FF00FF0100010001FFFF00005B
:10F5B00000FF00FF0000000001FF0000000000014C
:10F5C00000000000000001FFFF01FF010100FF003B
:10F5D000010001000001FF000001010100FF010125
:10F5E00000FF00000100FF01000000010100010117
:10F5F00001FF00FFFF00010001FF00FFFF0000FF0F
:10F60000000001000000FF010100000000010001F6
:10F6100001FF01FF00000100010001FFFF0000FFEA
:10F62000FF00FF00000001000001FFFF00010101D9
:10F6300000000000010101FFFFFFFF0000000101C9
:10F64000010001FF0000000100010000010001FFB6
:10F650000101FF00FF00FF00FF000000000100FFAC
:10F66000010001FF0101000001FFFF00000100FF98
:10F670000001010000FF01000000000001FF00FF89
:10F680000100FF0001FF0100FF000000FFFF00007C
:10F69000FF000000FF00000000000001000001006A
:10F6A0000001FF000100000101FF00FF0101000057
:10F6B000FF0101000000010100FF01000001FF0047
:10F6C0000000000000FF000000FFFFFFFF0100013D
:10F6D000000001FF0001000000FF00FFFF0101002A
:10F6E000FF0100FFFF010001FF0101010101000016
:10F6F0000000FF00010001FF000000010000010107
:10F7000001FF0000FF000100000100000100FF01F7
:10F710000001000100FF0000000000FFFF000001E9
:10F7200000000000FF01FF00FFFF010000000000DB
:10F730000100FFFF00000000FF0000000001FFFFCC
:10F7400000FF000000FF01000000010000FF0101B8
:10F7500000000100010000010100FF0000FF0001A6
:10F7600001010100FF000101FF00FF01FF00000097
:10F770000101FF01000001FF0000FF0000FF000089
:10F780000001000100010001010001FF0000010172
:10F79000FF01FFFFFF0001FF000100FF000000006C
:10F7A000000001010001FF0100010000FFFF000057
:10F7B000FF0101010001000100FF00000001FF0145
:10F7C00001FF01FF0000FF000000000000FF00FF3C
:10F7D000010000000000FF010100FF000000000127
:10F7E0000000FF01FF000000FFFF00FF000001001C
:10F7F00000FF0001FF0100010100FF010100000105
:10F80000010001FF0000FF000100010100FF0001F5
:10F81000010101FF000101FFFF00000000FFFF00E8
:10F8200000000100000000FF0000FF0101FFFF00D9
:10F8300000FF01010000010000FF000000010100C5
:10F8400000FFFF00FF01FF01000000000000FF01BA
:10F85000FF000100010000000100FFFFFF000000A9
:10F86000FFFF01010001FFFF00FF0100FF0001FF9A
:10F87000010101010100010000010100000000FF81
:10F88000010001000000000100010000FF0001FF75
:10F8900000FF010000FF000100FF00010100000067
:10F8A00001000000000000000101000100FF01FF55
:10F8B00000FF0000FF000100010001010001FFFF47
:10F8C00000000100000000FF000000010000010036
:10F8D00000FF01010100FF00010000000000010025
:10F8E0000101FF0100000101FF0001FF010101FF13
:10F8F000FF00FFFF0000FF00FFFF00000001FF000E
:10F900000001FF00FF0100010000000101FFFFFFF7
:10F91000000000000101FF000000FF00010000FFE7
:10F9200001000000010001FF00FF0000000101FFD5
:10F93000010000000000010000FFFF0001FF0000C7
:10F940000000FF00FF00000000000001FFFF00FFBB
:10F95000010001FFFF0101000001FFFFFFFF0101A6
:10F96000000100000100000100FF00FF01FF00FF97
:10F970000001000100000101010000000101000080
:10F980000100FF010000FFFF000000FF000101FF78
:10F990000100FFFF01000001000000010000000065
:10F9A000010100FF000000000100FF000101010053
:10F9B00001FF00000001FF0101010000FF0100FF45
:10F9C000000000010001FF00010001000000FF0134
:10F9D0000100FF01FFFFFF00000100000101000026
:10F9E00000FF01000101000000FF01FF0101000014
:10F9F000010100010000FF00000000FF000100FF06
:10FA00000000000001FF0000FF0000FF01010101F4
:10FA10000001FF010000000100FF00010100FFFFE5
:10FA20000001FF0000010101FF01000000FF0100D3
:10FA300001010100FF000100000000FF00000101C2
:10FA40000000010000FFFFFF01FF000101FF0000B7
:10FA50000001000100FF01000100000000010000A2
:10FA6000000001FF00010001000001000000010092
:10FA70000101FFFFFF00FF010000FF010001000086
:10FA8000FF00FF00010100000000FFFF010000FF78
:10FA900001000101FF010100010000FF000101015F
:10FAA00001FFFF01FFFF01FF01010101FF01FFFF56
:10FAB000FF0101FFFF010101010101FF0101FF0140
:10FAC000000001FFFF0100FFFF0100010101010132
:10FAD000FFFF010101FFFF00FFFF0001FF01FFFF2A
:10FAE000FFFF00FF01FF01FF010001FFFF0101FF18
:10FAF00001FF0101010001010001FF01FFFFFF0102
:10FB000001010101FF01FF0101FFFF01FFFF0101F1
:10FB1000FFFFFF01FF0001010100FF01010101FFE3
:10FB200001000100FFFF0001FF0101FF01010101D0
:10FB30000101FFFF01FF01010000010101FFFF00C2
:10FB400001FFFFFFFFFF01FF0001FF01FF01FFFFBA
:10FB5000FF010101FFFF010101FFFFFF01FF01FFA5
:10FB600000FF01FFFF000101FF01FF0100FF010194
:10FB70000101010101010101FFFF01FFFF0101FF7F
:10FB80000101000101FF01FF01FFFF01FFFF010172
:10FB900001FFFFFF00FF010101FF00010000FFFF67
:10FBA000FF0101FF01FFFF00FF0101000101010151
:10FBB00001FFFF010101FF0101FFFFFF01FF01FF45
:10FBC000FF000101FFFFFF01FF010001FFFFFFFF39
:10FBD000FF0100010101FFFF01FF01FFFF01FF0124
:10FBE00001FF0101010100FF00FF0101000001FF11
:10FBF000010101FF0101FF0100FF0100FFFF01FF03
:10FC0000FFFF010101000101FF00FFFF01FF0101F2
:10FC1000FFFF00010100000101FF0101FFFFFFFFE5
:10FC2000FF010101010101FF0001FFFF01FF0101CF
:10FC3000FFFF01FF010101FFFF01010101010101BE
:10FC4000FF0101010001FF01FF00FF00FF0101FFB3
:10FC5000FFFF0100FFFFFF010100FF01FF01FF01A6
:10FC600001FFFF010100FFFF000101FF0000FFFF96
:10FC70000101FF0101FF01FFFF0101010101FFFF80
:10FC8000FF010101FF01FF0001FF01FF0100010170
:10FC9000010101FF010101FF010101FF0100FFFF5F
:10FCA000FFFFFFFF0101FF0101FF0100FFFFFFFF59
:10FCB00001FF01FF00010001FF010101FFFF01FF42
:10FCC000010100010101FFFF0101FF00010100002E
:10FCD000FFFF0101FFFF010101FF01FFFFFFFFFF28
:10FCE000FF00010101FF0101010101FFFF01FF010F
:10FCF00001FFFFFF01FF01FFFFFF01FF0100FF0107
:10FD0000FFFF00010001FF0101FF01010001FF01F0
:10FD1000FFFF000101010101FF01010101010101DA
:10FD200001010101FFFFFF01FF0101FFFF010100D0
:10FD300000FF01FF0100FF01FF00FF0101FFFF01C4
:10FD40000101FF01010100FFFF000101FF01FF01AF
:10FD5000FF00FFFFFF0101FF00FFFFFFFF010101A7
:10FD600001FF01FF000100FF01FF0101FF0101FF91
:10FD7000FF01FF0400000404040404040404000060
:10FD8000A0FD00000890010250050000080B0000D3
:10FD900098FF0000589501029C3A00000EE2000016
:10FDA0005152033280420137010101000F013375C6
:10FDB000B1820142013420A107420342144926B80E
:10FDC0000300900050084202C203001515C0C1C2D2
:10FDD000C3C4C5C6C7C8C9CACBCCCDCECF000101EC
:10FDE000014B01800305090203020501330203658B
:10FDF00009020301420257140019412717901D07F9
:10FE000006050403020100F29798DDC89D5CB81C4A
:10FE1000C0DEA7DB615BCA01020003524048051047
:10FE20000406010001522D2C280004007C007B01F7
:10FE300005020308FF5B0F010065F901417B07071D
:10FE4000010160002000881333E0536420ACFF50B0
:10FE50001B0D070E080E080E080E080C030D050BEF
:10FE6000050D070D070D070D0701012E0104020006
:10FE70004003FFFF7F00FFFF7F0816FFFFFF00FF2B
:10FE8000FFFF3A010001000A00010106401E400583
:10FE900012051200051504020102030102400402CA
:10FEA000010303020C0E0900087A023241342800D3
:10FEB0002A820303455006C570014013E6207001F5
:10FEC00040144C07001000D6FF00B000500B420257
:10FED000820345FFFF0F203204420832010455100F
:10FEE000000134B4000305502000500746010028EB
:10FEF00000049901020100FFFFFFFF37909001020B
:10FF0000D3EB0051151EC135BF80F3E2BDC0B46410
:10FF1000BF871699BDAD178DBF941799BD33A876CD
:10FF2000BFC4780DBD2BC162BA0CB0AFBEA9F6E953
:10FF3000BAFC567BBE07254CBBEC8823BE5DC0CB0C
:10FF4000BB0CCE20BD7BA095BCD40F3A3E2D5EAC41
:10FF5000BD5913073F6401004242094403000632C1
:10FF600001451001400FC20E42014201C2030210BE
:10FF700003520145900140184204023D0545A0018D
:10FF800040194206024007830232454001400DC23B
:08FF9000010000000000000068
:020000040001F9
:1002F000A5A54B4D0000001000000002AAAA5A7FDD
:10030000F0020100000000000200000000000000F8
:1003100000000000000000000000000000000000DD
:1003200000000000000000000000000000000000CD
:1003300088030100000000000A56656E646F7209B0
:100340003A204D4B53454D490A43686970093A209C
:100350004D4B383030300A44617465093A2041759C
:100360006720313620323032350A56657273696F34
:100370006E093A2056302E362E3200000000000062
:08038000000000000000000075
:04000005000000C136
:00000001FF
